:020000040000FA
:0400000007EF00F016
:1000080075827CED4EF065EF56F066C0D9FF67C08B
:10001800DAFFDE6ADD6A68C00BF086EC51F00BC0CF
:10002800B6F00CC0B7F00001B7BF0B0CD890B635CE
:10003800D96EB735DA6EA00ED926010EDA22DECFD8
:10004800D0F0DDCFD1F0D051D11101E10C0C66C058
:10005800D9FF67C0DAFFD0C0DEFFD1C0DDFFD0C056
:10006800D9FFD1C0DAFFDF5012E020EE01F0D05105
:10007800D926D151DA22DF50ECEC62F00001C26FD0
:10008800C2B105D06950D8A4C2A5000C0A0CD0C0D2
:10009800D9FFD1C0DAFFDF6A20EE01F0D051D926AE
:1000A800D151DA22B6C0DFFF20EE01F0D051D926B7
:1000B800D151DA22DF5004EC4DF00001C26FC2B119
:1000C800030C695002E0C2B50A0CC96BCA6BCB6B52
:1000D800CC6BD0C044F0D1C045F0466A476A486A44
:1000E800496A00EC46F00001CF6FCF0501E0D4D09B
:1000F800CD6BCE6BCE5105E1040ECD5D01E390D002
:1001080001D08ED0CDC080F0CEC081F0803B813B45
:10011800F00E811780510F0B8113F00E8017D0C09D
:1001280082F0D1C083F08051822781518323EC0E65
:100138008225C36F010E8321C46F20EE04F0C351E2
:10014800D926C451DA22DF5005E1A86BA96BAA6B46
:10015800AB6B55D020EE09F0C351D926C451DA2231
:10016800DF50816F806B20EE0AF0C351D926C4514D
:10017800DA22DF50826F82C083F0846B856B866BD6
:1001880084C086F083C085F0846B836B20EE0BF00F
:10019800C351D926C451DA22DF50876F87C088F04F
:1001A800896B8A6B8B6B88C08BF08A6B896B886BC9
:1001B800835188118C6F845189118D6F85518A11F3
:1001C8008E6F86518B118F6F80518C11906F81517A
:1001D8008D11916F000E8E11926F000E8F11936F1B
:1001E80020EE08F0C351D926C451DA22DF5090110D
:1001F800A86F9151A96F9251AA6F9351AB6FCD51CE
:10020800040DF350980FD96EDA6AA8C0DEFFA9C0B2
:10021800DEFFAAC0DEFFABC0DEFFCD4BCE2B6AD718
:10022800CD6BCE6BCD51CE1103E0CD07D8A0CE0754
:10023800CD51040DF350980FD96EDA6ADECFC9F0AC
:10024800DECFCAF0DECFCBF0DECFCCF0C951CA1179
:10025800CB11CC1105E1000EAD6F020EAC6F11D0C1
:10026800D0C044F0D1C045F0C9C046F0CAC047F07C
:10027800CBC048F0CCC049F000EC46F00001AC6FB0
:10028800AD6BACC0CFF0CF5107E0CD4BCE2BCE51EC
:1002980003E1040ECD5DCCE3030ECF1901E1010C9F
:1002A800CF5101E00D0C20EE3AF0D051D926D151B2
:1002B800DA22DF50816F806B20EE39F0D051D926D9
:1002C800D151DA22DF508013020E8119801101E02A
:1002D8000D0C20EE45F0D051D926D151DA22DF504D
:1002E800816F806B20EE44F0D051D926D151DA22AB
:1002F800DF50801380C0C5F081C0C6F0C76BC86BE3
:10030800C551C611C711C81155E120EE53F0D0519F
:10031800D926D151DA22DF50816F806B20EE54F05C
:10032800D051D926D151DA22DF50826F82C083F0B2
:10033800846B856B866B84C086F083C085F0846B84
:10034800836B20EE55F0D051D926D151DA22DF50F7
:10035800876F87C088F0896B8A6B8B6B88C08BF03E
:100368008A6B896B886B835188118C6F84518911D2
:100378008D6F85518A118E6F86518B118F6F8051C9
:100388008C11906F81518D11916F000E8E11926FAB
:10039800000E8F11936F20EE52F0D051D926D15113
:1003A800DA22DF509011C56F9151C66F9251C76F15
:1003B8009351C86F20EE16F0D051D926D151DA22C8
:1003C800C5C0DEFFC6C0DEFFC7C0DEFFC8C0DEFF97
:1003D80020EE3EF0D051D926D151DA2210EE03F0AA
:1003E800D051E126D151E222DFCFE7FF20EE03F022
:1003F800D051D926D151DA22DE040AE020EE03F0EA
:10040800D051D926D151DA22020EDE1801E00D0CA6
:10041800C5C00BF0C6C00CF0C7C00DF0C8C00EF0C8
:1004280020EE03F0D051D926D151DA22DF500F6ED9
:10043800106A116A126A56EC5BF00BC0C5F00CC06A
:10044800C6F00DC0C7F00EC0C8F020EE3BF0D0518A
:10045800D926D151DA2210EE02F0D051E126D1513D
:10046800E222DFCFE7FF20EE02F0D051D926D151AA
:10047800DA22DF50D8B40D0C20EE02F0D051D92684
:10048800D151DA22DF50806F20EE02F0D051D92608
:10049800D151DA22DF50816F8105801501E00D0C02
:1004A80020EE40F0D051D926D151DA22DF50816FA9
:1004B800806B20EE3FF0D051D926D151DA22DF509F
:1004C800801320EE08F0D051D926D151DA2280C00D
:1004D800DEFF81C0DDFF20EE08F0D051D926D151D2
:1004E800DA22DF50806F0F0E801701E00D0C20EE2E
:1004F80042F0D051D926D151DA22DF50816F806B7A
:1005080020EE41F0D051D926D151DA22DF508013A4
:1005180080C0BAF081C0BBF0BC6BBD6BBA51BB11D7
:10052800BC11BD1155E120EE4FF0D051D926D15163
:10053800DA22DF50816F806B20EE50F0D051D9263F
:10054800D151DA22DF50826F82C083F0846B856BD1
:10055800866B84C086F083C085F0846B836B20EE45
:1005680051F0D051D926D151DA22DF50876F87C098
:1005780088F0896B8A6B8B6B88C08BF08A6B896B70
:10058800886B835188118C6F845189118D6F8551C7
:100598008A118E6F86518B118F6F80518C11906FDD
:1005A80081518D11916F000E8E11926F000E8F1177
:1005B800936F20EE4EF0D051D926D151DA22DF5078
:1005C8009011BA6F9151BB6F9251BC6F9351BD6F2F
:1005D80020EE3CF0D051D926D151DA22DF50806F7D
:1005E80020EE3DF0D051D926D151DA22DF50816F6B
:1005F8008051B86F81C0B9F0B851B91101E10D0C43
:1006080020EE08F0D051D926D151DA22DECF80F081
:10061800DDCF81F0040E826FD89081338033822F32
:10062800FBD7B8518025836FB9518121846F856BC1
:10063800D8B0852B866BC5518325B26FC6518421EE
:10064800B36FC7518521B46FC8518621B56FB251B8
:10065800BA5DB351BB59B451BC59B551BD5901E24A
:100668000D0CB251BA5D0B6EB351BB590C6EB4513F
:10067800BC590D6EB551BD590E6E20EE02F0D05129
:10068800D926D151DA22DF500F6E106A116A126A28
:10069800D0EC5CF00BC0BEF00CC0BFF00DC0C0F0D9
:1006A8000EC0C1F00001BE51BF11C011C11101E15E
:1006B8000D0C010ECF6FC151C01105E1F60EBE5DE4
:1006C8000F0EBF5902E3020ECF6FC151C01105E1F1
:1006D800F60EBE5DFF0EBF5902E3030ECF6F020E8A
:1006E800BE25806F000EBF21816F000EC021826F72
:1006F800000EC121836F20EE12F0D051D926D151BE
:10070800DA2280C0DEFF81C0DEFF82C0DEFF83C048
:10071800DEFF20EE1AF0D051D926D151DA22C9C015
:10072800DEFFCAC0DEFFCBC0DEFFCCC0DEFFB851A3
:10073800C925806FB951CA21816F000ECB21826F04
:10074800000ECC21836F20EE1EF0D051D926D15156
:10075800DA2280C0DEFF81C0DEFF82C0DEFF83C0F8
:10076800DEFFB251C925806FB351CA21816FB451E0
:10077800CB21826FB551CC21836F20EE26F0D0516A
:10078800D926D151DA2280C0DEFF81C0DEFF82C0C7
:10079800DEFF83C0DEFF030ECF1901E08CD020EE10
:1007A80008F0D051D926D151DA22DE50DE1001E00E
:1007B8000D0C20EE5BF0D051D926D151DA22DF5052
:1007C800816F806B20EE5CF0D051D926D151DA22AE
:1007D800DF50826F82C083F0846B856B866B84C028
:1007E80086F083C085F0846B836B20EE5DF0D0517A
:1007F800D926D151DA22DF50876F87C088F0896BFC
:100808008A6B8B6B88C08BF08A6B896B886B835182
:1008180088118C6F845189118D6F85518A118E6F63
:1008280086518B118F6F80518C11906F81518D1172
:10083800916F000E8E11926F000E8F11936F20EE44
:100848005AF0D051D926D151DA22DF509011946F45
:100858009151956F9251966F9351976F20EE22F0B8
:10086800D051D926D151DA2294C0DEFF95C0DEFFDF
:1008780096C0DEFF97C0DEFF20EE12F0D051D926D9
:10088800D151DA22DECF80F0DECF81F0DECF82F0E8
:10089800DECF83F0020ED8908037813782378337D6
:1008A800E82EF9D780C0AEF081C0AFF082C0B0F0BA
:1008B80083C0B1F0B7D020EE08F0D051D926D1517D
:1008C800DA22DE50DE1001E10D0C20EE1EF0D051D0
:1008D800D926D151DA22DECF80F0DECF81F0DECF0B
:1008E80082F0DECF83F0C5518025846FC651812107
:1008F800856FC7518221866FC8518321876F20EE8B
:1009080022F0D051D926D151DA2284C0DEFF85C029
:10091800DEFF86C0DEFF87C0DEFF020ECF196BE068
:1009280020EE12F0D051D926D151DA22DECF80F054
:10093800DECF81F0DECF82F0DECF83F0010E8015AE
:10094800846F856B866B876B20EE12F0D051D926A9
:10095800D151DA22DECF88F0DECF89F0DECF8AF0FF
:10096800DECF8BF0030E8803F3CF8CF0F4CF8DF03D
:100978008E6B8F6B8903F3508D27F4508E23000EF6
:100988008F238803F3508D27F4508E23000E8F2376
:10099800030E8A03F3508E27F4508F23000E890329
:1009A800F3508E27F4508F23000E8803F3508E27C0
:1009B800F4508F23030E8B03F3508F27000E8A0306
:1009C800F3508F27000E8903F3508F27000E8803FA
:1009D800F3508F27D8908F338E338D338C338451D7
:1009E8008C25AE6F85518D21AF6F86518E21B06FEA
:1009F80087518F2116D020EE12F0D051D926D1512F
:100A0800DA22DECF80F0DECF81F0DECF82F0DECFDB
:100A180083F0D8908035AE6F8135AF6F8235B06F77
:100A28008335B16FFF0EAE25806F010EAF21816F48
:100A3800000EB021826F000EB121836F0A0E05D01F
:100A4800D8908333823381338033E82EF9D720EE70
:100A580016F0D051D926D151DA228051DE5C81516D
:100A6800DE588251DE588351DE5801E20D0C20EE2B
:100A78000EF0D051D926D151DA22DE68DE68DE6860
:100A8800DD68DD52DD5210EE0AF0D051E126D15179
:100A9800E222DECFE6FFDECFE6FFDECFE6FFDECFE7
:100AA800E6FF20EE05F0D051D926D151DA22800E8A
:100AB800DF6E030ECF1901E0D3D120EE5FF0D051E5
:100AC800D926D151DA22DF50816F806B20EE5EF09B
:100AD800D051D926D151DA22DF50801380058111F7
:100AE80001E0BED1D0C039F0D1C03AF0C9293B6E7F
:100AF800000ECA213C6E000ECB213D6E000ECC21AB
:100B08003E6E5BEC59F0000901E0AAD1000120EE2D
:100B180005F0D051D926D151DA22DF6A22EE2DF024
:100B2800D051D926D151DA22DF50816F806B22EE65
:100B38002CF0D051D926D151DA22DF508013550E2E
:100B4800801903E1AA0E8119D8A48AD120EE2FF0CA
:100B5800D051D926D151DA22DF50816F806B20EE37
:100B680030F0D051D926D151DA22DF50826F82C0BD
:100B780083F0846B856B866B84C086F083C085F0B8
:100B8800846B836B20EE31F0D051D926D151DA2213
:100B9800DF50876F87C088F0896B8A6B8B6B88C042
:100BA8008BF08A6B896B886B835188118C6F8451A9
:100BB80089118D6F85518A118E6F86518B118F6FB8
:100BC80080518C11906F81518D11916F000E8E1193
:100BD800926F000E8F11936F20EE2EF0D051D92610
:100BE800D151DA22DF509011946F9151956F925143
:100BF800966F9351976F520E941909E1520E9519F9
:100C080006E1610E961903E1410E9719D8A428D17F
:100C180022EE13F0D051D926D151DA22DF50816F5C
:100C2800806B22EE14F0D051D926D151DA22DF5050
:100C3800826F82C083F0846B856B866B84C086F07C
:100C480083C085F0846B836B22EE15F0D051D926D2
:100C5800D151DA22DF50876F87C088F0896B8A6BA1
:100C68008B6B88C08BF08A6B896B886B835188117A
:100C78008C6F845189118D6F85518A118E6F8651C1
:100C88008B118F6F80518C11906F81518D11916FE5
:100C9800000E8E11926F000E8F11936F22EE12F0DC
:100CA800D051D926D151DA22DF509011946F915149
:100CB800956F9251966F9351976F720E941909E13F
:100CC800720E951906E1410E961903E1610E971906
:100CD800D8A4C6D022EE17F0D051D926D151DA22A5
:100CE800DF50816F806B22EE18F0D051D926D15198
:100CF800DA22DF50826F82C083F0846B856B866B4B
:100D080084C086F083C085F0846B836B22EE19F073
:100D1800D051D926D151DA22DF50876F87C088F0A9
:100D2800896B8A6B8B6B88C08BF08A6B896B886B3D
:100D3800835188118C6F845189118D6F85518A1167
:100D48008E6F86518B118F6F80518C11906F8151EE
:100D58008D11916F000E8E11926F000E8F11936F8F
:100D680022EE16F0D051D926D151DA22DF50901157
:100D7800946F9151956F9251966F9351976F20EEA2
:100D88000EF0D051D926D151DA2294C0DEFF95C099
:100D9800DEFF96C0DEFF97C0DEFF22EE1BF0D051CB
:100DA800D926D151DA22DF50816F806B22EE1CF0F8
:100DB800D051D926D151DA22DF50826F82C083F018
:100DC800846B856B866B84C086F083C085F0846BEA
:100DD800836B22EE1DF0D051D926D151DA22DF5093
:100DE800876F87C088F0896B8A6B8B6B88C08BF0A4
:100DF8008A6B896B886B835188118C6F8451891138
:100E08008D6F85518A118E6F86518B118F6F80512E
:100E18008C11906F81518D11916F000E8E11926F10
:100E2800000E8F11936F22EE1AF0D051D926D151AE
:100E3800DA22DF509011946F9151956F9251966F0D
:100E48009351976F20EE0AF0D051D926D151DA226A
:100E580094C0DEFF95C0DEFF96C0DEFF97C0DEFFC0
:100E6800D0C0D9FFD1C0DAFFCFC0DFFF01019E4B50
:100E78009F2B000120EE06F0D051D926D151DA225D
:100E88009EC1DEFF9FC1DDFF000C0C6A0B6A96EC69
:100E980062F00F0B0101E86FAB6B070E966E010E47
:100EA800E96FB56B0F0EC16E926893689468948E63
:100EB800929092928982020EE76FE5EC61F092942B
:100EC800898492988998929E899E95689368370E2E
:100ED8000001806FF40E816FA40E826FFF0E836F86
:100EE8008A0E846FFE0E856F050E866FFF0E876F64
:100EF800B7EC62F07DEC62F017D0300E0001806F25
:100F0800FE0E816F82CF82F0836BB7EC62F0150E14
:100F18000101E46F4B0EE36FBE0EE82EFED7E32F00
:100F2800FCD7E42FFAD700F082B2E7D72FEC53F0C2
:100F38000101E86FD20E0001806FFA0E816FE8C1DF
:100F480082F0836BB7EC62F00400150E0101E46FC8
:100F58004B0EE36FBE0EE82EFED7E32FFCD7E42F2F
:100F6800FAD700F0CD929D90CF0ECD16CD8ECD80C4
:100F7800F286F180F288F19CF28E8AEC5EF089921A
:100F8800899423EC55F023EC55F0000E0B6E340ECB
:100F98007FEC5FF0200E0F6EFF0E106E1CEC5CF005
:100FA800A40E0F6EFF0E106E1CEC5CF0000E0B6EA4
:100FB800390E7FEC5FF08980040046EC41F01AECB2
:100FC8004BF0A0EC57F0000E0B6E800E7FEC5FF03C
:100FD8000101E8510F0D8E0EF3240F6E0C0EF42054
:100FE800106E1CEC5CF0725001E1F2D0F30E0001BF
:100FF800806FFC0E816FB7EC62F044EC5DF00FC0BF
:101008004CF410C04DF411C04EF412C04FF404015A
:101018004C514D114E114F1117E1300E0001806FE8
:10102800FB0E816F4CC482F04DC483F04EC484F033
:101038004FC485F0B7EC62F00A0E0E6E000E0F6A10
:10104800106A116A08EC5FF00401506B516B51BFD4
:1010580005D0515119E1040E505D16E2D90E000178
:10106800806FFF0E816F4C0E04015025D96E040E5F
:101078005121DA6EDF500001826F836BB7EC62F0AA
:101088000401504B512BE3D7DC0E0001806FFB0E9F
:10109800816FB7EC62F0BE0E0001806FF90E816FB0
:1010A800B7EC62F022EE00F000EECAF01F0EDBCFC4
:1010B800EBFFE806FCE2D10E0001EA6FFF0EEB6FD2
:1010C80081EC42F0CAC08CF1CBC08DF1CCC08EF15E
:1010D800CDC08FF101018C518D118E118F1178E0E7
:1010E800A40E0001806FF90E816F8CC182F08DC152
:1010F80083F08EC184F08FC185F0B7EC62F0000EEA
:101108000001A36F020EA46F8CC1E4F18DC1E5F15B
:101118008EC1E6F10101E36B000EE3250001A56F26
:10112800010E0101E4210001A66F000E0101E52175
:101138000001A76F000E0101E6210001A86F9EECD7
:1011480015F0000E626E020E636E8E0E646E0A0E4D
:10115800656E676A080E666E480E686E040E696EE4
:1011680088EC18F00401526B536B53BF05D05351F0
:1011780019E1080E525D16E2D50E0001806FFF0ED0
:10118800816F8E0E04015225D96E0A0E5321DA6E34
:10119800DF500001826F836BB7EC62F00401524BA1
:1011A800532BE3D72AEE8EF0DF50406F416B426B32
:1011B800436BEA0E0001806FFD0E816F40C482F020
:1011C80041C483F042C484F043C485F0B7EC62F0B4
:1011D8000101B5AF13D0946889928982150E010177
:1011E800E46F4B0EE36FBE0EE82EFED7E32FFCD75D
:1011F800E42FFAD700F016EC4CF0EED7E9510CE0EA
:10120800130E0001806FFD0E816FB7EC62F0020EC5
:101218000101AF6F220E0BD0030E0001806FFD0E8F
:10122800816FB7EC62F0010E0101AF6F040EAE6F73
:101238000401466B476B546B899E000E566F010E76
:10124800556F56BF05D056516BE1040E555D68E2E7
:101258000F0E5503F3CFE3F1F4CFE4F15603F35047
:101268000101E4277E0EE3250B6E0D0EE4210C6EC2
:1012780007EC60F00C5003E1030E0B5C4DE3720EBB
:101288000001806FFD0E816F0F0E04015503F3CF2F
:10129800E3F1F4CFE4F15603F3500101E4277E0EA5
:1012A800E3250001826F0D0E0101E4210001836F27
:1012B800B7EC62F055C4E3F156C4E4F1050ED890DA
:1012C8000101E337E437E82EFAD7000EE3250001E1
:1012D800D26F020E0101E4210001D36F0F0E040149
:1012E8005503F3CFE5F1F4CFE6F15603F3500101CE
:1012F800E6277E0EE5250001D46F0D0E0101E621DB
:101308000001D56F030ED66FA1EC1DF004014A6FE2
:101318004B6B4A5131EC5FF00401554B562B91D77A
:10132800899E000E0B6EC00E7FEC5FF035EC62F00C
:10133800000E0B6EC00E7FEC5FF0800E0F6EFF0E7E
:10134800106E1CEC5CF017D181A89394F2EC62F05B
:101358000B500401456F455101E1E4D054C444F4F5
:10136800570E0B6E040E0C6ECDEC5AF00401546F40
:1013780057B9549F0E0E0001806FFF0E816F54C441
:1013880082F0836B0401010E57A9000E0001846FDF
:10139800856BB7EC62F0040157A925D0600E54198B
:1013A80022E15F0E44191FE16E0E0001806FFF0EEF
:1013B800816FB7EC62F00101E7832AEE8EF0AFC1CE
:1013C800DFFF2AEE8FF0AEC1DFFF8984656A020E67
:1013D800646EDCEC44F08994E793716A55EC62F032
:1013E8000401546BC8D00101E95147E00401575189
:1013F800100B0001C96F000ECA6F04015451AFEC05
:1014080043F0C9C058F4CAC059F4080E0401581969
:10141800591101E100F0070E04015819591102E1B0
:1014280059EC5CF004015805591102E190EC55F0B3
:10143800020E04015819591102E119EC49F0030E82
:1014480004015819591106E104EC20F0E1C046F4F2
:10145800E2C047F4050E04015819591106E175EC6C
:101468003AF0F0C046F4F1C047F4090E04015819E7
:10147800591155E10AEC59F052D004015751100B9B
:101488005A6E000E5B6E545132EC29F05AC058F473
:101498005BC059F4070E04015819591102E195EC83
:1014A8005CF0020E04015819591102E1A9EC5DF033
:1014B80004015805591102E13CEC12F0030E040135
:1014C8005819591102E19DEC3EF0040E0401581917
:1014D800591102E128EC60F0050E04015819591160
:1014E80002E14FEC35F0060E04015819591102E1DA
:1014F800A2EC62F0080E04015819591102E13DEC02
:101508001BF0090E04015819591102E121EC37F0BA
:101518000A0E04015819591102E132EC54F0010184
:10152800B06B29D02FEC53F00101AB6FAC5123E025
:10153800E851AB1920E0898E000E0B6EC00E7FECCF
:101548005FF035EC62F0000E0B6EC00E7FEC5FF0C2
:10155800BA0E0F6EFE0E106E1CEC5CF0ABC1E8F11B
:10156800CB0E0001806FFB0E816FE8C182F0836BA8
:10157800B7EC62F032D082B230D0050E04014619C1
:1015880047112BE0E1D6300E0001806FFE0E816F0F
:1015980082CF82F0836BB7EC62F0150E0101E46F25
:1015A8004B0EE36FBE0EE82EFED7E32FFCD7E42FD9
:1015B800FAD700F00400000E0B6EC00E7FEC5FF04F
:1015C80035EC62F0000E0B6EC00E7FEC5FF0280E5B
:1015D8000F6EFF0E106E1CEC5CF082B2D4D7150EA5
:1015E8000101E46F4B0EE36FBE0EE82EFED7E32F2A
:1015F800FCD7E42FFAD700F0000EECEC62F0010102
:10160800AA6FDF0E0001806FFB0E816FAAC182F006
:10161800836BB7EC62F0150E0101E46F4B0EE36FBC
:10162800BE0EE82EFED7E32FFCD7E42FFAD700F042
:10163800899489920001D26BD36BDE0ED46FFB0EB6
:10164800D56FD66BA9EC59F0B7D45B6E5A6A2CD318
:101658005B5015E1FE5113E08C0E806FFB0E816F1D
:10166800CFCF82F0836BCECF84F0856BB7EC62F07E
:101678005A6A0101996B0A0EC4D0899087D3020E69
:101688005B1813E1FE5111E0020E806FFB0E816FB3
:10169800CFCF82F0836BCECF84F0856BB7EC62F04E
:1016A8005A6A0101996B140EACD01F0E5B6446D0C8
:1016B800300E5B6043D0FE5141E05B50E00F736E2B
:1016C800750E806FF80E816FCFCF82F0836BCECF0F
:1016D80084F0856B73C086F0876BB7EC62F05A6A4A
:1016E8000F0E731805E1A6C16BF00101A66B99D224
:1016F8007350200D0A0EF324D96E020EF420DA6E10
:10170800DE50DE10DE10DE1003E0030E736489D2B3
:10171800010E6B6E7350140D130EF324D96E010E67
:10172800F420DA6E7350140D130EF324E16E010EDB
:10173800F420E26EE7500409DF6E73D23F0E5B645B
:101748002AD0500E5B6027D0FE5125E07350140D4F
:10175800000EF324D96E010EF420DA6E5B50C00F30
:10176800DF6EDD0E806FF70E816FCFCF82F0836B57
:10177800CECF84F0856B7350140D000EF324D96E10
:10178800010EF420DA6EDF50866F876BB7EC62F0DB
:101798005A6A6B6A46D2310E5B1807E1FE5105E0C2
:1017A8000C0E0101996F1D0E6AD2340E5B1813E1FD
:1017B800FE5111E0A20E806FFB0E816FCFCF82F039
:1017C800836BCECF84F0856BB7EC62F00101986B28
:1017D800996B5A6A52D7350E5B1815E1FE5113E022
:1017E800700E806FF90E816FCFCF82F0836BCECFF2
:1017F80084F0856BB7EC62F05A6A0D0E0101996F9F
:10180800AC0E986F3AD7370E5B1808E1FE5106E028
:1018180089800E0E0101996F750E31D20D0E5B187D
:1018280017E1FE5115E05A6A020E0101996FBC0ECC
:10183800986F89903A0E0001806FF90E816FCFCFB3
:1018480082F0836BCECF84F0856BB7EC62F09ED2CA
:10185800100E5B1807E1FE5105E0030E0101996FB8
:10186800E90E0DD2180E5B1807E1FE5105E0070ED0
:101878000101996F090E03D23B0E5B1807E1FE5177
:1018880005E00E0E0101996F7E0EF9D13E0E5B1830
:1018980007E1FE5105E00F0E0101996F3D0EEFD1F2
:1018A800E80E806FF80E816FCFCF82F0836BCECFBA
:1018B80084F0856B5BC086F0876BB7EC62F066D20C
:1018C8007350140D010EF324D96E010EF420DA6E54
:1018D8005BC0DFFF030E0101996FEA0ED0D1735090
:1018E800140D020EF324D96E010EF420DA6E5BC0DB
:1018F800DFFF030E0101996FEB0EC1D17350140D78
:10190800030EF324D96E010EF420DA6E5BC0DFFFFC
:10191800030E0101996FEC0EB2D17350140D040E31
:10192800F324D96E010EF420DA6E5BC0DFFF030EDC
:101938000101996FED0EA3D17350140D050EF32418
:10194800D96E010EF420DA6E5BC0DFFF030E0101D1
:10195800996FEE0E94D17350140D060EF324D96EC0
:10196800010EF420DA6E5BC0DFFF7350140D060E13
:10197800F324D96E010EF420DA6EDF50A66FA6C0EC
:10198800A7F0A86BA96BAA6BA9C0AAF0A8C0A9F078
:10199800A7C0A8F0A76B7350140D050EF324D96ED9
:1019A800010EF420DA6EDF50AB6FABC0ACF0AD6B5C
:1019B800AE6BAF6BADC0AFF0ACC0AEF0AD6BAC6BA7
:1019C8007350140D040EF324D96E010EF420DA6E50
:1019D800DF50B06FB0C0B1F0B26BB36BB46BB1C0D5
:1019E800B4F0B36BB26BB16B7350140D030EF324E8
:1019F800D96E010EF420DA6EDF50B125B56F000EF6
:101A0800B221B66F000EB321B76F000EB421B86FC4
:101A1800AC51B525B96FAD51B621BA6FAE51B721EA
:101A2800BB6FAF51B821BC6FA751B925BD6FA85185
:101A3800BA21BE6FA951BB21BF6FAA51BC21C06F8B
:101A48007350140D070EF324D96E010EF420DA6ECC
:101A5800BDC0DEFFBEC0DEFFBFC0DEFFC0C0DEFF10
:101A6800FB0E806FF60E816FCFCF82F0836BCECFE7
:101A780084F0856B7350140D070EF324D96E010E94
:101A8800F420DA6EDECF86F0DECF87F0DECF88F086
:101A9800DECF89F0B7EC62F0C4D07350140D120E8B
:101AA800F324D96E010EF420DA6E5BC0DFFF070E57
:101AB8000101996F0A0EE3D07350140D110EF3242F
:101AC800D96E010EF420DA6E5BC0DFFF070E01014C
:101AD800996F0B0ED4D07350140D100EF324D96ED9
:101AE800010EF420DA6E5BC0DFFF070E0101996F6B
:101AF8000C0EC5D07350140D0F0EF324D96E010EC1
:101B0800F420DA6E5BC0DFFF9D0E806FF70E816FE9
:101B1800CFCF82F0836BCECF84F0856B7350140DDA
:101B28000F0EF324D96E010EF420DA6EDECF86F0A4
:101B3800DECF87F0DECF88F0DECF89F0B7EC62F039
:101B480089900101986B996B21D10101986B996B70
:101B58007D0E0001806FF70E816FCFCF82F0836B0F
:101B6800CECF84F0856B5BC086F0876BB7EC62F0F4
:101B78006B6A83D55BC080F10F0E0101996F3E0E31
:101B88007ED05BC081F10F0E0101996F3F0E77D0B7
:101B98005BC082F10F0E0101996F400E70D05BC0DF
:101BA80083F10F0E0101996F410E69D05BC084F17A
:101BB8000F0E0101996F420E62D05BC085F10F0EC6
:101BC8000101996F430E5BD05BC086F10F0E0101D6
:101BD800996F440E54D05BC087F1CC0E806FF30E22
:101BE800816FCFCF82F0836BCECF84F0856B80C1BD
:101BF80086F0876B81C188F0896B82C18AF08B6B14
:101C080083C18CF08D6B84C18EF08F6B85C190F091
:101C1800916B86C192F0936B87C194F0956BB7EC8A
:101C280062F00101986B996B28D5A20E806FFB0EAC
:101C3800816FCFCF82F0836BCECF84F0856BB7EC0A
:101C480062F07FD70C0E0101996F1E0E18D0FC0EA2
:101C5800806FF70E816FCFCF82F0836BCECF84F089
:101C6800856BB7EC62F00C0E0101996F1C0E986F32
:101C78000A0E5A6E02D50E0E0101996F760E986FF4
:101C880085D01F0E806FF90E816FCFCF82F0836BE6
:101C9800CECF84F0856BB7EC62F00101986B996B3D
:101CA800090E5A6E898072D098C1A6F099C1A7F022
:101CB8000001A75111E0030A13E0040A25E00B0A0A
:101CC80031E0010A35E0030A39E0010A40E0130A6D
:101CD80058E03B0A59E05AD0A65101E1B9D456D090
:101CE800A651E90A01E1ECD5030A01E1F8D5010A98
:101CF80001E104D6070A01E110D6010A01E11CD668
:101D0800030A01E128D642D0A651090A01E1C5D645
:101D1800030A01E1D1D6010A01E1DDD6070A01E192
:101D2800E9D634D0A6511D0A8DE0030A90E02ED0E2
:101D3800A651480A01E179D7E40A28D0A651750AC4
:101D48009AE0030A9EE0080A01E1FFD61FD0A651D7
:101D58003D0A01E10FD7030A01E113D7010A01E1A6
:101D680017D77F0A01E11BD7010A01E11FD7030A30
:101D780001E123D7010A01E127D7070A01E12BD79F
:101D880005D0A6512A0A02D0A6510F0A5A501200AD
:101D9800A5C0B8F0A6C0B9F0A9C0D9FFAAC0DAFF9B
:101DA800DE6ADD6AA3C00CF0A4C00DF086EC5AF020
:101DB8000001B76FB75102E0B751120020EE05F0ED
:101DC800A351D926A451DA22DF5008E020EE05F00D
:101DD800A351D926A451DA22DF50120020EE04F0D4
:101DE800A351D926A451DA22DFA2070C20EE06F06F
:101DF800A351D926A451DA2210EE06F0A351E12608
:101E0800A451E222E6CFAFF0E6CFB0F0E6CFB1F0D2
:101E1800E6CFB2F0A751AF25B36FA851B021B46F88
:101E2800000EB121B56F000EB221B66FDE50B35D62
:101E3800DE50B459DE50B559DE50B65901E3E2D24E
:101E4800A76BA86BDFD220EE06F0A351D926A451C8
:101E5800DA22FF0EDE14AB6F010EDE14AC6F000E3B
:101E6800DE14AD6F000EDE14AE6FAB51AC11AD11C8
:101E7800AE1101E032D220EE06F0A351D926A451CA
:101E8800DA22DECFABF0DECFACF0DECFADF0DECFC6
:101E9800AEF00A0E05D0D890AE33AD33AC33AB33C9
:101EA800E82EF9D7A3C0D9FFA4C0DAFF10EE02F0DC
:101EB800DE50E126DD50E222E750AF6FAF05AB15EB
:101EC800BA6FBA5101E099D020EE06F0A351D92695
:101ED800A451DA22DE50DE10DE10DE1022E120EE00
:101EE8000EF0A351D926A451DA22DECFC1F0DECFFD
:101EF800C2F0DECFC3F0DECFC4F0C151C211C311AE
:101F0800C4112FE1A3C0D9FFA4C0DAFFDECF8CF043
:101F1800DDCF8DF08E6B8F6B906B916B47EC3DF046
:101F280018D0A3C0D9FFA4C0DAFFDECF8CF0DDCF74
:101F38008DF020EE12F0A351D926A451DA22DECF7B
:101F48008EF0DECF8FF0DECF90F0DECF91F047EC51
:101F58003DF08CC0C1F08DC0C2F08EC0C3F08FC000
:101F6800C4F0C151C211C311C41101E14FD2C1055E
:101F7800C211C311C41109E120EE05F0A351D926FD
:101F8800A451DA22020EDF6E020CC1290FE1C22928
:101F98000DE1C3290BE1C42909E120EE05F0A351A5
:101FA800D926A451DA22010EDF6E010C20EE12F0C0
:101FB800A351D926A451DA22C1C0DEFFC2C0DEFF78
:101FC800C3C0DEFFC4C0DEFF20EE0EF0A351D92649
:101FD800A451DA22DE50DE10DE10DE100EE120EE13
:101FE8000EF0A351D926A451DA22C1C0DEFFC2C027
:101FF800DEFFC3C0DEFFC4C0DEFF20EE16F0A35133
:10200800D926A451DA22A3C0E1FFA4C0E2FF00EE62
:102018002AF0E650E926E550EA22DE50EE1816E1ED
:10202800DE50EE1813E1DE50EE1810E1DE50EE1827
:102038000DE1A3C0D9FFA4C0DAFFDECF24F0DDCFC5
:1020480025F021EC4FF0000901E083D1A3C0D9FFAE
:10205800A4C0DAFFDECF0BF0DDCF0CF0000120EEDC
:1020680012F0A351D926A451DA22DECF0DF0DECF2B
:102078000EF0DECF0FF0DECF10F0A8EC52F00BC060
:10208800BDF00CC0BEF00DC0BFF00EC0C0F0000126
:10209800BD51BE11BF11C01101E16ED7BA51BD27A4
:1020A800000EBE23BF23C023A7C0ABF0A8C0ACF06E
:1020B800090EAD6FD890AC33AB33AD2FFBD7ABC0A7
:1020C800BBF0ACC0BCF0BB51BC1101E1C3D0BA51EC
:1020D800BB25AB6F000EBC21AC6FA3C0D9FFA4C059
:1020E800DAFF10EE02F0DE50E126DD50E222E75082
:1020F800AD6FAE6BAB51AD5DAC51AE5912E2A3C042
:10210800D9FFA4C0DAFF10EE02F0DE50E126DD5060
:10211800E222E750AB6FBA51AB5DBB6FBC6BD8A086
:10212800BC07B8C01AF0B9C01BF0BDC01CF0BEC0D7
:102138001DF0BFC01EF0C0C01FF0BBC020F0BCC067
:1021480021F0A3C0D9FFA4C0DAFF10EE01F0DE50E1
:10215800E126DD50E222E750B1EC54F0000901E03D
:10216800F8D00001BB51AB6FBC51AC6FAD6BAE6B1F
:10217800A3C0D9FFA4C0DAFF10EE2AF0DE50E12692
:10218800DD50E222E6CFAFF0E6CFB0F0E6CFB1F017
:10219800E6CFB2F0BD51AF5DB36FBE51B059B46F69
:1021A800BF51B159B56FC051B259B66FAB51B35D9C
:1021B800AC51B459AD51B559AE51B6593CE2A3C072
:1021C800D9FFA4C0DAFFDECFABF0DDCFACF02E0E26
:1021D800AB250B6E000EAC210C6EA3C0D9FFA4C0BA
:1021E800DAFF10EE2AF0DE50E126DD50E222E6CFDB
:1021F800ADF0E5CFAEF0BD51AD5FBE51AE5B090E9F
:10220800D890AD37AE37E82EFBD7AD51B8250D6E57
:10221800AE51B9210E6E020E106E0F6A48EC60F0D6
:10222800A3C0D9FFA4C0DAFF10EE04F0DE50E12607
:10223800DD50E222E76ABBC0ABF0BCC0ACF0090ECF
:10224800D890AB37AC37E82EFBD7ABC0C5F0ACC0E5
:10225800C6F0BBD020EE0AF0A351D926A451DA2249
:1022680010EE06F0A351E126A451E222DE50E65C0E
:10227800DE50E658DE50E658DE50E6581FE3A3C0AD
:10228800D9FFA4C0DAFFDECF24F0DDCF25F021ECA2
:102298004FF0000901E05DD0A3C0D9FFA4C0DAFF68
:1022A80010EE2AF0DE50E126DD50E222BDC0E6FF46
:1022B800BEC0E6FFBFC0E6FFC0C0E6FF000120EEDB
:1022C80016F0A351D926A451DA22BDC0DEFFBEC044
:1022D800DEFFBFC0DEFFC0C0DEFFAB69010EAC6F22
:1022E80020EE06F0A351D926A451DA22DECFADF0B4
:1022F800DDCFAEF0AB51AD17AC51AE17AD51000804
:10230800C56FAE51D8A0E82A0208C66FC551A75DAF
:10231800C651A85904E2A7C0C5F0A8C0C6F0A3C01A
:10232800D9FFA4C0DAFFDECF39F0DDCF3AF020EED6
:1023380016F0A351D926A451DA22DECF3BF0DECF26
:102348003CF0DECF3DF0DECF3EF05BEC59F000090B
:1023580002E0000122D60001AB69010EAC6F20EE4D
:1023680006F0A351D926A451DA22DECFADF0DDCF95
:10237800AEF0AB51AD17AC51AE17A3C0D9FFA4C096
:10238800DAFFDECFAFF0DDCFB0F0AD51AF27AE5101
:10239800B0232E0EAF250B6E000EB0210C6EB8C008
:1023A8000DF0B9C00EF0C5C00FF0C6C010F048EC73
:1023B80060F0A3C0D9FFA4C0DAFF10EE04F0DE502D
:1023C800E126DD50E222010EE76EC551B827C6515D
:1023D800B92320EE06F0A351D926A451DA22C5511B
:1023E800DE26C651DE22000EDE22DE22A9C0D9FF7B
:1023F800AAC0DAFFC551DE26C651DD22C551A75F46
:10240800C651A85BA751A81101E01DD520EE06F022
:10241800A351D926A451DA2210EE0AF0A351E126DD
:10242800A451E222DE50E65CDE50E658DE50E65863
:10243800DE50E65814E220EE06F0A351D926A45146
:10244800DA2210EE0AF0A351E126A451E222DECFEF
:10245800E6FFDECFE6FFDECFE6FFDECFE6FF20EECB
:1024680004F0A351D926A451DA22000EDB8A000C0D
:1024780073500C0D500EF324D96E010EF420DA6E51
:102488000001CC69CD6973500C0D580EF324E16E30
:10249800010EF420E26EE6CFCEF0E5CFCFF0CC51BE
:1024A800CE27CD51CF23DE50CE5DCF51800AD06FDD
:1024B800DE50800AD0594AE373500C0D520EF324B3
:1024C800D96E010EF420DA6EDF50CA6FCB6BCC697F
:1024D800CD6973500C0D5A0EF324D96E010EF420F9
:1024E800DA6EDF50CE6FCF6BCC51CE27CD51CF23D4
:1024F800CA51CE5DCF51800AD06FCB51800AD059D6
:1025080025E373500C0D530EF324D96E010EF420FD
:10251800DA6EDF50CA6FCB6BCC69CD6973500C0D86
:102528005B0EF324D96E010EF420DA6EDF50CE6F05
:10253800CF6BCC51CE27CD51CF23CA51CE5DCF51D1
:10254800800AD06FCB51800AD05961E21F0E010179
:10255800B26F010EB46F8990080E0001806FF60EFD
:10256800816F73500C0D500EF324D96E010EF420B8
:10257800DA6EDECF82F0DDCF83F073500C0D580E8B
:10258800F324D96E010EF420DA6EDECFCAF0DDCF67
:10259800CBF0FF0ECA25846FFF0ECB21856F7350D9
:1025A8000C0D520EF324D96E010EF420DA6EDF50B2
:1025B800866F876B73500C0D5A0EF324D96E010E7B
:1025C800F420DA6EDF50CC6FFF0ECC25886F896B54
:1025D800FF0E892373500C0D530EF324D96E010E90
:1025E800F420DA6EDF508A6F8B6B73500C0D5B0E24
:1025F800F324D96E010EF420DA6EDF50CD6FFF0E92
:10260800CD258C6F8D6BFF0E8D23B7EC62F0735068
:102618000C0D530EF324D96E010EF420DA6EDF5040
:102628000001CA6FCAC0CBF0CC6BCD6BCE6BCDC0EE
:10263800CEF0CCC0CDF0CBC0CCF0CB6B73500C0D32
:102648005B0EF324D96E010EF420DA6EDF50CF6FE3
:10265800CFC0D0F0D16BD26BD36B73500C0D520E30
:10266800F324D96E010EF420DA6EDF50D46FD4C093
:10267800D5F0D66BD76BD86BD7C0D8F0D6C0D7F00B
:10268800D5C0D6F0D56BD551D003F3CFD9F0F4CF60
:10269800DAF0DB6BDC6BD103F350DA27F450DB2381
:1026A800000EDC23D651D003F350DA27F450DB2395
:1026B800000EDC23D551D203F350DB27F450DC2382
:1026C800D651D103F350DB27F450DC23D751D00384
:1026D800F350DB27F450DC23D351D503F350DC2728
:1026E800D651D203F350DC27D751D103F350DC275E
:1026F800D851D003F350DC2773500C0D5A0EF32435
:10270800D96E010EF420DA6EDF50DD6FDDC0DEF029
:10271800DF6BE06BE16B73500C0D5B0EF324D96E2D
:10272800010EF420DA6EDF50E26FE2C0E3F0E46BF2
:10273800E56BE66B73500C0D500EF324D96E010E49
:10274800F420DA6EDECFE7F0DDCFE8F0E7C0E9F09D
:10275800E8C0EAF0000EEABFFF0EEB6FEC6FE9513C
:10276800E303F3CFEDF0F4CFEEF0EF6BF06BE4039F
:10277800F350EE27F450EF23000EF023EA51E30361
:10278800F350EE27F450EF23000EF023E951E50350
:10279800F350EF27F450F023EA51E403F350EF2706
:1027A800F450F023EB51E303F350EF27F450F023F8
:1027B800E651E903F350F027EA51E503F350F02717
:1027C800EB51E403F350F027EC51E303F350F02707
:1027D800EFC0F0F0EEC0EFF0EDC0EEF0ED6BED51B4
:1027E800DE03F3CFF1F0F4CFF2F0F36BF46BDF0319
:1027F800F350F227F450F323000EF423EE51DE03D6
:10280800F350F227F450F323000EF423ED51E003C4
:10281800F350F327F450F423EE51DF03F350F3277A
:10282800F450F423EF51DE03F350F327F450F4236C
:10283800E151ED03F350F427EE51E003F350F42790
:10284800EF51DF03F350F427F051DE03F350F42780
:10285800D951F125F56FDA51F221F66FDB51F321E9
:10286800F76FDC51F421F86FCB51F525FA6FCC5195
:10287800F621FB6FCD51F721FC6FCE51F821FD6F8A
:10288800570E806FF80E816F73C082F0836B7350A0
:102898000C0D500EF324D96E010EF420DA6EDECF43
:1028A80084F0DDCF85F073500C0D520EF324D96EF1
:1028B800010EF420DA6EDF50866F876B73500C0DB3
:1028C800530EF324D96E010EF420DA6EDF50886FB0
:1028D800896B73500C0D5B0EF324D96E010EF42036
:1028E800DA6EDF50CA6F73500C0D520EF324D96E96
:1028F800010EF420DA6EDF50CA03F3CFCBF0F4CF29
:10290800CCF073500C0D5A0EF324D96E010EF4203E
:10291800DA6EDF50CD6FCDC0CEF0CF6BD06BD16B00
:1029280073500C0D5B0EF324D96E010EF420DA6E91
:10293800DF50D26FD2C0D3F0D46BD56BD66B735047
:102948000C0D500EF324D96E010EF420DA6EDECF92
:10295800D7F0DDCFD8F0D7C0D9F0D8C0DAF0000E64
:10296800DABFFF0EDB6FDC6FD951D303F3CFDDF095
:10297800F4CFDEF0DF6BE06BD403F350DE27F450C6
:10298800DF23000EE023DA51D303F350DE27F4509F
:10299800DF23000EE023D951D503F350DF27F4508D
:1029A800E023DA51D403F350DF27F450E023DB515E
:1029B800D303F350DF27F450E023D651D903F35063
:1029C800E027DA51D503F350E027DB51D403F35065
:1029D800E027DC51D303F350E027DD51CE03F3CFDA
:1029E800E1F0F4CFE2F0E36BE46BCF03F350E227BE
:1029F800F450E323000EE423DE51CE03F350E22724
:102A0800F450E323000EE423DD51D003F350E32711
:102A1800F450E423DE51CF03F350E327F450E423CA
:102A2800DF51CE03F350E327F450E423D151DD0303
:102A3800F350E427DE51D003F350E427DF51CF03EE
:102A4800F350E427E051CE03F350E427CB51E125BE
:102A5800E56FCC51E221E66F000EE321E76F000E2F
:102A6800E421E86F73500C0D530EF324D96E010E58
:102A7800F420DA6EDF50E5258A6F000EE6218B6FB1
:102A8800000EE7218C6F000EE8218D6FB7EC62F025
:102A9800750E0001806FFB0E816FFAC082F0FBC0DB
:102AA80083F0FCC084F0FDC085F0FAC086F0FBC05E
:102AB80087F0FCC088F0FDC089F0B7EC62F0735075
:102AC800200D000EF3240001A36F020EF420A46F62
:102AD800FAC0A5F0FBC0A6F0FCC0A7F0FDC0A8F0A6
:102AE8009EEC15F0F96FF95111E0EA0E806FFA0EBD
:102AF800816FFAC082F0FBC083F0FCC084F0FDC097
:102B080085F0F9C086F0876BB7EC62F073500C0D56
:102B1800540EF324D96E010EF420DA6EFAC0DEFFEB
:102B2800FBC0DEFFFCC0DEFFFDC0DEFF0101B46BB1
:102B380089901200A3C00CF0A4C00DF086EC5AF0E6
:102B48000001BD6FBD5102E0BD51120020EE05F03D
:102B5800A351D926A451DA22DF5008E020EE05F06F
:102B6800A351D926A451DA22DF50120020EE0AF030
:102B7800A351D926A451DA22A551DE5CA651DE580C
:102B8800A751DE58A851DE5816E220EE04F0A351F2
:102B9800D926A451DA22DFB20ED020EE0AF0A351D2
:102BA800D926A451DA22DECFA5F0DECFA6F0DECFFB
:102BB800A7F0DECFA8F020EE06F0A351D926A45145
:102BC800DA22DECFB9F0DECFBAF0DECFBBF0DECF4F
:102BD800BCF0BE6BBF6BC06BC16B20EE06F0A3519F
:102BE800D926A451DA22BEC0DEFFBFC0DEFFC0C0B6
:102BF800DEFFC1C0DEFFA551A611A711A81101E192
:102C080019D2A3C0D9FFA4C0DAFF10EE02F0DE503B
:102C1800E126DD50E222E750A96FA9C0AAF0AB6B0C
:102C2800AC6BAD6B090ED890AA37AB37AC37AD3764
:102C3800E82EF9D7AAC0C2F0ABC0C3F0ACC0C4F04C
:102C4800ADC0C5F0B951BA11BB11BC1101E196D0A4
:102C5800FF0EA5250B6EFF0EA6210C6EFF0EA721F9
:102C68000D6EFF0EA8210E6EC2C00FF0C3C010F08B
:102C7800C4C011F0C5C012F0D0EC5CF00BC0A9F0D4
:102C88000CC0AAF00DC0ABF00EC0ACF0FF0E0001F6
:102C9800B9250B6EFF0EBA210C6EFF0EBB210D6E0F
:102CA800FF0EBC210E6EC2C00FF0C3C010F0C4C02E
:102CB80011F0C5C012F0D0EC5CF00B500001A95D1A
:102CC8000C50AA590D50AB590E50AC5957E3FF0E92
:102CD800C225A96FFF0EC321AA6FFF0EC421AB6FD7
:102CE800FF0EC521AC6FA91DAD6FAA1DAE6FAB1D40
:102CF800AF6FAC1DB06FFF0EB925B16FFF0EBA21D3
:102D0800B26FFF0EBB21B36FFF0EBC21B46FAD5184
:102D1800B115B56FAE51B215B66FAF51B315B76FE8
:102D2800B051B415B86F20EE06F0A351D926A451BE
:102D3800DA22B5C0DEFFB6C0DEFFB7C0DEFFB8C01E
:102D4800DEFF20EE06F0A351D926A451DA22DE5088
:102D5800A55FDE50A65BDE50A75BDD50A85B20EECA
:102D680012F0A351D926A451DA22DECFC6F0DECF65
:102D7800C7F0DECFC8F0DECFC9F064D020EE0EF089
:102D8800A351D926A451DA22DECFC6F0DECFC7F090
:102D9800DECFC8F0DECFC9F0C651C711C811C911BE
:102DA80043E1A3C0D9FFA4C0DAFFDECF8CF0DDCFAA
:102DB8008DF08E6B8F6B906B916B47EC3DF08CC0F8
:102DC800C6F08DC0C7F08EC0C8F08FC0C9F0C60568
:102DD800C711C811C91109E120EE05F0A351D92680
:102DE800A451DA22020EDF6E020CC6290FE1C729B0
:102DF8000DE1C8290BE1C92909E120EE05F0A3512D
:102E0800D926A451DA22010EDF6E010C20EE0EF055
:102E1800A351D926A451DA22C6C0DEFFC7C0DEFFFF
:102E2800C8C0DEFFC9C0DEFF20EE12F0A351D926CC
:102E3800A451DA22C6C0DEFFC7C0DEFFC8C0DEFF6D
:102E4800C9C0DEFFC651C711C811C91101E095D02C
:102E5800F1D020EE04F0A351D926A451DA22DFA242
:102E680028D0A3C0D9FFA4C0DAFFDECF8CF0DDCF15
:102E78008DF0C6C08EF0C7C08FF0C8C090F0C9C032
:102E880091F047EC3DF08CC0C6F08DC0C7F08EC005
:102E9800C8F08FC0C9F0C651C711C811C91123E1C4
:102EA800C2C0A5F0C3C0A6F0C4C0A7F0C5C0A8F0B2
:102EB8006ED0A3C0D9FFA4C0DAFFDECF44F0DDCFC7
:102EC80045F0C6C046F0C7C047F0C8C048F0C9C002
:102ED80049F058EC2BF044C0C6F045C0C7F046C0D6
:102EE800C8F047C0C9F00001C62907E1C72905E1B4
:102EF800C82903E1C92901E180D7C951C811C711FF
:102F080004E1020EC65D01E267D7A3C0D9FFA4C0E1
:102F1800DAFF10EE12F0DE50E126DD50E222E65034
:102F2800C65DE650C759E650C859E650C95901E38D
:102F380053D720EE12F0A351D926A451DA22C6C0E5
:102F4800DEFFC7C0DEFFC8C0DEFFC9C0DEFF20EE5F
:102F580006F0A351D926A451DA22C251DE26C35164
:102F6800DE22C451DE22C551DE22C251A55FC35103
:102F7800A65BC451A75BC551A85BA551C25DA6510C
:102F8800C359A751C459A851C55901E262D720EEC7
:102F980006F0A351D926A451DA22A551DE26A6515E
:102FA800DE22A751DE22A851DE22A551A96F010E0B
:102FB800A615AA6FAB6BAC6BA911AB11AC113AE0BB
:102FC800A3C0D9FFA4C0DAFFDECF0BF0DDCF0CF031
:102FD800C6C00DF0C7C00EF0C8C00FF0C9C010F0D1
:102FE800A8EC52F00BC0BEF00CC0BFF00DC0C0F092
:102FF8000EC0C1F00001BE51BF11C011C11101E1E5
:10300800EBD6A5C0A9F0A6C0AAF0A7C0ABF0A8C08F
:10301800ACF00A0E05D0D890AC33AB33AA33A93341
:10302800E82EF9D7A951BE27AA51BF23AB51C02317
:10303800AC51C12320EE06F0A351D926A451DA22BF
:10304800FF0EDE14A96F010EDE14AA6F000EDE1447
:10305800AB6F000EDE14AC6FA951AA11AB11AC1105
:1030680020E020EE16F0A351D926A451DA22BE5151
:10307800DE1809E1BF51DE1806E1C051DE1803E190
:10308800C151DE180EE020EE16F0A351D926A45146
:10309800DA22BEC0DEFFBFC0DEFFC0C0DEFFC1C097
:1030A800DEFF20EE06F0A351D926A451DA2210EE55
:1030B8000AF0A351E126A451E222DE50E65CDE507C
:1030C800E658DE50E658DE50E65801E33DD520EEDE
:1030D80006F0A351D926A451DA2210EE0AF0A35122
:1030E800E126A451E222DECFE6FFDECFE6FFDECF07
:1030F800E6FFDECFE6FF20EE04F0A351D926A45167
:10310800DA22000EDB8A20D564C0A1F065C0A2F0E7
:1031180068C0D9FF69C0DAFFDE6ADD6A62C00CF0F8
:1031280063C00DF086EC5AF000019C6F9C5102E0E0
:103138009C51120020EE05F06250D9266350DA2225
:10314800DF5008E020EE05F06250D9266350DA22FD
:10315800DF50120020EE04F06250D9266350DA22C4
:10316800DFA0070C20EE06F06250D9266350DA2261
:10317800DECF8CF0DECF8DF0DECF8EF0DECF8FF09D
:1031880020EE0AF06250D9266350DA22DECF90F0A2
:10319800DECF91F0DECF92F0DECF93F08C51905DD0
:1031A800986F8D519159996F8E5192599A6F8F518D
:1031B80093599B6F66508C6F67508D6F8E6B8F6BBA
:1031C8008C51985D8D5199598E519A598F519B59AF
:1031D80001E34AD298C066F099C067F045D220EE64
:1031E80006F06250D9266350DA22FF0EDE148C6F87
:1031F800010EDE148D6F000EDE148E6F000EDE14CD
:103208008F6F8C518D118E118F1101E0A5D120EE99
:1032180006F06250D9266350DA22DECF8CF0DECF7A
:103228008DF0DECF8EF0DECF8FF00A0E05D0D8906D
:103238008F338E338D338C33E82EF9D762C0D9FFA4
:1032480063C0DAFF10EE02F0DE50E126DD50E22224
:10325800E750906F90058C15A36FA3516AE120EE9B
:1032680006F06250D9266350DA22DE50DE10DE10F6
:10327800DE100FE120EE0EF06250D9266350DA22FC
:10328800DECF9DF0DECF9EF0DECF9FF0DECFA0F048
:1032980020D062C0D9FF63C0DAFFDECF44F0DDCFB3
:1032A80045F020EE12F06250D9266350DA22DECFC4
:1032B80046F0DECF47F0DECF48F0DECF49F058ECDD
:1032C8002BF044C09DF045C09EF046C09FF047C01B
:1032D800A0F00001A0519F119E110CE1020E9D5D0E
:1032E80009E220EE05F06250D9266350DA22020E78
:1032F800DF6E020C9D290FE19E290DE19F290BE14C
:10330800A02909E120EE05F06250D9266350DA229F
:10331800010EDF6E010C20EE12F06250D9266350C8
:10332800DA229DC0DEFF9EC0DEFF9FC0DEFFA0C088
:10333800DEFF62C0D9FF63C0DAFFDECF0BF0DDCF5E
:103348000CF020EE12F06250D9266350DA22DECF5C
:103358000DF0DECF0EF0DECF0FF0DECF10F0A8ECD0
:1033680052F00BC0A4F00CC0A5F00DC0A6F00EC022
:10337800A7F00001A451A511A611A71101E1B1D729
:10338800A351A427000EA523A623A72366C08CF06B
:1033980067C08DF0090E8E6FD8908D338C338E2FC9
:1033A800FBD78CC0A8F08DC0A9F0A851A91101E1E4
:1033B800C5D0A351A8258C6F000EA9218D6F62C0BE
:1033C800D9FF63C0DAFF10EE02F0DE50E126DD50CF
:1033D800E222E7508E6F8F6B8C518E5D8D518F5925
:1033E80012E262C0D9FF63C0DAFF10EE02F0DE50CD
:1033F800E126DD50E222E7508C6FA3518C5DA86F67
:10340800A96BD8A0A907A1C01AF0A2C01BF0A4C03C
:103418001CF0A5C01DF0A6C01EF0A7C01FF0A8C0D4
:1034280020F0A9C021F062C0D9FF63C0DAFF10EE16
:1034380001F0DE50E126DD50E222E750B8EC58F00A
:10344800000901E05FD762C0D9FF63C0DAFF10EE60
:1034580004F0DE50E126DD50E222E7505FE0000193
:10346800A8518C6FA9518D6F8E6B8F6B62C0D9FF7D
:1034780063C0DAFF10EE2AF0DE50E126DD50E222CA
:10348800E6CF90F0E6CF91F0E6CF92F0E6CF93F05A
:10349800A451905D946FA5519159956FA651925979
:1034A800966FA7519359976F8C51945D8D5195598B
:1034B8008E5196598F51975931E262C0D9FF63C036
:1034C800DAFF10EE2AF0DE50E126DD50E222E6CFE8
:1034D8008CF0E5CF8DF0A4518C5FA5518D5B090E62
:1034E800D8908C378D37E82EFBD78C51A1250B6EE1
:1034F8008D51A2210C6E62C0D9FF63C0DAFFDECF06
:103508008EF0DDCF8FF02E0E8E250D6E000E8F21E2
:103518000E6E020E106E0F6A48EC60F0A8C08CF0B8
:10352800A9C08DF0090ED89000018C378D37E82E90
:10353800FAD78CC0AAF08DC0ABF079D020EE16F087
:103548006250D9266350DA22A4C0DEFFA5C0DEFF90
:10355800A6C0DEFFA7C0DEFF8C69010E8D6F20EECE
:1035680006F06250D9266350DA22DECF8EF0DDCF26
:103578008FF08C518E178D518F178E510008AA6FBE
:103588008F51D8A0E82A0208AB6FAA51665CAB51EC
:10359800675804E266C0AAF067C0ABF062C0D9FF02
:1035A80063C0DAFFDECF39F0DDCF3AF020EE16F057
:1035B8006250D9266350DA22DECF3BF0DECF3CF0F2
:1035C800DECF3DF0DECF3EF05BEC59F0000901E0C4
:1035D80099D6A1C00BF0A2C00CF000018C69010EB5
:1035E8008D6F20EE06F06250D9266350DA22DECFC6
:1035F8008EF0DDCF8FF08C518E178D518F1762C0F2
:10360800D9FF63C0DAFFDECF90F0DDCF91F08E51A5
:1036180090278F5191232E0E90250D6E000E91212B
:103628000E6EAAC00FF0ABC010F048EC60F0AA51C3
:10363800A127AB51A22320EE06F06250D926635091
:10364800DA22AA51DE26AB51DE22000EDE22DE226D
:1036580068C0D9FF69C0DAFFAA51DE26AB51DD2266
:10366800AA51665EAB51675A6650671001E0B7D53C
:10367800000C0001CE6B010ECD6F960E806FF40E1C
:10368800816FCFCF82F0836BCECF84F0856B735080
:103698000C0D500EF324D96E010EF420DA6EDECF35
:1036A80086F0DDCF87F073500C0D520EF324D96EDF
:1036B800010EF420DA6EDF50886F896B73500C0DA1
:1036C800530EF324D96E010EF420DA6EDF508A6FA0
:1036D8008B6B73500C0D5B0EF324D96E010EF42026
:1036E800DA6EDF50AC6F73500C0D520EF324D96EA6
:1036F800010EF420DA6EDF50AC03F3CFADF0F4CF57
:10370800AEF073500C0D5A0EF324D96E010EF4204E
:10371800DA6EDF50AF6FAFC0B0F0B16BB26BB36BA6
:1037280073500C0D5B0EF324D96E010EF420DA6E83
:10373800DF50B46FB4C0B5F0B66BB76BB86B7350ED
:103748000C0D500EF324D96E010EF420DA6EDECF84
:10375800B9F0DDCFBAF0B9C0BBF0BAC0BCF0000E0A
:10376800BCBFFF0EBD6FBE6FBB51B503F3CFBFF03B
:10377800F4CFC0F0C16BC26BB603F350C027F4504E
:10378800C123000EC223BC51B503F350C027F45027
:10379800C123000EC223BB51B703F350C127F45015
:1037A800C223BC51B603F350C127F450C223BD5104
:1037B800B503F350C127F450C223B851BB03F350EB
:1037C800C227BC51B703F350C227BD51B603F3500B
:1037D800C227BE51B503F350C227BF51B003F3CF80
:1037E800C3F0F4CFC4F0C56BC66BB103F350C42764
:1037F800F450C523000EC623C051B003F350C427AC
:10380800F450C523000EC623BF51B203F350C52799
:10381800F450C623C051B103F350C527F450C62352
:10382800C151B003F350C527F450C623B351BF03A9
:10383800F350C627C051B203F350C627C151B10394
:10384800F350C627C251B003F350C627AD51C32564
:10385800C76FAE51C421C86F000EC521C96F000ED5
:10386800C621CA6F73500C0D530EF324D96E010E86
:10387800F420DA6EDF50C7258C6F000EC8218D6FDB
:10388800000EC9218E6F000ECA218F6FB7EC62F04F
:1038980089800001D76BD86BD96BDA6B30D1735044
:1038A800200D000EF324626E020EF420636E8E0E5D
:1038B800646E0A0E656E010E676E666AD50E686ED6
:1038C800696A88EC18F00001DB6FDB5118E0180E0C
:1038D8000101B26F010EB46F0001D66BD56FB80E3F
:1038E800806FF60E816F73C082F0836BDBC084F04B
:1038F800856BD5C086F0D6C087F0B7EC62F0C30EF2
:103908000001806FFE0E816FD5C082F0D6C083F0B3
:10391800B7EC62F0725066E073500C0D540EF3244D
:10392800D96E010EF420DA6E8CC1B1F08DC1B2F0FF
:103938008EC1B3F00001B06B000EB025B46F010E5C
:10394800B121B56F000EB221B66F000EB321B76F6B
:10395800DE50B41947E1DE50B51944E1DE50B6191E
:1039680041E1DE50B7193EE144EC5DF00FC0D1F003
:1039780010C0D2F011C0D3F012C0D4F0000EE8CFBE
:103988008EFA2AEE8FF0D4C0DFFFE8CF90FA2AEE45
:1039980091F0D3C0DFFFE8CF92FA2AEE93F0D2C0BD
:1039A800DFFFE8CF94FA2AEE95F0D1C0DFFFE30EEF
:1039B8000001806FF50E816F2AEE8FF0DF50826F65
:1039C800836B2AEE91F0DF50846F856B2AEE93F0BB
:1039D800DF50866F876B2AEE95F0DF50886F896B12
:1039E800B7EC62F00101E793B25101E0E783D5C07B
:1039F80064F0D6C065F0DCEC44F064C0CFF065C07C
:103A0800D0F00001CF51D727D051D823000ED923A9
:103A1800DA2381AC79D0D551CF1903E1D651D01929
:103A280025E0CD6BCE6B73500C0D530EF324D96E7D
:103A3800010EF420DA6EDF500EE173500C0D500EBB
:103A4800F324D96E010EF420DA6EDE50DE1003E1A5
:103A5800050EDDEC62F0710E0001806FFE0E816FC5
:103A6800CFC082F0D0C083F0B7EC62F055EC62F0C2
:103A7800F2EC62F00B500C1011E0DB0E0001806FCD
:103A8800FD0E816FF2EC62F00BC082F00CC083F087
:103A9800B7EC62F0010E0101B46F36D00001CC6BB7
:103AA800050ECB6F1CD0680E0001AC6FE40EE82E3B
:103AB800FED7AC2FFCD700F0F2EC62F00B500C10E4
:103AC8000EE00001CD6BCE6B430E806FFD0E816F53
:103AD800CBC082F0CCC083F0B7EC62F008D0000114
:103AE800CB07D8A0CC07CB29DEE1CC29DCE1F2EC6E
:103AF80062F00B500C1003E00001CD6BCE6B00019F
:103B0800CD51CE1101E0CBD60C0E0001806FFA0E1C
:103B1800816FCFCF82F0836BCECF84F0856BD7C017
:103B280086F0D8C087F0D9C088F0DAC089F0B7EC41
:103B380062F00101B46B89901200D251D31101E1F6
:103B4800090CD2C0D9FFD3C0DAFFDE6ADD6AA0C192
:103B5800CDF1A1C1CEF11F0ED617CD0E666E010EA6
:103B6800676ED40E686ED651FE0B696E09EC00F0D4
:103B78000101CA6FCA5101E040D2B60EE16F010ED1
:103B8800E26FCD0E0001BC6F010EBD6FD4C0BEF058
:103B9800D5C0BFF0C2EC4DF00101CA6FDFC1CBF157
:103BA800E0C1CCF1CA5105E1CB51CC1102E1060EBE
:103BB800CA6FD6C0D7F01C0E0001D71701E114D187
:103BC8000101CA5113E0040ECA1909E1CD0E000122
:103BD800C06F010EC16F02EC58F00101CA6F0001FD
:103BE800D687DFC1CBF1E0C1CCF113D020EE0BF0CA
:103BF800CB51D926CC51DA22DF500001D76F110EF4
:103C0800D71702E0070E03D0D6A503D0080E01018E
:103C1800CA6F0101CA5101E002D10001D6A7FFD045
:103C28000101C66BC76B210EC86F460EC96F20EE27
:103C38000EF0CB51D926CC51DA22DF6A20EE0FF0F4
:103C4800CB51D926CC51DA22C7C1DFFF20EE10F0C4
:103C5800CB51D926CC51DA22C8C1DFFF20EE11F0B2
:103C6800CB51D926CC51DA22C9C1DFFF20EE16F09C
:103C7800CB51D926CC51DA22DF6A20EE17F0CB518E
:103C8800D926CC51DA22C7C1DFFF20EE18F0CB517C
:103C9800D926CC51DA22C8C1DFFF20EE19F0CB516A
:103CA800D926CC51DA22C9C1DFFF20EE0BF0CB5167
:103CB800D926CC51DA22DF6A20EE1CF0CB51D92666
:103CC800CC51DA22DF6A20EE1DF0CB51D926CC5137
:103CD800DA22DF6A20EE1EF0CB51D926CC51DA2247
:103CE800DF6A20EE1FF0CB51D926CC51DA22DF6AE9
:103CF800CDC10BF0CEC10CF0CBC10DF0CCC10EF094
:103D080063EC58F00BC0C2F10CC0C3F10DC0C4F194
:103D18000EC0C5F1CBC10BF0CCC10CF00D6A0E6A18
:103D28000F6A106AE6EC5FF0010120EE04F0CD5155
:103D3800D926CE51DA22010EDF6EC251C311C41149
:103D4800C5116DE020EE2AF0CD51D926CE51DA22E8
:103D5800DECFC6F1DECFC7F1DECFC8F1DECFC9F1C5
:103D6800CDC18CF0CEC18DF0C2C18EF0C3C18FF031
:103D7800C4C190F0C5C191F0F0EC50F00101CA6FD8
:103D8800CA514DE1FF0EC2250001D76FFF0E010198
:103D9800C3210001D86FFF0E0101C4210001D96FB2
:103DA800FF0E0101C5210001DA6F010120EE0AF0C2
:103DB800CD51D926CE51DA22D7C0DEFFD8C0DEFFDA
:103DC800D9C0DEFFDAC0DEFFCDC139F0CEC13AF08E
:103DD800C6C13BF0C7C13CF0C8C13DF0C9C13EF007
:103DE8005BEC59F001011AD00101CA5118E120EE2B
:103DF8000BF0CB51D926CC51DA22DFA802D0040E21
:103E08000DD00001D6A30BD0010120EE0BF0CB5151
:103E1800D926CC51DA22DFA002D0070ECA6F0101E1
:103E2800CA5123E10001D6B7D68B010120EE2AF052
:103E3800CD51D926CE51DA22000110EE1AF0D25116
:103E4800E126D351E222DECFE6FFDECFE6FFDECF6A
:103E5800E6FFDECFE6FF20EE1EF0D251D926D35181
:103E6800DA22CBC1DEFFCCC1DDFF0101CA5101E07E
:103E7800C4D0000120EE04F0D251D926D351DA2261
:103E8800D6C0DFFF20EE05F0D251D926D351DA2271
:103E9800DF6ACDC10BF0CEC10CF0CBC10DF0CCC1A7
:103EA8000EF063EC58F0000120EE0EF0D251D92646
:103EB800D351DA220BC0DEFF0CC0DEFF0DC0DEFFDF
:103EC8000EC0DEFF010120EE1DF0CB51D926CC51EA
:103ED800DA22DF500001D86FD76B010120EE1EF007
:103EE800CB51D926CC51DA22DF500001D96FD9C085
:103EF800DAF0DB6BDC6BDD6BDBC0DDF0DAC0DCF04D
:103F0800DB6BDA6B010120EE1FF0CB51D926CC51C7
:103F1800DA22DF500001DE6FDEC0DFF0E06BE16B1C
:103F2800E26BDFC0E2F0E16BE06BDF6BDA51DF11CF
:103F3800E36FDB51E011E46FDC51E111E56FDD5116
:103F4800E211E66FD751E311E76FD851E411E86F3A
:103F5800000EE511E96F000EE611EA6F010120EE8F
:103F68001CF0CB51D926CC51DA22DF500001E711E1
:103F7800EB6FE851EC6FE951ED6FEA51EE6F20EE0F
:103F88000AF0D251D926D351DA22EBC0DEFFECC0B9
:103F9800DEFFEDC0DEFFEEC0DEFF20EE06F0D25100
:103FA800D926D351DA22DE6ADE6ADE6ADD6A20EEBD
:103FB80016F0D251D926D351DA22DE6ADE6ADE6AD9
:103FC800DD6AD2C0D9FFD3C0DAFFCDC1DEFFCEC1D2
:103FD800DDFFD2C0D9FFD3C0DAFF10EE06F0DE5005
:103FE800E126DD50E22220EE02F0D251D926D3514B
:103FF800DA22E6CFDEFFE5CFDDFF0101CA5112006C
:104008008980DA0E0001806FF60E816FCFCF82F0C3
:10401800836BCECF84F0856B7350140D070EF32499
:10402800D96E010EF420DA6EDECF86F0DECF87F08F
:10403800DECF88F0DECF89F07350140D070EF3241D
:10404800D96E010EF420DA6EDECF8AF0DECF8BF067
:10405800DECF8CF0DECF8DF0B7EC62F01DEC4AF0CD
:10406800CAC0BEF1CBC0BFF10101BE51BF111AE0F9
:104078007350140D130EF324D96E010EF420DA6E6A
:104088007350140D130EF324E16E010EF420E26E4A
:10409800E7500409DF6E8DEC61F0BEC1E1F0BFC1ED
:1040A800E2F0120072507DE073507BE17350140D02
:1040B800070EF324D96E010EF420DA6E8CC1E8F0F5
:1040C8008DC1E9F08EC1EAF00001E76B000EE7252B
:1040D800EB6F010EE821EC6F000EE921ED6F000E89
:1040E800EA21EE6FDE50EB195CE1DE50EC1959E184
:1040F800DE50ED1956E1DE50EE1953E144EC5DF067
:104108000FC0C3F110C0C4F111C0C5F112C0C6F18F
:10411800000EE8CF8EFA2AEE8FF0C6C1DFFFE8CF97
:1041280090FA2AEE91F0C5C1DFFFE8CF92FA2AEEA5
:1041380093F0C4C1DFFFE8CF94FA2AEE95F0C3C12B
:10414800DFFF0101E793010E656E646ADCEC44F061
:10415800E793C50E0001806FF40E816FCFCF82F018
:10416800836BCECF84F0856B2AEE8FF0DF50866F9D
:10417800876B2AEE91F0DF50886F896B2AEE93F0F7
:10418800DF508A6F8B6B2AEE95F0DF508C6F8D6B4A
:10419800B7EC62F06B6A89906BC0E1F00001E26BEA
:1041A80012007350140D0F0EF324D96E010EF42073
:1041B800DA6EDECFE3F0DECFE4F0DECFE5F0DECF7F
:1041C800E6F0E4C0E3F0E5C0E4F0E6C0E5F00001A5
:1041D800E66BE3C0BAF1E4C0BBF17350140D0F0EE7
:1041E800F324D96E010EF420DA6EDECFE3F0DDCFD2
:1041F800E4F0E3510101C06FC16BE793B66BB76B95
:10420800B86BB96BBC6BBD6BA9D0E369E469BAC183
:10421800E5F0BBC1E6F0E351E527E451E6230101EF
:10422800BC510001E5190AE10101BD510001E6197F
:1042380005E10101C051C11101E1E7837350200D6F
:10424800000EF324626E020EF420636E8E0E646E0E
:104258000A0E656E010E676E666AC70E686E010EFD
:10426800696E88EC18F00101C26F510E0001806F71
:10427800F60E816FCFCF82F0836BCECF84F0856B43
:10428800C2C186F0876BC7C188F0C8C189F0B7EC96
:1042980062F00101C25101E0EBD6C7C164F0C8C1A8
:1042A80065F0DCEC44F0C751B627C851B723000EBF
:1042B800B823B9237350140D070EF324D96E010ED9
:1042C800F420DA6E000EDE240001E36F010EDE201A
:1042D800E46F000EDE20E56F000EDE20E66F7350FF
:1042E800140D070EF324D96E010EF420DA6EE3C024
:1042F800DEFFE4C0DEFFE5C0DEFFE6C0DEFFCC0E79
:10430800806FF80E816FCFCF82F0836BCECF84F0B1
:10431800856B7350140D070EF324D96E010EF4202B
:10432800DA6EDECF86F0DECF87F0DECF88F0DECF24
:1043380089F07350140D070EF324D96E010EF42082
:10434800DA6EDECF8AF0DECF8BF0DECF8CF0DECFF8
:104358008DF0B7EC62F00101BC4BBD2BBA51BC5DCE
:10436800BD51800A0001E36F0101BB51800A0001C1
:10437800E35901E24AD70101C1BF8CD0C15103E121
:10438800C00501E287D07350200D000EF324626E41
:10439800020EF420636E8E0E646E0A0E656EC0C146
:1043A80066F0C1C167F0C70E686E010E696E88ECD1
:1043B80018F00101C26F5E0E0001806FF60E816F6A
:1043C800C2C182F0836BC7C184F0C8C185F0B7EC65
:1043D80062F00101C25101E04BD6C751C81101E199
:1043E80047D6E783C0C164F0C1C165F0DCEC44F096
:1043F800C751B627C851B723000EB823B923735045
:10440800140D070EF324D96E010EF420DA6E000E97
:10441800DE240001E36F010EDE20E46F000EDE20D3
:10442800E56F000EDE20E66F7350140D070EF324BF
:10443800D96E010EF420DA6EE3C0DEFFE4C0DEFFC1
:10444800E5C0DEFFE6C0DEFF1B0E806FFC0E816F4D
:104458007350140D070EF324D96E010EF420DA6E92
:10446800DECF82F0DECF83F0DECF84F0DECF85F0C2
:104478007350140D070EF324D96E010EF420DA6E72
:10448800DECF86F0DECF87F0DECF88F0DECF89F092
:10449800B7EC62F00101E7933F0E0001806FFA0E5E
:1044A800816FCFCF82F0836BCECF84F0856BB6C19E
:1044B80086F0B7C187F0B8C188F0B9C189F0B7EC08
:1044C80062F068D649504810471003E1020E465C76
:1044D80010E320EE12F04450D9264550DA22DE507F
:1044E800465CDE504758DE504858DE50495801E2D5
:1044F8002FD2020E866F41D246C084F047C085F0A5
:10450800D89085314F6E84314E6E4E5084274F506F
:10451800852344C039F045C03AF020EE1EF04450DF
:10452800D9264550DA22DECF4EF0DECF4FF0DECF6F
:1045380050F0DECF51F084C052F085C053F0090E20
:10454800546ED89053325232542EFBD752504E24C8
:104558003B6E53504F203C6E000E50203D6E000EB7
:1045680051203E6E5BEC59F00001866F865101E0E8
:1045780004D24E68010E4F6E84C050F085C051F0D1
:104588004E5050164F50511644C052F045C053F08B
:1045980050505226515053222E0E5224876F000E2F
:1045A8005320886F844B852B46B004D04AC080F0D6
:1045B800816B1AD04A504E6E4F6A4E3A4F3AF00EFF
:1045C8004F164E500F0B4F12F00E4E1687C0D9FFE4
:1045D80088C0DAFFDF500F0B506E516A4E505010F2
:1045E800806F4F505110816F87C0D9FF88C0DAFFA4
:1045F80080C0DFFF20EE04F04450D9264550DA226F
:10460800010EDF6E44C039F045C03AF020EE1EF0CE
:104618004450D9264550DA22DECF4EF0DECF4FF097
:10462800DECF50F0DECF51F084C052F085C053F099
:10463800090E546ED89053325232542EFBD7525032
:104648004E243B6E53504F203C6E000E50203D6E62
:10465800000E51203E6E5BEC59F00001866F8651CA
:1046680001E08BD14E68010E4F6E84C050F085C0BA
:1046780051F04E5050164F50511644C052F045C09C
:1046880053F050505226515053222E0E5224876F09
:10469800000E5320886F46B00CD04BC04EF00F0E62
:1046A8004E1687C0D9FF88C0DAFFDF50F00B4E10D6
:1046B80012D04AC04EF04BC04FF04CC050F04DC025
:1046C80051F0050E05D0D890513250324F324E324B
:1046D800E82EF9D74E50826F836B87C0D9FF88C008
:1046E800DAFF82C0DFFF2BD144C039F045C03AF071
:1046F80020EE1EF04450D9264550DA22DECF4EF087
:10470800DECF4FF0DECF50F0DECF51F04750526E83
:104718004850536E4950546E556A4E5052243B6E61
:104728004F5053203C6E505054203D6E51505520F0
:104738003E6E5BEC59F00001866F865101E01DD199
:104748004E68010E4F6E46C050F047C051F0D890E9
:10475800503651364E5050164F50511644C052F0F4
:1047680045C053F050505226515053222E0E522419
:10477800876F000E5320886F87C0D9FF88C0DAFF83
:104788004AC0DFFF20EE01F08751D9268851DA228E
:104798004BC0DFFFD4D044C039F045C03AF020EE1A
:1047A8001EF04450D9264550DA22DECF4EF0DECF37
:1047B8004FF0DECF50F0DECF51F046C052F047C088
:1047C80053F048C054F049C055F0080E05D0D890B1
:1047D8005532543253325232E82EF9D74E505224C1
:1047E8003B6E4F5053203C6E505054203D6E5150FC
:1047F80055203E6E5BEC59F00001866F865101E052
:10480800BCD04E68010E4F6E46C050F047C051F004
:10481800D89050365136D890503651364E505016A2
:104828004F50511644C052F045C053F050505226D4
:10483800515053222E0E5224876F000E5320886F3A
:1048480020EE01F08751D9268851DA22DF504F6EC9
:104858004E6A20EE02F08751D9268851DA22DF50BD
:10486800506E50C051F0526A536A546A52C054F0A4
:1048780051C053F0526A516A20EE03F08751D9268D
:104888008851DA22DF50556E55C056F0576A586A7B
:10489800596A56C059F0586A576A566A51505610A4
:1048A8005A6E525057105B6E535058105C6E5450ED
:1048B80059105D6E4E505A105E6E4F505B105F6E11
:1048C800000E5C10606E000E5D10616E87C0D9FF2F
:1048D80088C0DAFFDF505E10626E5F50636E605012
:1048E800646E6150656E666A676A686AF00E651480
:1048F800696E66504A1267504B1268504C126950E4
:104908004D1287C0D9FF88C0DAFF4AC0DFFF20EE0A
:1049180001F08751D9268851DA224BC0DFFF20EEFB
:1049280002F08751D9268851DA224CC0DFFF20EEE9
:1049380003F08751D9268851DA224DC0DFFF20EED7
:1049480004F04450D9264550DA22010EDF6E15D006
:1049580044C0D9FF45C0DAFFDF504E6E4F6A4F5052
:1049680001E0C7D54E50010A01E1C6D5030A01E1AD
:10497800BBD6010A01E10FD7BCD58651120018C079
:10498800F6FF19C0F7FF000EF86E0F0EF76403D09C
:104998000800F55005D0F6CFE9FFF7CFEAFFEF5052
:1049A800586E184A192A585001E11200250E581855
:1049B80004E05850C1EC62F0E2D7516A526A536A77
:1049C800546A18C0F6FF19C0F7FF000EF86E0F0EF4
:1049D800F76403D00800F55005D0F6CFE9FFF7CF0C
:1049E800EAFFEF50586E184A192A300E581818E185
:1049F800546A010E536E18C0F6FF19C0F7FF000E77
:104A0800F86E0F0EF76403D00800F55005D0F6CF06
:104A1800E9FFF7CFEAFFEF50586E184A192A06D077
:104A28002D0E581803E1546A020EE4D72A0E5818BE
:104A380059E11A50D96EDA6A020EDF26DF5CD96EA8
:104A4800DA6ADECF49F0DECF4AF04AAE0BD04950E1
:104A58000008496E4A50D8A0E82A00084A6E546AED
:104A6800020E536E49C051F04AC052F018C0F6FF0A
:104A780019C0F7FF000EF86E0F0EF76403D0080098
:104A8800F55005D0F6CFE9FFF7CFEAFFEF50586EA3
:104A9800184A192A2DD00A0E5102F3CF1BF0F4CF71
:104AA8001CF05202F3501C2658501B26000E1C22E4
:104AB800D00E1B24516EFF0E1C20526E18C0F6FF3C
:104AC80019C0F7FF000EF86E0F0EF76403D0080048
:104AD800F55005D0F6CFE9FFF7CFEAFFEF50586E53
:104AE800184A192A2F0E586403D0390E5864D3D7A0
:104AF8006C0E581803E04C0E581815E1538418C072
:104B0800F6FF19C0F7FF000EF86E0F0EF76403D01A
:104B18000800F55005D0F6CFE9FFF7CFEAFFEF50D0
:104B2800586E184A192A585001E1120058C057F017
:104B3800600E576472D0200E575E6FD01A50D96E2F
:104B4800DA6A020EDF26DF5CD96EDA6ADECF41F060
:104B5800DECF42F04F6A506A02D04F4A502A4F5077
:104B680041241B6E505042201C6E1BC0F6FF1CC017
:104B7800F7FF000EF86E0F0EF76403D00800F5502B
:104B880005D0F6CFE9FFF7CFEAFFEF50000904E0C0
:104B9800E4D7200EC1EC62F053B20BD04F501B6E1D
:104BA80050501C6E4F4A502A51501B5C52501C5892
:104BB800F0E341C00CF042C00DF0DEEC5EF003D033
:104BC800200EC1EC62F04F501B6E50501C6E4F4AC5
:104BD800502A51501B5C52501C5801E3D0D6F0D7D4
:104BE8001A50D96EDA6ADF50DF2ADF2AD96EDA6AFC
:104BF800DF50C1EC62F0C3D6446A020E08D0446AA2
:104C0800080E05D0446A0A0E02D0446A100E436E9C
:104C180019D05850C1EC62F0B2D657501B6E1C6ABE
:104C28001C50F7E11B50420AE7E0010AD9E0070AE5
:104C3800E9E00B0AE4E01C0A81E0060AE3E00D0A59
:104C4800E4E0E7D753A411D01A50D96EDA6A040EFB
:104C5800DF26DF5CD96EDA6ADECF4BF0DECF4CF0B0
:104C6800DECF4DF0DECF4EF027D0440E571813E0BC
:104C78001A50D96EDA6ADF50DF2ADF2AD96EDA6A6B
:104C8800DECF1BF0DDCF1CF01BC04BF01CC04CF07E
:104C98004D6A4E6A11D01A50D96EDA6ADF50DF2A8F
:104CA800DF2AD96EDA6ADECF4BF0DDCF4CF0000E8A
:104CB8004CBEFF0E4D6E4E6E440E57180CE14EAEB4
:104CC8000AD04B6C4C1ED8B04C2A4D1ED8B04D2A79
:104CD800000E4E565388556A566A4BC045F04CC074
:104CE80046F04DC047F04EC048F045C00BF046C0F6
:104CF8000CF047C00DF048C00EF043C00FF044C0A0
:104D080010F0116A126A78EC5DF00B50576E45C0CE
:104D18000BF046C00CF047C00DF048C00EF043C081
:104D28000FF044C010F0116A126AD0EC5CF00BC0AE
:104D380045F00CC046F00DC047F00EC048F0090E13
:104D480057640BD0780E581803E03E6A070E02D05D
:104D58003E6A270E3D6E3D50572655501D0FD96EA1
:104D6800DA6A5750300FDF6E554A562A45504610BA
:104D78004710481005E0565003E1200E555CB5E396
:104D880053A808D055501D0FD96EDA6A2D0EDF6E64
:104D9800554A562A55C04FF056C050F053B003D06C
:104DA800406A200E02D0406A300E3F6E3FC057F076
:104DB80003D05750C1EC62F053B20BD04F501B6E6A
:104DC80050501C6E4F4A502A51501B5C52501C5870
:104DD800F0E35506D8A0560655501D0FD96EDA6A6D
:104DE800DF50C1EC62F05550561004E0F2D7200EA7
:104DF800C1EC62F04F501B6E50501C6E4F4A502A47
:104E080051501B5C52501C5801E3B9D5F0D7735070
:104E18000C0D530EF324D96E010EF420DA6EDF2A3E
:104E280073500C0D530EF324D96E010EF420DA6E74
:104E3800DF500001CA6FCB6BCC69CD6973500C0D84
:104E48005B0EF324D96E010EF420DA6EDF50CE6FBC
:104E5800CF6BCC51CE27CD51CF23CA51CE5DCF5188
:104E6800800AD06FCB51800AD0594BE273500C0D99
:104E7800530EF324D96E010EF420DA6EDF6A7350F4
:104E88000C0D520EF324D96E010EF420DA6EDF2ACF
:104E980073500C0D520EF324D96E010EF420DA6E05
:104EA800DF50CA6FCB6BCC69CD6973500C0D5A0EAD
:104EB800F324D96E010EF420DA6EDF50CE6FCF6B7B
:104EC800CC51CE27CD51CF23CA51CE5DCF51800AC8
:104ED800D06FCB51800AD05914E273500C0D520E8A
:104EE800F324D96E010EF420DA6EDF6A73500C0DCC
:104EF800500EF324D96E010EF420DA6EDE2A000E6D
:104F0800DD2273500C0D530EF324D96E010EF420DC
:104F1800DA6EDF50CA6FCAC0CBF0CC6BCD6BCE6BEC
:104F2800CDC0CEF0CCC0CDF0CBC0CCF0CB6B7350A5
:104F38000C0D5B0EF324D96E010EF420DA6EDF50EF
:104F4800CF6FCFC0D0F0D16BD26BD36B73500C0D39
:104F5800520EF324D96E010EF420DA6EDF50D46FAE
:104F6800D4C0D5F0D66BD76BD86BD7C0D8F0D6C025
:104F7800D7F0D5C0D6F0D56BD551D003F3CFD9F043
:104F8800F4CFDAF0DB6BDC6BD103F350DA27F450A3
:104F9800DB23000EDC23D651D003F350DA27F4507C
:104FA800DB23000EDC23D551D203F350DB27F4506A
:104FB800DC23D651D103F350DB27F450DC23D7513F
:104FC800D003F350DB27F450DC23D351D503F3503F
:104FD800DC27D651D203F350DC27D751D103F35045
:104FE800DC27D851D003F350DC2773500C0D5A0E30
:104FF800F324D96E010EF420DA6EDF50DD6FDDC0C8
:10500800DEF0DF6BE06BE16B73500C0D5B0EF3248D
:10501800D96E010EF420DA6EDF50E26FE2C0E3F0E1
:10502800E46BE56BE66B73500C0D500EF324D96EF0
:10503800010EF420DA6EDECFE7F0DDCFE8F0E7C04E
:10504800E9F0E8C0EAF0000EEABFFF0EEB6FEC6F84
:10505800E951E303F3CFEDF0F4CFEEF0EF6BF06B33
:10506800E403F350EE27F450EF23000EF023EA5147
:10507800E303F350EE27F450EF23000EF023E95139
:10508800E503F350EF27F450F023EA51E403F3501B
:10509800EF27F450F023EB51E303F350EF27F450DC
:1050A800F023E651E903F350F027EA51E503F35002
:1050B800F027EB51E403F350F027EC51E303F350EE
:1050C800F027EFC0F0F0EEC0EFF0EDC0EEF0ED6BC2
:1050D800ED51DE03F3CFF1F0F4CFF2F0F36BF46BA4
:1050E800DF03F350F227F450F323000EF423EE51BC
:1050F800DE03F350F227F450F323000EF423ED51AE
:10510800E003F350F327F450F423EE51DF03F35098
:10511800F327F450F423EF51DE03F350F327F45050
:10512800F423E151ED03F350F427EE51E003F3507B
:10513800F427EF51DF03F350F427F051DE03F35067
:10514800F427D951F125F56FDA51F221F66FDB51C9
:10515800F321F76FDC51F421F86FCB51F525F96F86
:10516800CC51F621FA6FCD51F721FB6FCE51F821C2
:10517800FC6F73500C0D540EF324D96E010EF420FD
:10518800DA6EF9C0DEFFFAC0DEFFFBC0DEFFFCC04E
:10519800DEFFF20E806FF90E816F73C082F0836BB1
:1051A80073500C0D500EF324D96E010EF420DA6EF4
:1051B800DECF84F0DDCF85F073500C0D520EF32452
:1051C800D96E010EF420DA6EDF50866F876B73504C
:1051D8000C0D530EF324D96E010EF420DA6EDF5055
:1051E800886F896BB7EC62F07350200D000EF324C2
:1051F8000001A36F020EF420A46F73500C0D540E1F
:10520800F324D96E010EF420DA6EDECFA5F0DECFDE
:10521800A6F0DECFA7F0DECFA8F09EEC15F06A6E00
:105228006A5019E0EA0E806FFA0E816F73500C0D08
:10523800540EF324D96E010EF420DA6EDECF82F01C
:10524800DECF83F0DECF84F0DECF85F06AC086F053
:10525800876BB7EC62F00101B46B12005F6E5B50B4
:1052680002E0A0EC57F05E6A5A5001E1BFD15F9EA0
:10527800040E5F1803E0140E5F1807E10101A26B2A
:10528800A36B5B6A070E5A6E070C3F0E5F1807E1A7
:105298006F6A0101A26BA36B5A6A5B6A12005F0E08
:1052A8005F1807E1706A0101A26BA36B5A6A5B6A17
:1052B80012003F0E5F640AD05F0E5F6007D0400E99
:1052C8005F1804E0706A5A6A5B6A1200400E5F1841
:1052D80010E1010E706E6F6A0101A26BA36B9E0E46
:1052E8000001806FFF0E816FB7EC62F05A6A5B6A4B
:1052F8001200200E5F1801E079D1010E6F6E0101D6
:10530800A26BA36B980E0001806FFF0E816FB7EC44
:1053180062F0ECD7600E5F1809E1705007E00101F8
:10532800B351080ED8B4030E5E6E7AD0600E5F18C3
:1053380009E16F5007E00101B35102E0090E14D0F2
:10534800050E12D0680E5F1809E16F5007E01A0EBB
:105358000101A36F900E3DD18980A2D1680E5F181C
:1053680005E1705003E0020E5E6E5AD06A0E5F18B7
:1053780007E16F5005E01A0E0101A36FF40E29D161
:105388006C0E5F1807E16F5005E01A0E0101A36F5C
:105398002C0E1FD1700E5F180FE170500DE0920EA9
:1053A8000001806FFF0E816FB7EC62F0040E5E6E35
:1053B8000101A26BA36BD0D7700E5F1801E070D10A
:1053C8006F5001E16DD11B0E0101A36F620E01D177
:1053D8008980020E5F1805E11A0E0101A36F920E73
:1053E800A26F050E5F1805E11A0E0101A36FAE0E3C
:1053F800A26F070E5F1805E11A0E0101A36FB80E20
:10540800A26F080E5F1805E11A0E0101A36FCC0EFA
:10541800A26F030E5F1802E05F2806E15E6A8990BA
:105428000101A26BA36B3CD1160E5F1801E038D1C5
:105438001A0E0101A36FA40EBDD0050E5F1805E179
:105448001A0E0101A36FF50EA26F080E5F1801E096
:1054580027D11A0E0101A36FCC0EA26F010EB36FF4
:105468001FD15FC073F01A0E0101A36F9B0EA2D06B
:105478005F505D6E5C6A73500C0D500EF324D96E4C
:10548800010EF420DA6E5CC0DEFF5DC0DDFF1A0E8F
:105498000101A36F9C0E8ED05F505C6E5D6A7350E5
:1054A8000C0D500EF324D96E010EF420DA6E5CC098
:1054B800DEFF5DC0DDFF1A0E0101A36F9D0E7AD0DD
:1054C80073500C0D520EF324D96E010EF420DA6ECF
:1054D8005FC0DFFF1A0E0101A36F9E0E6BD07350E1
:1054E8000C0D530EF324D96E010EF420DA6E5FC052
:1054F800DFFF0101A26BA36B010E62D01A0E01013E
:10550800A36FB90E66D01A0E0101A36FBA0E52D05E
:105518001A0E0101A36FBB0EA26F640E0001806F0B
:10552800FE0E816FB7EC62F00101B46BA26BA36B46
:1055380048D00101A26BA36B640E0001806FFE0EC0
:10554800816FB7EC62F03DD00101A26BA36B060E30
:105558005E6EA6D05FC073F00101A26BA36B5E6A9A
:1055680030D00101B36B1A0EA36FF70EA26F29D0CA
:105578001A0E0101A36FF70E1DD08990270E0101A5
:10558800A36F0F0E17D0180E5F1801E089D01A0EFE
:105598000101A36F2D0E0ED01A0E0101A36F2E0E5E
:1055A80009D01A0E0101A36F2F0E04D01A0E0101A3
:1055B800A36F300EA26F74D00101A26BA36B0A0E09
:1055C8005E6E89906DD0040E5E6E270E0101A36F8A
:1055D8000F0EA26FC1D68980010104D08990010EF7
:1055E8000101B36FA26BA36B5E6A5AD0A2C15CF0D3
:1055F800A3C15DF05D5007E01A0A09E0010A48E01E
:105608003C0A4CE04DD05C5001E184D649D05C5056
:105618002C0AB9E0010AC0E0030AC3E0010AC6E0A7
:105628001F0ACAE0A00A01E1D3D6020A01E119D78C
:10563800090A01E11DD7070A01E12ED7010A01E194
:105648003FD7030A01E14BD73A0A01E17DD70A0A9D
:10565800C5E0160A01E152D7010A01E154D7030A4D
:1056680001E156D7010A01E164D7790A01E17BD645
:105678000E0A01E16FD7380A01E1DFD6010A01E11C
:1056880070D7030A01E174D7010A01E176D708D07F
:105698005C50580A98E03A0A9EE002D05C500F0A23
:1056A8005EC05AF05B6A120049504810471003E187
:1056B800020E465C0FE320EE12F04450D926455006
:1056C800DA22DE50465CDE504758DE504858DE503D
:1056D800495808E3010E0001846F000E856B866B44
:1056E800876BEFD100018469856986698769D4D1A0
:1056F80046C088F047C089F0D89089314B6E883110
:105708004A6E4A5088274B50892344C039F045C017
:105718003AF020EE1EF04450D9264550DA22DECF6A
:105728004AF0DECF4BF0DECF4CF0DECF4DF088C034
:105738004EF089C04FF0090E506ED8904F324E325D
:10574800502EFBD74E504A243B6E4F504B203C6E98
:10575800000E4C203D6E000E4D203E6E5BEC59F065
:10576800000901E0AED14A68010E4B6E88C04CF0CA
:1057780089C04DF04A504C164B504D1644C04EF05F
:1057880045C04FF04C504E264D504F222E0E4E2401
:10579800D96E000E4F20DA6EDF500001826F836BE6
:1057A800884B892B44C039F045C03AF020EE1EF0F2
:1057B8004450D9264550DA22DECF4AF0DECF4BF0EE
:1057C800DECF4CF0DECF4DF088C04EF089C04FF0F0
:1057D800090E506ED8904F324E32502EFBD74E5095
:1057E8004A243B6E4F504B203C6E000E4C203D6EC1
:1057F800000E4D203E6E5BEC59F0000901E061D1CE
:105808004A68010E4B6E88C04CF089C04DF04A5072
:105818004C164B504D1644C04EF045C04FF04C50FE
:105828004E264D504F222E0E4E24D96E000E4F207C
:10583800DA6EDF50516E506A505000018213515099
:10584800831346B006D08251806F0F0E8315816F87
:105858000FD082C04AF083C04BF0040E4C6ED89033
:105868004B324A324C2EFBD74AC080F04BC081F0F5
:1058780080C084F081C085F05BD044C039F045C059
:105888003AF020EE1EF04450D9264550DA22DECFF9
:105898004AF0DECF4BF0DECF4CF0DECF4DF0475074
:1058A8004E6E48504F6E4950506E516A4A504E24C1
:1058B8003B6E4B504F203C6E4C5050203D6E4D502F
:1058C80051203E6E5BEC59F0000901E0FAD04A68BD
:1058D800010E4B6E46C04CF047C04DF0D8904C3688
:1058E8004D364A504C164B504D1644C04EF045C0EC
:1058F8004FF04C504E264D504F222E0E4E24000194
:105908008A6F000E4F208B6F20EE01F08A51D92646
:105918008B51DA22DF504B6E4A6A8AC0D9FF8BC09E
:10592800DAFFDF504A12000E4AC084F04BC085F0FF
:10593800866B876BC6D044C039F045C03AF020EE7C
:105948001EF04450D9264550DA22DECF4AF0DECF89
:105958004BF0DECF4CF0DECF4DF046C04EF047C0E6
:105968004FF048C050F049C051F0080E05D0D8900B
:10597800513250324F324E32E82EF9D74A504E2427
:105988003B6E4B504F203C6E4C5050203D6E4D505E
:1059980051203E6E5BEC59F0000901E092D04A6854
:1059A800010E4B6E46C04CF047C04DF0D8904C36B7
:1059B8004D36D8904C364D364A504C164B504D16F5
:1059C80044C04EF045C04FF04C504E264D504F222B
:1059D8002E0E4E2400018A6F000E4F208B6F20EE92
:1059E80001F08A51D9268B51DA22DF504B6E4A6A70
:1059F80020EE02F08A51D9268B51DA22DF504C6E04
:105A08004CC04DF04E6A4F6A506A4EC050F04DC0BF
:105A18004FF04E6A4D6A20EE03F08A51D9268B5119
:105A2800DA22DF50516E51C052F0536A546A556AF7
:105A380052C055F0546A536A526A4D505210566E0D
:105A48004E505310576E4F505410586E50505510BA
:105A5800596E4A5056105A6E4B5057105B6E000ED6
:105A680058105C6E000E59105D6E8AC0D9FF8BC04D
:105A7800DAFFDF505A105E6E5B505F6E5C50606EEE
:105A88005D50616E5E50846F5F50856F6050866FA9
:105A98000F0E6114876F15D044C0D9FF45C0DAFFD7
:105AA800DF504A6E4B6A4B5001E014D64A50010A47
:105AB80001E11ED6030A01E1E0D6010A01E13BD764
:105AC80009D684C044F085C045F086C046F087C03A
:105AD80047F012002A6E1BC041F01CC042F02A5049
:105AE80001E0040C010E3F6E74B0030CE9D18AEC9E
:105AF80062F0000901E1FDD13F6AFBD1146A156A21
:105B0800166A176A090EDAEC60F0000901E0F1D1B3
:105B18002B0E0B6E0C6A0E6A100E0D6E33EC5EF0D7
:105B2800000901E1E6D12B44E846030BE8064DE104
:105B380032C01DF03F0E1D161DC01EF01F6A206AE0
:105B4800216A1FC021F01EC020F01F6A1E6A335050
:105B5800236E226A3450246E256A2250242623504C
:105B6800252224501E24266E25501F20276E000E45
:105B78002020286E000E2120296E26283B6E000E5C
:105B880027203C6E000E28203D6E000E29203E6E18
:105B98003BC01DF03CC01EF03DC01FF03EC020F0D1
:105BA8000A0ED8901D361E361F362036E82EF9D735
:105BB8001BC0D9FF1CC0DAFF1DC0DEFF1EC0DEFF00
:105BC8001FC0DEFF20C0DEFF97D71D6A35AE01D0AB
:105BD8001D2A010E1D1630C01EF00F0E1E16345061
:105BE800030B020DF3501E241D24020F406E31508A
:105BF800030B1D6E1E6A0A0ED8901D361E36E82E3F
:105C0800FBD732501F6E206AD8901F362036D890A6
:105C18001F3620363344E846030B216E226A1F5094
:105C28002126205022221D5021261E502222212AC0
:105C3800000E222221C03BF022C03CF03D6A3E6AA1
:105C480040C01DF0F70E1D263BC01EF03CC01FF0E3
:105C58003DC020F03EC021F01D2A05D0D8901E3648
:105C68001F36203621361D2EF9D734D06EA43FD0EA
:105C7800146A156A166A176A8D0EDAEC60F0000964
:105C880001E037D1E5EC62F02B0E0B6E0C6A0E6A60
:105C9800100E0D6E33EC5EF0000901E12AD1300ED2
:105CA800406E03D0E5EC62F040064050FBE135C0A1
:105CB8001DF01D3A0F0E1D16100E1E6E1F6A206A6B
:105CC800216A1D2A05D0D8901E361F362036213667
:105CD8001D2EF9D71BC0D9FF1CC0DAFF1EC0DEFF7E
:105CE8001FC0DEFF20C0DEFF21C0DEFF05D7146A1B
:105CF800156A166A176A090EDAEC60F0000901E005
:105D0800F8D02B0E0B6E0C6A0E6A100E0D6E33EC6B
:105D18005EF0000901E1EDD06EA232D038C01DF06E
:105D2800060E1E6ED8901D321E2EFCD7FF0E1D26A5
:105D380035503F0B1F6E206AD8901F3620363644E8
:105D4800010B1F26000E20221F2A20221D2A03D005
:105D5800D8901F3620361D2EFBD71F50216E20509D
:105D6800226E236A246A1BC0D9FF1CC0DAFF21C037
:105D7800DEFF22C0DEFF23C0DEFF24C0DEFFBCD66C
:105D88003650030B1D6E1E6AD8901D361E36D890ED
:105D98001D361E36D8901D361E363638E842070B9B
:105DA8001D26000E1E221D2A1E223540E8423F0BEA
:105DB8001F0B1F6E206A1F2A000E20221D501F0273
:105DC800F3CF21F0F4CF22F02002F35022261E5008
:105DD8001F02F35022262150236E2250246E256A7A
:105DE800266A1BC0D9FF1CC0DAFF23C0DEFF24C00F
:105DF800DEFF25C0DEFF26C0DEFF7ED641C0D9FF0C
:105E080042C0DAFF6EC0DFFF77D6146A156A166AD9
:105E1800176A090EDAEC60F000096BE141C00BF07B
:105E280042C00CF00E6A100E0D6E33EC5EF00009E5
:105E380001E062D65ED0146A156A166A176A0A0EFD
:105E4800DAEC60F0000955E141C00BF042C00CF0FB
:105E58000E6A100E0D6E33EC5EF0E9D7146A156AFF
:105E6800166A176A3A0EDAEC60F0000942E1040E8D
:105E7800406E0AD0E5EC62F041C0D9FF42C0DAFFBB
:105E8800DF6E414A422A4006405001E135D6F2D73A
:105E9800146A156A166A176A8D0EDAEC60F0000942
:105EA80028E1E5EC62F041C00BF042C00CF00E6A4C
:105EB800400E0D6E33EC5EF0BAD7040E3F6E19D06B
:105EC8001A501D6E1E6A1E50F8E11D5001E10FD6D2
:105ED800010A01E113D6020A01E1C8D6090A8EE0D7
:105EE800010A93E0070AA7E0010AB8E0030AD0E034
:105EF800E4D7F7EC62F03F50120055C058F056C096
:105F080059F00101906B916BF6D154C046F0580ED0
:105F1800476E57C048F04750D96EDA6ADECFF6FFB1
:105F2800DDCFF7FFF86A000EF86E0800F550250A75
:105F3800D8A4C3D14750D96EDA6ADE2A000EDD2212
:105F48000101926B936B966B976B946995694750B7
:105F5800D96EDA6ADECFF6FFDDCFF7FFF86A000EFA
:105F6800F86E0800F550780AD8B40FD04750D96EAB
:105F7800DA6ADECFF6FFDDCFF7FFF86A000EF86EBB
:105F88000800F550580AD8A46ED14750D96EDA6A7D
:105F9800DECFF6FFDDCFF7FFF86A000EF86E0800D7
:105FA800F5CF53F04750D96EDA6ADE2A000EDD22AB
:105FB8004850D96EDA6ADF50DF2ADF2AD96EDA6AEA
:105FC800DECF49F0DDCF4AF049C04BF04AC04CF073
:105FD8004D6A4E6A4F6A506A516A526A46C024F046
:105FE8004BC025F04CC026F04DC027F04EC028F01D
:105FF8004FC029F050C02AF051C02BF052C02CF0ED
:1060080053C02DF095BF01D0969395BF05D09551FB
:1060180007E19405D8B004D0376A010E366E04D073
:1060280094C136F095C137F092C140F093C141F068
:1060380096A904D0FE0E4026FF0E412225C038F056
:1060480026C039F027C03AF028C03BF029C03CF000
:106058002AC03DF02BC03EF02CC03FF0436A1F0E13
:10606800426E02019F6B6DD04206D8A043060F0E08
:106078003814446E456A45BE08D0455004E10A0EFE
:10608800445CD8A002D0570E01D0300E4426000E32
:106098004522BF0E2E6E2F682D50306E316A2E505D
:1060A80030262F503122315005E11A0E305C02E2C1
:1060B800010E01D0000E326E336A32503310D8B45C
:1060C80025D09F0E2E6E2F68200E4410306E000EC5
:1060D8004510316E2E5030262F503122315005E1B7
:1060E8001A0E305C02E2010E01D0000E346E356AE1
:1060F80034503510D8B40AD044C011F045C012F05D
:10610800A3EC5FF011C044F012C045F0800E4224A9
:10611800D96E020E4320DA6E44C0DFFF3606D8A0DF
:1061280037064006D8A04106040E2E6ED8903F329E
:106138003E323D323C323B323A32393238322E2E00
:10614800F5D743BE21D0435004E1020E425CD8A0EB
:106158001BD0385039103A103B103C103D103E10FF
:106168003F10D8A481D737BE05D0375002E1360496
:10617800D8B07AD741BE08D0415003E14004D8A036
:1061880003D0010196B370D7010196A916D0420633
:10619800D8A04306800E4224D96E020E4320DA6E40
:1061A8002DC0DFFF4206D8A04306800E4224D96ED8
:1061B800020E4320DA6E300EDF6E24C01AF0800E15
:1061C80042241B6E020E43201C6E40C01DF041C0CD
:1061D8001EF096A108D01BC014F01CC015F01AC000
:1061E80016F076EC61F01EBE05D01DC022F01EC070
:1061F80023F002D0226A236A206A216A0AD0000E9C
:106208000D6E200E0C6E1AC00EF012EC5BF0204AD8
:10621800212A2250205C2150800A1F6E2350800AB8
:106228001F58D8A0ECD7010196B108D01BC014F0B4
:106238001CC015F01AC016F076EC61F01BC00BF00C
:106248001CC00CF007EC60F022500B241A6E23508F
:106258000C201B6E1AC024F01BC025F024C046F089
:1062680025C047F043D04750D96EDA6ADECFF6FF33
:10627800DDCFF7FFF86A000EF86E0800F550250A22
:10628800D8A412D04750D96EDA6ADE2A000EDD2271
:10629800000E0D6E250E0C6E46C00EF012EC5BF073
:1062A800476A010E466E22D04750D96EDA6ADE2A56
:1062B800000EDD22466A476A19D04750D96EDA6A5D
:1062C800DECFF6FFDDCFF7FFF86A000EF86E0800A4
:1062D800F5500C6E0D6A46C00EF012EC5BF047509C
:1062E800D96EDA6ADE2A000EDD22DAD746500101BD
:1062F80090274750912358C0F6FF59C0F7FF080070
:10630800F55001E002D690C154F091C155F0120049
:1063180020EE04F0A351D926A451DA22DECFA7F04B
:10632800DDCFA8F0A729B06F000EA821B16FB0117A
:10633800D8B4040C20EE0EF0A351D926A451DA22C9
:10634800DE50DE10DE10DE1001E1040CB0C0A7F054
:106358000F0EA71701E094D120EE0EF0A351D92615
:10636800A451DA22DE2A000EDE22DE22DE2220EE10
:106378000AF0A351D926A451DA22DE50DE10DE102D
:10638800DE1011E1A3C0D9FFA4C0DAFF10EE08F0B7
:10639800DE50E126DD50E222E650B05DE650B1590C
:1063A80001E26ED1040CB0C0A7F0B1C0A8F0040E91
:1063B800A96FD890A833A733A92FFBD7AA69AB69CF
:1063C800A3C0D9FFA4C0DAFF10EE02F0DE50E12628
:1063D800DD50E222E750AC6FAD6BAA51AC27AB5150
:1063E800AD23A751AC17A851AD17AC51AD1101E0C1
:1063F80047D1A3C0D9FFA4C0DAFFDECF44F0DDCF78
:1064080045F020EE0AF0A351D926A451DA22DECFB6
:1064180046F0DECF47F0DECF48F0DECF49F058EC4B
:106428002BF044C0B2F045C0B3F046C0B4F047C04A
:10643800B5F00001B551B411B31104E1020EB25D1B
:1064480001E2020CB22907E1B32905E1B42903E10D
:10645800B52901E1010CA3C0D9FFA4C0DAFF10EEF1
:1064680012F0DE50E126DD50E222E650B25DE65041
:10647800B359E650B459E650B55901E2D2D0A55106
:10648800A61101E1040CA3C0D9FFA4C0DAFFDECF36
:106498008CF0DDCF8DF020EE0AF0A351D926A4515F
:1064A800DA22DECF8EF0DECF8FF0DECF90F0DECFB7
:1064B80091F047EC3DF08CC0B2F08DC0B3F08EC0C7
:1064C800B4F08FC0B5F0B251B311B411B51101E1F8
:1064D800070CB205B311B411B51101E1020CB229D0
:1064E80007E1B32905E1B42903E1B52901E1010C6C
:1064F800A3C0D9FFA4C0DAFFDECF24F0DDCF25F09A
:1065080021EC4FF0000901E0010CA3C0D9FFA4C0A1
:10651800DAFFDECFA7F0DDCFA8F02E0E0001A72509
:106528000B6E000EA8210C6E0E6A0D6A020E106E1C
:106538000F6AFAEC61F0A3C0D9FFA4C0DAFFDECF7E
:106548000BF0DDCF0CF0B2C00DF0B3C00EF0B4C04C
:106558000FF0B5C010F0A8EC52F0A3C0D9FFA4C04A
:10656800DAFF10EE2AF0DE50E126DD50E2220BC001
:10657800E6FF0CC0E6FF0DC0E6FF0EC0E6FF000117
:10658800AE6BAF6B2BD0A3C0D9FFA4C0DAFF10EE5F
:1065980004F0DE50E126DD50E222010EE76EA3C0D2
:1065A800D9FFA4C0DAFFDECF24F0DDCF25F021EC3F
:1065B8004FF0000901E0010CA3C0D9FFA4C0DAFF25
:1065C80010EE2AF0DE50E126DD50E222E62A000E27
:1065D800E622E622E6220001AE4BAF2BA3C0D9FF8C
:1065E800A4C0DAFF10EE02F0DE50E126DD50E22210
:1065F800E750A76FA86BA751AE5DA851AF59C3E389
:10660800A3C0D9FFA4C0DAFF10EE2AF0DE50E126BD
:10661800DD50E222AE51E65EAF51E65A000EE65A70
:10662800E65A20EE0AF0A351D926A451DA22B2C0C4
:10663800DEFFB3C0DEFFB4C0DEFFB5C0DEFFA3C01F
:10664800D9FFA4C0DAFFDECF0BF0DDCF0CF0B2C06B
:106658000DF0B3C00EF0B4C00FF0B5C010F0A8EC48
:1066680052F0000120EE0EF0A351D926A451DA22EF
:106678000BC0DEFF0CC0DEFF0DC0DEFF0EC0DEFF6C
:1066880020EE04F0A351D926A451DA22B0C0DEFFCF
:10669800B1C0DDFF0F0EB015A76FA86B050ED8901F
:1066A800A737A837E82EFBD7A3C0D9FFA4C0DAFFC5
:1066B800DECFA9F0DDCFAAF0A751A927A851AA23B8
:1066C8002E0EA927000EAA2320EE12F0A351D926D8
:1066D800A451DA22A9C0DEFFAAC0DDFF000C000E1B
:1066E800626E020E636E8E0E646E0A0E656E020E88
:1066F800676E666ADD0E686E696A88EC18F06C6E03
:10670800330E0001806FFD0E816FDDC082F0DEC0A8
:1067180083F0B7EC62F00001DF6BE06BDB6BDC6BE6
:10672800E16BE26BE151BD0FD96EDA6ADF6AE151C4
:10673800CC0FD96EDA6A000EDF6EE14BE22BE2BFB6
:10674800F1D7E25103E10F0EE15DECE3E36BE46B9B
:106758002DD18E0EE325D96E0A0EE421DA6E0D0EC8
:10676800DE1801E0E8D0000E806F040E816F960EEF
:10677800826FFE0E836FBD0E846F856BCC0E866FA5
:10678800876BB7EC62F07A0E0B6EFF0E0C6EBD0EC7
:106798000D6EF4EC59F00B500C1007E1CC0E126E94
:1067A800B1EC53F012500101E96F740E0B6EFF0E3D
:1067B8000C6EBD0E0D6EF4EC59F00B500C1007E189
:1067C800CC0E126EB1EC53F012500101B56F370EBA
:1067D8000B6EFF0E0C6EBD0E0D6EF4EC59F00B50E7
:1067E8000C1007E1CC0E126EB1EC53F012500101FF
:1067F800AC6FD10E0B6EFF0E0C6EBD0E0D6EF4EC71
:1068080059F00B500C1006E1CC0E126EB1EC53F09F
:106818001250726E0001E56BE66BAE0E5A6E5B6A43
:106828003E0E5C6EFF0E5D6EE5C05EF0E6C05FF08A
:10683800BEEC60F0AE0E0B6E0C6ABD0E0D6EF4EC85
:1068480059F00B500C1018E10F0E0001E503F3CFBF
:10685800ACF0F4CFADF0E603F350AD278E0EAC25C7
:106868000B6E0C0EAD210C6ECC0E0D6E0E6A106AFE
:106878000F0E0F6E5FEC5EF00001E54BE62BE6BFF6
:10688800CCD7E65103E1100EE55DC7E3E66B010ED8
:10689800E56FAE0E5A6E5B6A450E5C6EFF0E5D6E5E
:1068A800E5C05EF0E6C05FF0BEEC60F0AE0E0B6EC9
:1068B8000C6ABD0E0D6EF4EC59F00B500C1018E17B
:1068C8000F0E0001E503F3CFACF0F4CFADF0E60313
:1068D800F350AD277E0EAC250B6E0D0EAD210C6E60
:1068E800CC0E0D6E0E6A106A0F0E0F6E5FEC5EF026
:1068F8000001E54BE62BE6BFCCD7E65103E1040ED9
:10690800E55DC7E3E16BE26BE151BD0FD96EDA6A71
:10691800DF6AE151CC0FD96EDA6A000EDF6EE14B07
:10692800E22BE2BFF1D7E25103E10F0EE15DECE3A8
:10693800DB6BDC6B15D08E0EE325D96E0A0EE421D5
:10694800DA6E0A0EDE1830E08E0EE325D96E0A0ED6
:10695800E421DA6E200EDE1806E1DC6B010EDB6F37
:10696800DF6BE06B21D0DB51DC1109E08E0EE325F3
:10697800D96E0A0EE421DA6EDF51CC0F08D08E0EE4
:10698800E325D96E0A0EE421DA6EDF51BD0FE16E00
:10699800E26ADFCFE7FFE0BF05D0E05105E10F0E67
:1069A800DF5D02E2DF4BE02BE34BE42BDD51E35DDF
:1069B800DE51E45901E2CDD6230E806FFD0E816FC2
:1069C800ACC182F0836BB7EC62F0900E0001806F6F
:1069D800FD0E816FE9C182F0836BB7EC62F0810E26
:1069E8000001806FFD0E816FB5C182F0836BB7EC3B
:1069F80062F00001E56BE66BAF0E806FFC0E816FF5
:106A0800E5C082F0E6C083F00F0EE503F3CFACF0EB
:106A1800F4CFADF0E603F350AD278E0EAC25846FAE
:106A28000C0EAD21856FB7EC62F00001E54BE62B4B
:106A3800E6BFE2D7E65103E1100EE55DDDE3E46B66
:106A4800010EE36FC00E806FFC0E816FE3C082F011
:106A5800E4C083F00F0EE303F3CFACF0F4CFADF056
:106A6800E403F350AD277E0EAC25846F0D0EAD21E7
:106A7800856FB7EC62F00001E34BE42BE4BFE2D78B
:106A8800E45103E1040EE35DDDE3DC0E806FFB0EF1
:106A9800816FB7EF62F0200E0001806FF50E816FF5
:106AA800CFCF82F0836BCECF84F0856B73500C0D03
:106AB800500EF324D96E010EF420DA6EDECF86F084
:106AC800DDCF87F073500C0D520EF324D96E010EF2
:106AD800F420DA6EDF50886F896B73500C0D530EFB
:106AE800F324D96E010EF420DA6EDF508A6F8B6BB7
:106AF80073500C0D5B0EF324D96E010EF420DA6E80
:106B0800DF500101B66F73500C0D520EF324D96E8D
:106B1800010EF420DA6EDF50B603F3CFB7F1F4CFED
:106B2800B8F173500C0D5A0EF324D96E010EF420EF
:106B3800DA6EDF50B96FB9C1BAF1BB6BBC6BBD6B14
:106B480073500C0D5B0EF324D96E010EF420DA6E2F
:106B5800DF50BE6FBEC1BFF1C06BC16BC26B73505B
:106B68000C0D500EF324D96E010EF420DA6EDECF30
:106B7800C3F1DDCFC4F1C3C1C5F1C4C1C6F1000E74
:106B8800C6BFFF0EC76FC86FC551BF03F3CFC9F1AA
:106B9800F4CFCAF1CB6BCC6BC003F350CA27F450C7
:106BA800CB23000ECC23C651BF03F350CA27F450A1
:106BB800CB23000ECC23C551C103F350CB27F4508F
:106BC800CC23C651C003F350CB27F450CC23C75174
:106BD800BF03F350CB27F450CC23C251C503F35065
:106BE800CC27C651C103F350CC27C751C003F3507B
:106BF800CC27C851BF03F350CC27C951BA03F3CFF0
:106C0800CDF1F4CFCEF1CF6BD06BBB03F350CE27D1
:106C1800F450CF23000ED023CA51BA03F350CE2725
:106C2800F450CF23000ED023C951BC03F350CF2713
:106C3800F450D023CA51BB03F350CF27F450D023CC
:106C4800CB51BA03F350CF27F450D023BD51C90319
:106C5800F350D027CA51BC03F350D027CB51BB0304
:106C6800F350D027CC51BA03F350D027B751CD25D4
:106C7800D16FB851CE21D26F000ECF21D36F000E45
:106C8800D021D46F73500C0D530EF324D96E010E1E
:106C9800F420DA6EDF50D12500018C6F000E01015F
:106CA800D22100018D6F000E0101D32100018E6FEA
:106CB800000E0101D42100018F6FB7EC62F08980CA
:106CC800DBEC5BF05AC0D6F15BC0D7F1040E0101D2
:106CD800D75D07E3000ED625D86FFC0ED721D96FF4
:106CE80004D0D6C1D8F1D7C1D9F1725054E073504D
:106CF8000C0D540EF324D96E010EF420DA6E8CC1FB
:106D0800BBF18DC1BCF18EC1BDF1BA6B000EBA25C5
:106D1800BE6F010EBB21BF6F000EBC21C06F000EFD
:106D2800BD21C16FDE50BE1936E1DE50BF1933E117
:106D3800DE50C01930E1DE50C1192DE101C3DDF18B
:106D480003C3DCF105C3DBF107C3DAF1DAC10EF0E6
:106D5800DBC10FF0DCC110F0DDC111F008EC5FF011
:106D6800720E0001806FF50E816F2AEE8EF0DF50F3
:106D7800826F836B2AEE8FF0DF50846F856B2AEE6B
:106D880090F0DF50866F876B2AEE91F0DF50886FA6
:106D9800896BB7EC62F082B418D07350200D000EE6
:106DA800F3240001A36F020EF420A46F000EA56F58
:106DB800030EA66F010EA86FA76BD80EA96F010E60
:106DC800AA6FCCEC0EF00101D56F0101D5510AE094
:106DD800530E0001806FFD0E816FD5C182F0836B69
:106DE800B7EC62F0000E0001A66F030EA76F010E4C
:106DF800A96F000EA86F610EAA6FFF0EAB6F12ECA1
:106E080048F0710E0001806FFA0E816FD8C182F0D0
:106E1800D9C183F0B7EC62F00BEC27F0B46B899022
:106E2800E20E0001806FFC0E816FCFCF82F0836B82
:106E3800CECF84F0856BB7EF62F00101D76B980E67
:106E48000001806FF50E816F73500C0D500EF32406
:106E5800D96E010EF420DA6EDECF82F0DDCF83F03A
:106E680073500C0D520EF324D96E010EF420DA6E15
:106E7800DF50846F856B73500C0D530EF324D96E5D
:106E8800010EF420DA6EDF50866F876B73500C0D9D
:106E98005B0EF324D96E010EF420DA6EDF50010187
:106EA800B66F73500C0D520EF324D96E010EF420F8
:106EB800DA6EDF50B603F3CFB7F1F4CFB8F1735001
:106EC8000C0D5A0EF324D96E010EF420DA6EDF5041
:106ED800B96FB9C1BAF1BB6BBC6BBD6B73500C0D0C
:106EE8005B0EF324D96E010EF420DA6EDF50BE6F0C
:106EF800BEC1BFF1C06BC16BC26B73500C0D500E9D
:106F0800F324D96E010EF420DA6EDECFC3F1DDCFA3
:106F1800C4F1C3C1C5F1C4C1C6F1000EC6BFFF0E9E
:106F2800C76FC86FC551BF03F3CFC9F1F4CFCAF11A
:106F3800CB6BCC6BC003F350CA27F450CB23000EA5
:106F4800CC23C651BF03F350CA27F450CB23000EFD
:106F5800CC23C551C103F350CB27F450CC23C651E1
:106F6800C003F350CB27F450CC23C751BF03F350D1
:106F7800CB27F450CC23C251C503F350CC27C651BC
:106F8800C103F350CC27C751C003F350CC27C851D5
:106F9800BF03F350CC27C951BA03F3CFCDF1F4CFD7
:106FA800CEF1CF6BD06BBB03F350CE27F450CF2379
:106FB800000ED023CA51BA03F350CE27F450CF2382
:106FC800000ED023C951BC03F350CF27F450D0236F
:106FD800CA51BB03F350CF27F450D023CB51BA0387
:106FE800F350CF27F450D023BD51C903F350D02715
:106FF800CA51BC03F350D027CB51BB03F350D02761
:10700800CC51BA03F350D027B751CD25D16FB85121
:10701800CE21D26F000ECF21D36F000ED021D46FB6
:1070280073500C0D530EF324D96E010EF420DA6E52
:10703800DF50D1250001886F000E0101D221000127
:10704800896F000E0101D32100018A6F000E010132
:10705800D42100018B6FB7EC62F08980A2D0DBEC01
:107068005BF05AC0D5F15BC0D6F1040E0101D65DC4
:1070780003E3010ED76F03D0D8C1D9F1DA6B82B41C
:1070880018D07350200D000EF3240001A36F020ED8
:10709800F420A46F000EA56F030EA66F010EA86F53
:1070A800A76BD90EA96F010EAA6FCCEC0EF00101E7
:1070B800D86FD8510AE0530E0001806FFD0E816F22
:1070C800D8C182F0836BB7EC62F0000E0001A66FA6
:1070D800030EA76F010EA96F000EA86F610EAA6FAD
:1070E800FF0EAB6F12EC48F072504DE073500C0D70
:1070F800540EF324D96E010EF420DA6E8CC1BBF164
:107108008DC1BCF18EC1BDF10101BA6B000EBA256B
:10711800BE6F010EBB21BF6F000EBC21C06F000EF9
:10712800BD21C16FDE50BE192EE1DE50BF192BE123
:10713800DE50C01928E1DE50C11925E101C3DEF196
:1071480003C3DDF105C3DCF107C3DBF1DBC10EF0DE
:10715800DCC10FF0DDC110F0DEC111F008EC5FF00A
:10716800720E0001806FF50E816F00C382F0836B91
:1071780001C384F0856B02C386F0876B03C388F074
:10718800896BB7EC62F0550E0001806FF90E816FC4
:10719800D9C182F0DAC183F0B7EC62F00BEC27F0CA
:1071A800B46B0101D75101E15AD78990120043C04D
:1071B80024F044C025F021EC4FF04D6E4D5001E015
:1071C8008ED143C0D9FF44C0DAFF030EDE1801E0B8
:1071D80076D120EE05F04350D9264450DA22DE0459
:1071E80001E06DD12E0E43240B6E000E44200C6E70
:1071F8000E6A0D6A020E106E0F6AFAEC61F022EE4A
:107208002CF04350D9264450DA22550EDF6E22EE78
:107218002DF04350D9264450DA22AA0EDF6E20EE14
:107228002EF04350D9264450DA22520EDF6E20EE5B
:107238002FF04350D9264450DA22520EDF6E20EE4A
:1072480030F04350D9264450DA22610EDF6E20EE2A
:1072580031F04350D9264450DA22410EDF6E22EE37
:1072680012F04350D9264450DA22720EDF6E22EE15
:1072780013F04350D9264450DA22720EDF6E22EE04
:1072880014F04350D9264450DA22410EDF6E22EE24
:1072980015F04350D9264450DA22610EDF6E20EEF5
:1072A8000EF04350D9264450DA2212EE16F043501D
:1072B800E1264450E222DFCFE7FF22EE17F04350E9
:1072C800D9264450DA2210EE0EF04350E1264450FD
:1072D800E222E6CF45F0E5CF46F046C045F0466AE3
:1072E8004550DF6E22EE18F04350D9264450DA227A
:1072F80010EE0EF04350E1264450E222E6CF45F06E
:10730800E6CF46F0E6CF47F0E6CF48F0110E05D0BD
:10731800D8904832473246324532E82EF9D74550A0
:10732800DF6E22EE19F04350D9264450DA2210EECF
:107338000EF04350E1264450E222E6CF45F0E6CF76
:1073480046F0E6CF47F0E6CF48F0190E05D0D890C2
:107358004832473246324532E82EF9D74550DF6E7B
:1073680020EE0AF04350D9264450DA2212EE1AF0E1
:107378004350E1264450E222DFCFE7FF22EE1BF024
:107388004350D9264450DA2210EE0AF04350E12641
:107398004450E222E6CF45F0E5CF46F046C045F03E
:1073A800466A4550DF6E22EE1CF04350D926445001
:1073B800DA2210EE0AF04350E1264450E222E6CFEA
:1073C80045F0E6CF46F0E6CF47F0E6CF48F0110E9D
:1073D80005D0D8904832473246324532E82EF9D7A0
:1073E8004550DF6E22EE1DF04350D9264450DA2274
:1073F80010EE0AF04350E1264450E222E6CF45F071
:10740800E6CF46F0E6CF47F0E6CF48F0190E05D0B4
:10741800D8904832473246324532E82EF9D745509F
:10742800DF6E20EE1AF04350D9264450DA22DECF20
:1074380045F0DECF46F0DECF47F0DECF48F04528F6
:10744800496E000E46204A6E000E47204B6E000E15
:1074580048204C6E20EE2AF04350D9264450DA22B8
:1074680049C0DEFF4AC0DEFF4BC0DEFF4CC0DEFF76
:107478002E0E43241A6E000E44201B6E20EE2AF0B6
:107488004350D9264450DA22DECF1CF0DECF1DF05F
:10749800DECF1EF0DECF1FF0216A010E206E20EE37
:1074A80001F04350D9264450DA22DF50B1EC54F0B1
:1074B80020EE05F04350D9264450DA22DF6A1A6AD2
:1074C8001B6A1C6A20EE01F04350D9264450DA2288
:1074D800DF506EEC2DF0000902E0010E4D6E4D50AC
:1074E800120089806B6A740E0001806FF60E816F3E
:1074F800CFCF82F0836BCECF84F0856B7350140DA1
:10750800070EF324D96E010EF420DA6EDECF86F072
:10751800DECF87F0DECF88F0DECF89F07350140D10
:10752800070EF324D96E010EF420DA6EDECF8AF04E
:10753800DECF8BF0DECF8CF0DECF8DF0B7EC62F0D3
:107548001DEC4AF0CAC0BEF1CBC0BFF10101BE516B
:10755800BF1105E0BEC1F0F0BFC1F1F01200716AC1
:10756800BA6BBB6BBC6BBD6BB86B010EB76FC26BF4
:107578000FD1C06BC16B1CD0F2EC62F00B500C1039
:1075880013E0C20E0B6E010E0C6ECDEC5AF0010129
:10759800B66F000E7124D96EDA6A030EDA22B6C10C
:1075A800DFFF712AC04BC12B0101C2AB81AC04D0F3
:1075B800C1BFE2D7C105E0E3C0C1F2F0C1C1F3F039
:1075C800000E0001F3BFFF0EF46FF56FF2510101D9
:1075D800BA270001F3510101BB230001F451010155
:1075E800BC230001F5510101BD237350140D0F0E8A
:1075F800F324D96E010EF420DA6EDE50BA5DDE5047
:10760800BB59DE50BC59DE50BD5902E3B76BB86BAD
:10761800C2AB02D0B76BB86B81BC02D0B76BB86B8A
:1076280071500EE08A0E0001806FFA0E816FBEC1A4
:1076380082F0BFC183F071C084F0856BB7EC62F053
:107648000101C1BF02D0C10519E2000E71240B6E01
:107658000C6A030E0C22FF0E7124D96EDA6A020E30
:10766800DA22DF500D6E0E6A715000080F6E000EA0
:10767800D8A0E82A0108106E5AEC50F072505DE06C
:1076880073505BE17350140D070EF324D96E010E8D
:10769800F420DA6E8CC1F7F08DC1F8F08EC1F9F0E4
:1076A8000001F66B000EF625FA6F010EF721FB6F4D
:1076B800000EF821FC6F000EF921FD6FDE50FA195B
:1076C8003CE1DE50FB1939E1DE50FC1936E1DE50B1
:1076D800FD1933E101C3C6F103C3C5F105C3C4F104
:1076E80007C3C3F1C3C10EF0C4C10FF0C5C110F088
:1076F800C6C111F008EC5FF0670E0001806FF40E50
:10770800816FCFCF82F0836BCECF84F0856B2AEE6A
:107718008EF0DF50866F876B2AEE8FF0DF50886F10
:10772800896B2AEE90F0DF508A6F8B6B2AEE91F00E
:10773800DF508C6F8D6BB7EC62F018EC52F0E151B2
:107748000101B96FB95124E0BA0E0001806FFA0E39
:10775800816FB9C182F0836BB7EC62F0010E6B6E7A
:107768007350140D130EF324D96E010EF420DA6E43
:107778007350140D130EF324E16E010EF420E26E23
:10778800E7500409DF6E6BC0F0F00001F16B1200E6
:10779800B751B81101E0EDD64C0E0001806FF50E1F
:1077A800816FCFCF82F0836BCECF84F0856BBAC167
:1077B80086F0BBC187F0BCC188F0BDC189F0B7ECC9
:1077C80062F082A402D0010E6B6E89900001F06B0A
:1077D800F16B12001550D96EDA6ADECF22F0DDCFD8
:1077E80023F002D0224A232A22C0F6FF23C0F7FF43
:1077F800000EF86E0F0EF76403D00800F55005D0A0
:10780800F6CFE9FFF7CFEAFFEF502F0AEBE022C0EF
:10781800F6FF23C0F7FF000EF86E0F0EF76403D0D3
:107828000800F55005D0F6CFE9FFF7CFEAFFEF5093
:107838005C0AD8E020EE14F01350D9261450DA224E
:10784800DECF24F0DDCF25F024C00BF025C00CF0EE
:107858000E6A200E0D6E106A0B0E0F6EFAEC61F0B8
:107868001E6A1EC026F0276A26C01CF027C01DF01D
:10787800206A080E1F6E1C502224166E1D502320ED
:10788800176E16C0F6FF17C0F7FF000EF86E0F0E42
:10789800F76403D00800F55005D0F6CFE9FFF7CF1D
:1078A800EAFFEF50286E1C4A1D2A200E2864A7D034
:1078B8002F0E281801E1A3D05C0E281801E19FD0F3
:1078C8002E0E281805E01F50265C2050275814E378
:1078D800080E1F182010D8A4060C2E0E281801E038
:1078E800060C276A080E266E206A0B0E1F6ED890AB
:1078F8001E36D8901E36BFD77F0E286402D0030EDE
:107908001E12800E286403D09F0E286406D0DF0E56
:1079180028644CD0FD0E286049D01C502224166ED5
:107928001D502320176E16C0F6FF17C0F7FF000E74
:10793800F86E0F0EF76403D00800F55005D0F6CFA7
:10794800E9FFF7CFEAFFEF50216E1C4A1D2A3F0ED0
:10795800216403D07E0E216406D07F0E2164060CBC
:10796800FD0E2160060C166817681FC018F020C0AD
:1079780019F016501826175019221850265C19505D
:10798800275801E3060C26502424D96E27502520B9
:10799800DA6E28C0DFFF264A272A26502424D96E0B
:1079A80027502520DA6E21C0DFFF26D0CC0E0B6EC3
:1079B800FD0E0C6E28C00DF00E6AA2EC60F00B50A4
:1079C8000C1001E0060C400E286405D05B0E286000
:1079D80002D01E8209D0600E286406D07B0E286073
:1079E80003D01E80200E285E26502424D96E2750EE
:1079F8002520DA6E28C0DFFF264A272A3CD71C50EC
:107A08002224166E1D502320176E1550D96EDA6A7F
:107A180016C0DEFF17C0DDFF200E286403D01A6AE7
:107A28001B6A03D01B6A040E1A6E1AC028F026506F
:107A3800271001E1060C24C0D9FF25C0DAFFE50EA6
:107A4800DE1806E124C0D9FF25C0DAFF050EDF6E77
:107A5800080E1F18201004E1D8901E36D8901E3644
:107A68001E50030BE80601E128881E500C0B040A7F
:107A780001E1288620EE0BF02450D9262550DA2281
:107A880028C0DFFF000C8E518F119011911128E151
:107A980020EE0AF08C51D9268D51DA22DECF97F0EC
:107AA800DECF98F0DECF99F0DECF9AF0975198119B
:107AB80099119A110FE020EE12F08C51D9268D51B0
:107AC800DA22DE50975DDE509859DE509959DE5023
:107AD8009A5952E3010E976F986B996B9A6B4CD039
:107AE8008CC044F08DC045F08EC046F08FC047F082
:107AF80090C048F091C049F058EC2BF044C09FF07A
:107B080045C0A0F046C0A1F047C0A2F00001A251B4
:107B1800A111A01109E1020E9F5D06E2010E8C6F12
:107B28008D6B8E6B8F6B000C9F290FE1A0290DE1E7
:107B3800A1290BE1A22909E19FC08CF0A0C08DF01A
:107B4800A1C08EF0A2C08FF0120020EE12F08C516E
:107B5800D9268D51DA22DE509F5DDE50A059DE50C5
:107B6800A159DE50A259E8E38EC097F08FC098F073
:107B780090C099F091C09AF097C09BF098C09CF083
:107B880099C09DF09AC09EF09B2B000E9C239D23CC
:107B98009E2320EE12F08C51D9268D51DA22DE5028
:107BA8009B5DDE509C59DE509D59DE509E5911E375
:107BB800020E9B6F9C6B9D6B9E6B9A51991198114D
:107BC80008E1020E975D05E28C6B8D6B8E6B8F6BF7
:107BD80012008CC044F08DC045F09BC046F09CC09C
:107BE80047F09DC048F09EC049F058EC2BF044C0C7
:107BF8009FF045C0A0F046C0A1F047C0A2F0000128
:107C08009F51A011A111A2111AE09F2906E1A029F4
:107C180004E1A12902E1A2298FE09F05A011A11189
:107C2800A2118AE097519B19AFE198519C19ACE1D8
:107C380099519D19A9E19A519E19C6E0A5D78CC002
:107C480044F08DC045F09BC046F09CC047F09DC0F5
:107C580048F09EC049F04A684B684C680F0E4D6E5C
:107C680066EC22F0966F96511CE18E518F1190119F
:107C7800911117E08CC044F08DC045F08EC046F0DD
:107C88008FC047F090C048F091C049F09BC04AF0BF
:107C98009CC04BF09DC04CF09EC04DF066EC22F0AD
:107CA800966F965130E120EE0AF08C51D9268D510D
:107CB800DA229BC0DEFF9CC0DEFF9DC0DEFF9EC0B7
:107CC800DEFF20EE0EF08C51D9268D51DA22DE2807
:107CD80006E1DE2804E1DE2802E1DE2821E020EECC
:107CE8000EF08C51D9268D51DA22DE06000EDE5AAE
:107CF800DE5ADE5A20EE05F08C51D9268D51DA2253
:107D0800000EDB800DD0960507E0010E9B6F000E7C
:107D18009C6B9D6B9E6B04D09B699C699D699E6959
:107D28009BC08CF09CC08DF09DC08EF09EC08FF0E3
:107D380012002D0E0001806FF60E816F73500C0D2E
:107D4800500EF324D96E010EF420DA6EDECF82F0E5
:107D5800DDCF83F073500C0D520EF324D96E010E53
:107D6800F420DA6EDF50846F856B73500C0D530E60
:107D7800F324D96E010EF420DA6EDF50866F876B1C
:107D880073500C0D5B0EF324D96E010EF420DA6EDD
:107D9800DF50AC6F73500C0D520EF324D96E010EE8
:107DA800F420DA6EDF50AC03F3CFADF0F4CFAEF0D1
:107DB80073500C0D5A0EF324D96E010EF420DA6EAE
:107DC800DF50AF6FAFC0B0F0B16BB26BB36B735035
:107DD8000C0D5B0EF324D96E010EF420DA6EDF5021
:107DE800B46FB4C0B5F0B66BB76BB86B73500C0D0D
:107DF800500EF324D96E010EF420DA6EDECFB9F0FE
:107E0800DDCFBAF0B9C0BBF0BAC0BCF0000EBCBF41
:107E1800FF0EBD6FBE6FBB51B503F3CFBFF0F4CFFC
:107E2800C0F0C16BC26BB603F350C027F450C12336
:107E3800000EC223BC51B503F350C027F450C12330
:107E4800000EC223BB51B703F350C127F450C2231D
:107E5800BC51B603F350C127F450C223BD51B5033A
:107E6800F350C127F450C223B851BB03F350C227C3
:107E7800BC51B703F350C227BD51B603F350C22714
:107E8800BE51B503F350C227BF51B003F3CFC3F0BF
:107E9800F4CFC4F0C56BC66BB103F350C427F450DC
:107EA800C523000EC623C051B003F350C427F450B5
:107EB800C523000EC623BF51B203F350C527F450A3
:107EC800C623C051B103F350C527F450C623C1518E
:107ED800B003F350C527F450C623B351BF03F35082
:107EE800C627C051B203F350C627C151B103F3509E
:107EF800C627C251B003F350C627AD51C325C76F7B
:107F0800AE51C421C86F000EC521C96F000EC6212D
:107F1800CA6F73500C0D530EF324D96E010EF42062
:107F2800DA6EDF50C725886F000EC821896F000EF2
:107F3800C9218A6F000ECA218B6FB7EC62F0898065
:107F48000001D06BD16BD26BD36B7350200D000E38
:107F5800F324626E020EF420636E8E0E646E0A0EB7
:107F6800656E010E676E666ACD0E686E696A88EC8A
:107F780018F00001CF6FAF0E806FF80E816FCFC081
:107F880082F0836BCDC084F0CEC085F0B7EC62F090
:107F98000101E793CDC064F0CEC065F0DCEC44F09D
:107FA80064C0CBF065C0CCF00001CB51D027CC51D8
:107FB800D123000ED223D3239D0E806FFC0E816F38
:107FC800D0C082F0D1C083F0D2C084F0D3C085F095
:107FD800B7EC62F00101B46B8990120020EE04F056
:107FE8006250D9266350DA2264C0DEFF65C0DDFF27
:107FF80020EE06F06250D9266350DA22DECF99F0DF
:10800800DECF9AF0DECF9BF0DECF9CF00001990521
:108018009A119B119C11D8B4020C62C0D9FF63C09D
:10802800DAFF10EE12F0DE50E126DD50E222E650D3
:10803800995DE6509A59E6509B59E6509C5901E3E0
:10804800020C99519A119B119C1121E162C0D9FF30
:1080580063C0DAFFDECF8CF0DDCF8DF08CC0D9FFA6
:108068008DC0DAFF030EDE1812E162C0D9FF63C0CB
:10807800DAFF10EE22F0DE50E126DD50E222E6CFF4
:1080880099F0E6CF9AF0E6CF9BF0E6CF9CF09951B5
:108098009A119B119C1123E162C0D9FF63C0DAFFDA
:1080A80010EE08F0DE50E126DD50E222E650645C76
:1080B800E650655801E3020C62C0D9FF63C0DAFFDD
:1080C80010EE22F0DE50E126DD50E222E6CF95F0F8
:1080D800E6CF96F0E6CF97F0E6CF98F074D062C07E
:1080E800D9FF63C0DAFF10EE02F0DE50E126DD5062
:1080F800E222E750100DF3CF93F0F4CF94F044D080
:1081080062C0D9FF63C0DAFFDECF44F0DDCF45F0AF
:1081180099C046F09AC047F09BC048F09CC049F00F
:1081280058EC2BF044C099F045C09AF046C09BF03B
:1081380047C09CF00001992907E19A2905E19B298C
:1081480003E19C2901E1010C9C519B119A1104E166
:10815800020E995DD8A0020C62C0D9FF63C0DAFF95
:1081680010EE12F0DE50E126DD50E222E650995D75
:10817800E6509A59E6509B59E6509C5901E3020C87
:108188009351645E9451655A9351645C9451655857
:10819800B7E262C0D9FF63C0DAFFDECF0BF0DDCFF4
:1081A8000CF099C00DF09AC00EF09BC00FF09CC067
:1081B80010F0A8EC52F00BC095F00CC096F00DC072
:1081C80097F00EC098F020EE0AF06250D92663505E
:1081D800DA2299C0DEFF9AC0DEFF9BC0DEFF9CC09A
:1081E800DEFF0001955196119711981101E1020CDB
:1081F80064C08CF065C08DF0040E8E6FD8908D33FE
:108208008C338E2FFBD78C5195258F6F8D519621EE
:10821800906F000E9721916F000E9821926F20EEBB
:108228000EF06250D9266350DA228FC0DEFF90C06C
:10823800DEFF91C0DEFF92C0DEFF0F0E64148C6F6C
:108248008D6B050ED8908C378D37E82EFBD762C022
:10825800D9FF63C0DAFFDECF8EF0DDCF8FF08C510F
:108268008E278D518F232E0E8E27000E8F2320EE02
:1082780012F06250D9266350DA228EC0DEFF8FC01A
:10828800DDFF000C000E0001F66F0A0EF56F000E00
:10829800F46F050EF36F28D1F66B140EF56F1CD131
:1082A800F30E0C6EFB0E0D6EDEEC5EF082B204D0A7
:1082B8000001F66B1E0EF56F150E0001F26F4B0EE6
:1082C800F16FBE0EE82EFED7F12FFCD7F22FFAD7AA
:1082D80000F002D17E0E0C6EFE0E0D6EDEEC5EF02E
:1082E800600E0001D26F080ED36FDE0ED46FFB0E46
:1082F800D56FD66BA9EC59F06C6E6C5031EC5FF011
:108308006C50DAE10001F66B230ED5D79F0E0C6E88
:10831800FD0E0D6EDEEC5EF0000E0001D26F020E57
:10832800D36FC50ED46FFE0ED56F010ED66FA1ECBC
:108338001DF06C6E6C5031EC5FF06C5009E173EC21
:1083480033F0000E5B6E020E5C6E2CEC61F06C6E0E
:108358006C5031EC5FF0000E0001F66F280EF56FDF
:108368000101AC510CE1E86B8E0E5A6E0C0E5B6E7F
:108378003D0E5C6EFE0E5D6EBEEC60F00DD0390EEB
:108388000001806FF80E816FACC182F0836BE8C189
:1083980084F0856BB7EC62F0AE0E0001806FFD0EC5
:1083A800816F0101E8510F0D8E0EF3240001826FD9
:1083B8000C0EF420836FB7EC62F07ED7190E806F35
:1083C800FB0E816F0101E8510F0D8E0EF3240001A1
:1083D800826F0C0EF420836FB7EC62F0000E000180
:1083E800D26F020ED36F0101E8510F0D8E0EF324E8
:1083F8000001D46F0C0EF420D56F030ED66FA1ECDC
:108408001DF06C6E6C5004E10001F66B3C0EF56FCC
:10841800040E6C1801E050D70001F66B320E4BD7F2
:108428008B0E806FFC0E816F0101E8510F0D8E0ECF
:10843800F3240001826F0C0EF420836FB7EC62F016
:10844800000E0001D26F020ED36F0101E8510F0D2B
:108458008E0EF3240001D46F0C0EF420D56F070E96
:10846800D66FA1EC1DF06C6E6C5001E025D70001B1
:10847800F66B3C0E20D72E0E806FFC0E816F01012B
:10848800E8510F0D8E0EF3240001826F0C0EF420BC
:10849800836FB7EC62F00001F06B010EEF6F010C17
:1084A800F5C0F1F0F6C0F2F0F25116E1F1510A0A06
:1084B80001E1F2D61E0A01E1F3D60A0A01E10AD760
:1084C8003D0A01E123D70B0A01E178D7050A04E048
:1084D8001F0AA6E00E0ACFE0140E0001F519F611E6
:1084E80003E0F307D8A0F407F4BF04D0F451D8E1AF
:1084F800F305D6E2EF6BF06B12008E0E0101C26F2E
:108508000A0EC36FEAC00BF0EBC00CF007EC60F08A
:108518000B500101B66FCA0E0001A36FA46BA56BC7
:10852800A66BA76BA86B9EEC15F00101BF6FBF513E
:108538000DE0580E0001806FFA0E816FB7EC62F003
:108548000001CA6BCB6BCC6BCD6B1200CA0E626E8E
:10855800636AC2C164F0C3C165F0010E676E666AE2
:10856800BD0E686E010E696E88EC18F00101BF6FD0
:10857800BF5108E05E0E0001806FFB0E816FB7EC03
:1085880062F0DED7C2C1D9FFC3C1DAFF800EDE18A0
:1085980008E0D10E0001806FFC0E816FB7EC62F02D
:1085A800CFD720EE0AF0C251D926C351DA22DF50C4
:1085B8000001ED6FEC6B010120EE0BF0C251D926E2
:1085C800C351DA22DF500001EC250101BB6F000E18
:1085D8000001ED210101BC6F470E0001806FFB0E09
:1085E800816FBBC182F0BCC183F0B7EC62F0CA0EE8
:1085F8000001A36FA46B0101BB510001ED6FEC6B8F
:10860800ECC0A5F0EDC0A6F0A76BA86B9EEC15F02A
:108618000101BF6FBF5194E1CA0E626E636AC2C1A5
:1086280064F0C3C165F0010E676E666ABD0E686EC0
:10863800010E696E88EC18F00101BF6FBF5180E12F
:10864800C06BC16BEAC00BF0EBC00CF0C0C1ECF022
:10865800C1C1EDF0050ED8900001EC37ED37E82EDA
:10866800FAD7EC510101C2250D6E0001ED5101014F
:10867800C3210E6EB6C10FF0106A3FEC5AF00B50D2
:108688000C105DE1C0C1ECF0C1C1EDF0050ED89051
:108698000001EC37ED37E82EFAD7C2C1EEF0C3C1BE
:1086A800EFF0EC51EE27ED51EF230E0EEE25D96ECB
:1086B800000EEF21DA6EDF50F16FF06BC0C1F2F0FF
:1086C800C1C1F3F0050ED890F237F337E82EFBD787
:1086D800C2C1F4F0C3C1F5F0F251F427F351F52308
:1086E8000F0EF425D96E000EF521DA6EDF50F66F05
:1086F800F76BF051F627F151F723F6C0B7F1F7C041
:10870800B8F10101000EB8BFFF0EB96FBA6FBD0E08
:108718000001806FFD0E816FB7C182F0B8C183F090
:10872800B9C184F0BAC185F0B7EC62F0B7C1CAF03C
:10873800B8C1CBF0B9C1CCF0BAC1CDF01200C04B72
:10874800C12BC1BF7FD7C15105E10F0EC05D01E349
:10875800F7D678D7F5D60001CE6FCA5102E01AECE9
:108768004BF00001CD6BC95101E108D1040ECE19BF
:1087780003E0140ECE1909E10101A76B986B996B00
:108788000001CA6B070EC96F070C3F0ECE1907E12F
:10879800FE6B0101A76B0001C96BCA6B12005F0E6B
:1087A800CE1907E10101A86BA76B0001C96BCA6B61
:1087B80012003F0ECE6506D05F0ECE6103D0400E8C
:1087C800CE19F0E1400ECE190FE1010E0101A86F9C
:1087D800A76B9E0E0001806FFF0E816FB7EC62F0F1
:1087E8000001C96BCA6B1200200ECE190CE1010EF4
:1087F800FE6F0101A76B980E0001806FFF0E816F5D
:10880800B7EC62F0EDD7650ECE1909E1FE5107E02D
:108818000101986B996B010EA76F8980E1D76E0EE5
:10882800CE1903E1020E0101A76F700E0001CE19E7
:1088380007E10101A85104E0986B996B030EA76F3B
:10884800700E0001CE1908E1FE5106E08980010191
:10885800986B996B040E0ED0720ECE1901E08ED073
:10886800FE5101E18BD089801C0E0101996F2A0EFF
:10887800986F050EA76FB4D7CE5129EC0BF0000105
:10888800CD6F91D0B70E806FFB0E816FCEC082F096
:10889800836BB7EC62F089800001CE5199EC5BF0F4
:1088A8000001CD6F0101A76B7ED089801B0E806F00
:1088B800F80E816FCFCF82F0836BCECF84F0856BBB
:1088C8006BC086F0876BB7EC62F08E0E0B6E0A0EEB
:1088D8000C6E0E6A0D6A010E106E0F6A5AEC50F09B
:1088E8000101E7832AEE8EF06BC0DFFF656A010E97
:1088F800646EDCEC44F0E793080ED2D78990CD6B18
:10890800BD0E806FF70E816FCFCF82F0836BCECF15
:1089180084F0856BCEC086F0876BB7EC62F043D0ED
:10892800080ECE1918E11C0E806FF70E816FCFCF9D
:1089380082F0836BCECF84F0856BCEC086F0876BD8
:10894800B7EC62F089900001CD6B6B6A0101A76BEF
:10895800986B996B28D0090ECE1925E1040E806F0B
:10896800F90E816FCFCF82F0836BCECF84F0856B09
:10897800CEC086F0876BB7EC62F0E4D70101A7514F
:108988000001CB6FCC6BCC510EE1CB510CE0010A4E
:1089980001E172D7030A01E175D7010A86E0070AE7
:1089A800ADE0010ABDE0CDC0C9F00001CA6B1200FC
:1089B8000101B16B9A6B9B6B93869380938293842E
:1089C800938895688A908A928A948A98010EB06FE3
:1089D800898E89B409D0BE0E0001806FF50E816FB3
:1089E800B7EC62F00101B06BF2981A0EE82EFED7D0
:1089F80000D007D0FC0E0001806FFF0E816FB7EC2E
:108A080062F081A8F7D78E0E0001A66F0A0EA76F35
:108A180064C0A8F065C0A9F0530EAA6FFF0EAB6F33
:108A280012EC48F0D4D081A881BA14D0570E0001B6
:108A3800806FFE0E816F010E80A0000E826F836B27
:108A4800010E89A0000E846F856BB1C186F0876B1B
:108A5800B7EC62F081A881AA18D001019BBF15D09C
:108A68009B5102E19A0511E395689380540E000129
:108A7800806FFC0E816F9AC182F09BC183F0B7ECC6
:108A880062F0630E0101B16FA8D0100E0101886F6A
:108A9800270E896F8A6B8B6B84D081B281A410D02A
:108AA8008807000E895B8A5B8B5B882906E1892928
:108AB80004E18A2902E18B29D8A489D0620E67D003
:108AC800010E65D0020E63D06668676864C068F0FE
:108AD80065C069F066506826675069229A5168181F
:108AE80005E19B51691802E1E7B3939A8E0E9A2526
:108AF800D96E0A0E9B21DA6EDF1C8C6E9A4B9B2B6B
:108B0800956A030E1ED0100E886F270E896F8A6B28
:108B18008B6B5DD081B20DD08807000E895B8A5BB4
:108B28008B5B882908E1892906E18A2904E18B29D8
:108B380002E1040EB16F81A24AD0040E28D09390AE
:108B4800050EB16FE0D7938481B40DD08807000E6D
:108B5800895B8A5B8B5B882908E1892906E18A2978
:108B680004E18B2902E1060EB16F81A430D0060E14
:108B78000ED0938A9380956864509A5D9B51800AC1
:108B8800666E6550800A66589BE3630E0101B16FFB
:108B98001ED08C0E0001806FFF0E816FB7EC62F063
:108BA800F4D7B151666E676A675011E1665001E10A
:108BB80074D7010A87E0030A87E0010AABE0070AD5
:108BC800BEE0010AC0E0030AD4E0640AE2E0630EF2
:108BD8000101B11902E081BC26D7F292F288B06B8C
:108BE8009380938293849388938A9568899E9AC187
:108BF80064F09BC165F0120020EE04F04450D926C1
:108C08004550DA22DF6A20EE2AF04450D926455032
:108C1800DA22DE68DE68DE68DD6844C039F045C007
:108C28003AF046C03BF047C03CF048C03DF049C070
:108C38003EF05BEC59F0000901E0030C22EE2DF048
:108C48004450D9264550DA22DF504B6E4A6A22EE4C
:108C58002CF04450D9264550DA22DF504A12550EDE
:108C68004A1803E1AA0E4B1801E0020C20EE65F049
:108C78004450D9264550DA22DF504B6E4A6A20EE1E
:108C880066F04450D9264550DA22DF504C6E4CC06D
:108C98004DF04E6A4F6A506A4EC050F04DC04FF0CA
:108CA8004E6A4D6A20EE67F04450D9264550DA22C4
:108CB800DF50516E51C052F0536A546A556A52C01F
:108CC80055F0546A536A526A4D505210566E4E50BF
:108CD8005310576E4F505410586E50505510596ECF
:108CE8004A5056105A6E4B5057105B6E000E581073
:108CF8005C6E000E59105D6E20EE64F04450D9266B
:108D08004550DA22DF505A105E6E5B505F6E5C5041
:108D1800606E5D50616E5E50626E5F50636E605053
:108D2800646E656A460E621808E1410E631805E133
:108D3800540E6418651001E1000C20EE81F04450D7
:108D4800D9264550DA22DF504B6E4A6A20EE82F06F
:108D58004450D9264550DA22DF504C6E4CC04DF0B5
:108D68004E6A4F6A506A4EC050F04DC04FF04E6A7E
:108D78004D6A20EE83F04450D9264550DA22DF5060
:108D8800516E51C052F0536A546A556A52C055F038
:108D9800546A536A526A4D505210566E4E505310D0
:108DA800576E4F505410586E50505510596E4A50C7
:108DB80056105A6E4B5057105B6E000E58105C6E72
:108DC800000E59105D6E20EE80F04450D9264550B3
:108DD800DA22DF505A105E6E5B505F6E5C50606E38
:108DE8005D50616E5E50626E5F50636E6050646E7F
:108DF800656A460E621808E1410E631805E1540ED3
:108E08006418651001E1000C010C4EC00CF04FC055
:108E18000DF086EC5AF0546E545001E0FDD020EE6F
:108E280004F04E50D9264F50DA22DFAAF5D04EC0B2
:108E3800D9FF4FC0DAFFDECF39F0DDCF3AF020EEB0
:108E48001AF04E50D9264F50DA22DECF3BF0DECF53
:108E58003CF0DECF3DF0DECF3EF05BEC59F0546ED7
:108E6800545001E0D9D020EE1EF04E50D9264F5074
:108E7800DA22DECF59F0DDCF5AF020EE0BF0595050
:108E8800D9265A50DA22000EDB8A20EE0AF04E501C
:108E9800D9264F50DA2210EE1CF05950E1265A50CC
:108EA800E222DFCFE7FF20EE1DF05950D9265A50B5
:108EB800DA2210EE0AF04E50E1264F50E222E6CFB9
:108EC80050F0E5CF51F051C050F0516A5050DF6E6C
:108ED80020EE1EF05950D9265A50DA2210EE0AF028
:108EE8004E50E1264F50E222E6CF50F0E6CF51F047
:108EF800E6CF52F0E6CF53F0110E05D0D89053329A
:108F0800523251325032E82EF9D75050DF6E20EEEF
:108F18001FF05950D9265A50DA2210EE0AF04E5056
:108F2800E1264F50E222E6CF50F0E6CF51F0E6CFEF
:108F380052F0E6CF53F0190E05D0D8905332523282
:108F480051325032E82EF9D75050DF6E59C00BF02D
:108F58005AC00CF020EE0EF04E50D9264F50DA22AF
:108F6800DECF0DF0DECF0EF0DECF0FF0DECF10F04B
:108F7800E6EC5FF0556A566A210E576E460E586E3B
:108F880020EE16F05950D9265A50DA22DF6A20EE20
:108F980017F05950D9265A50DA2256C0DFFF20EE72
:108FA80018F05950D9265A50DA2257C0DFFF20EE60
:108FB80019F05950D9265A50DA2258C0DFFF20EE4E
:108FC80012F05950D9265A50DA22DF6A20EE13F0EF
:108FD8005950D9265A50DA22DF6A20EE04F04E5052
:108FE800D9264F50DA22DF0EDF164EC0D9FF4FC008
:108FF800DAFF10EE04F0DE50E126DD50E222010E29
:10900800E76E4EC0D9FF4FC0DAFFDECF43F0DDCFA9
:1090180044F0DBEC38F0546E545012004A0E806F66
:10902800FE0E816FAAC082F0ABC083F0A6C084F0A8
:10903800A7C085F0A8C086F0A9C087F0B7EC62F099
:10904800606A616ACCD0DC0E806FFB0E816FB7EC72
:1090580062F0626A636A28D060C05AF061C05BF04F
:109068005A3A5B3AF00E5B165A500F0B5B12F00E31
:109078005A16A6C05CF0A7C05DF05A505C265B503B
:109088005D2262505C24D96E63505D20DA6EDF5039
:109098005F6E860E806FFF0E816F5FC082F0836BFC
:1090A800B7EC62F0624A632A63BE05D063501EE1E2
:1090B800100E625C1BE260C05AF061C05BF05A3A65
:1090C8005B3AF00E5B165A500F0B5B12F00E5A16F5
:1090D80062505A2663505B225A500001A85DA9517C
:1090E800800A5C6E5B50800A5C58B6E2DD0E0001B7
:1090F800806FFF0E816FB7EC62F0626A636A4BD0D3
:1091080060C05AF061C05BF05A3A5B3AF00E5B16E9
:109118005A500F0B5B12F00E5A16A6C05CF0A7C08F
:109128005DF05A505C265B505D2262505C24D96E1B
:1091380063505D20DA6E200EDF6425D0F90E806F53
:10914800FF0E816F60C05AF061C05BF05A3A5B3A1B
:10915800F00E5B165A500F0B5B12F00E5A16A6C093
:109168005CF0A7C05DF05A505C265B505D226250EF
:109178005C24D96E63505D20DA6EDF50826F836B9A
:10918800B7EC62F006D0C30E806FFE0E816FB7ECAD
:1091980062F0624A632A63BE05D063501EE1100E76
:1091A800625C1BE260C05AF061C05BF05A3A5B3AFD
:1091B800F00E5B165A500F0B5B12F00E5A166250E7
:1091C8005A2663505B225A500001A85DA951800AB3
:1091D8005C6E5B50800A5C5893E2604A612A61BE0B
:1091E80005D061501BE1500E605C18E260C05AF077
:1091F80061C05BF05A3A5B3AF00E5B165A500F0B9F
:109208005B12F00E5A160001A8515A5C5B50800A96
:109218005C6EA951800A5C5801E215D7DC0E00018A
:10922800806FFB0E816FB7EF62F0960E0001806FC2
:10923800F60E816FCFCF82F0836BCECF84F0856B33
:1092480073C086F0876BB7EC62F00101E7838E0E7E
:109258000B6E0A0E0C6E0E6A0D6A010E106E0F6A06
:109268005AEC50F02AEE8EF073C0DFFFFF0EE8CF05
:109278008FFA7350140D130EF324D96E010EF420D7
:10928800DA6EDFA403D0010EE8CF92FA7350140D02
:10929800130EF324D96E010EF420DA6EDFA003D08A
:1092A800020EE8CF94FA7350140D130EF324D96EFE
:1092B800010EF420DA6EDFA203D0020EE8CF94FA92
:1092C8007350140D130EF324D96E010EF420DA6EC8
:1092D800DFA603D0800EE8CF93FA82A403D0080E4D
:1092E800E8CF94FA0001AD6BAE6B5D0E806FF70EA0
:1092F800816FCFCF82F0836BCECF84F0856BADC00A
:1093080086F0AEC087F0900EAD25D96E0A0EAE215C
:10931800DA6EDF50886F896BB7EC62F0800E00015F
:10932800AD25D96E010EAE21DA6EDF1CAC6F900E42
:10933800AD25D96E0A0EAE21DA6E900EAD25E16E1E
:109348000A0EAE21E26EE750AC15DF6E300E806F6C
:10935800FF0E816F900EAD25D96E0A0EAE21DA6E22
:10936800DF50826F836BB7EC62F00001AD4BAE2B20
:10937800AEBFBBD7AE5103E1070EAD5DB6E3735088
:10938800140D130EF324D96E010EF420DA6EDF509B
:109398006B6E7350140D010EF324D96E010EF42078
:1093A800DA6EDF506A6E6AC099FA7350140D020EB5
:1093B800F324D96E010EF420DA6EDF506A6E6AC0AB
:1093C8009AFA7350140D030EF324D96E010EF4208B
:1093D800DA6EDF506A6E6AC09BFA7350140D040E81
:1093E800F324D96E010EF420DA6EDF506A6E6AC07B
:1093F8009CFA7350140D050EF324D96E010EF42057
:10940800DA6EDF506A6E6AC09DFA7350140D060E4C
:10941800F324D96E010EF420DA6EDF506A6E6AC04A
:109428009EFA656A140E646EDCEC44F0E79389904A
:1094380012007350140D070EF324D96E010EF42098
:10944800DA6EDECFDDF0DECFDEF0DECFDFF0DECFAE
:10945800E0F0F30E0001806FF40E816FCFCF82F041
:10946800836BCECF84F0856BDDC086F0DEC087F0DD
:10947800DFC088F0E0C089F0DDC08AF0DEC08BF084
:10948800DFC08CF0E0C08DF0B7EC62F07350140DC3
:10949800070EF324D96E010EF420DA6E7350140D02
:1094A8000B0EF324E16E010EF420E26EDE50E65C52
:1094B800DE50E658DE50E658DE50E6581CE2790EDB
:1094C8000001806FFC0E816FB7EC62F0010E6B6ECD
:1094D8007350140D130EF324D96E010EF420DA6EB6
:1094E8007350140D130EF324E16E010EF420E26E96
:1094F800E7500409DF6E7350140D0F0EF324D96E74
:10950800010EF420DA6EDECFCCF0DECFCDF0DECF68
:10951800CEF0DECFCFF07350140D070EF324D96EC2
:10952800010EF420DA6EDECFD0F0DECFD1F0DECF40
:10953800D2F0DECFD3F00001CC51D025D46FCD517D
:10954800D121D56FCE51D221D66FCF51D321D76F2C
:109558007350140D0B0EF324D96E010EF420DA6E3D
:10956800D451DE5CD551DE58D651DE58D751DE587D
:109578001BE2670E806FFC0E816FB7EC62F0010E84
:109588006B6E7350140D130EF324D96E010EF42074
:10959800DA6E7350140D130EF324E16E010EF420ED
:1095A800E26EE7500409DF6E6B6A7350200D000EFF
:1095B800F3240001A36F020EF420A46FDDC0A5F010
:1095C800DEC0A6F0DFC0A7F0E0C0A8F09EEC15F062
:1095D800DC6FDC5126E0EA0E806FFA0E816FDDC089
:1095E80082F0DEC083F0DFC084F0E0C085F0DCC02C
:1095F80086F0876BB7EC62F0010E6B6E7350140D3A
:10960800130EF324D96E010EF420DA6E7350140D84
:10961800130EF324E16E010EF420E26EE750040904
:10962800DF6E6BC0CAF00001CB6B1200736A736AFD
:10963800030E736401D0E9D0735003E15A6A5B6A80
:1096480003D05B6A010E5A6E7350140D130EF32487
:10965800D96E010EF420DA6EDF6A7350140D000E15
:10966800F324D96E010EF420DA6EDF6A7350140DFC
:10967800070EF324D96E010EF420DA6EDE6ADE6A74
:10968800DE6ADD6A0D0E5A02F3CFA6F0F4CFA7F01A
:109698005B02F3500001A727DB0EA625D96E020E48
:1096A800A721DA6EDF50A86FA8C0A9F0AA6BAB6B30
:1096B800AC6BABC0ACF0AAC0ABF0A9C0AAF0A96B68
:1096C8000D0E5A02F3CFADF0F4CFAEF05B02F350BB
:1096D800AE27DA0EAD25D96E020EAE21DA6EDF5056
:1096E800AF6FAFC0B0F0B16BB26BB36BB1C0B3F0DA
:1096F800B0C0B2F0B16BB06B0D0E5A02F3CFB4F03C
:10970800F4CFB5F05B02F350B527D90EB425D96E66
:10971800020EB521DA6EDF50B66FB6C0B7F0B86B7F
:10972800B96BBA6BB7C0BAF0B96BB86BB76B0D0E43
:109738005A02F3CFBBF0F4CFBCF05B02F350BC2766
:10974800D80EBB25D96E020EBC21DA6EDF50B725C4
:10975800BD6F000EB821BE6F000EB921BF6F000E9D
:10976800BA21C06FB051BD25C16FB151BE21C26FC2
:10977800B251BF21C36FB351C021C46FA951C125D4
:10978800C56FAA51C221C66FAB51C321C76FAC5177
:10979800C421C86F7350140D0B0EF324D96E010E3B
:1097A800F420DA6EC5C0DEFFC6C0DEFFC7C0DEFF2C
:1097B800C8C0DEFF3D0E806FF70E816F73C082F068
:1097C800836B7350140D0B0EF324D96E010EF42025
:1097D800DA6EDECF84F0DECF85F0DECF86F0DECF26
:1097E80087F07350140D0B0EF324D96E010EF4207C
:1097F800DA6EDECF88F0DECF89F0DECF8AF0DECFFA
:109808008BF0B7EC62F0732A13D70101A86B000143
:10981800FE6B0101A76B986B996B020E6B6EA66FBE
:109828008990020C81A605D0C80E0001A66FFB0E18
:1098380004D0B80E0001A66FFF0EA76F81AA04D04E
:10984800C80EA86FFB0E03D0B30EA86FFF0EA96F4A
:1098580081A804D0C80EAA6FFB0E03D0E10EAA6F30
:10986800FE0EAB6F81AE04D0C80EAC6FFB0E03D0FA
:10987800BD0EAC6FFF0EAD6F81AC04D0C80EAE6FDD
:10988800FB0E03D0AE0EAE6FFF0EAF6F81A404D0F7
:10989800C80EB06FFB0E03D0C70EB06FFF0EB16FCE
:1098A80081A204D0C80EB26FFB0E03D0CC0EB26FEB
:1098B800FF0EB36F81A004D0C80EB46FFB0E03D0A7
:1098C800C20EB46FFF0EB56F83AE04D0C80EB66F6C
:1098D800FB0E03D0F60EB66FFF0EB76F83AC04D045
:1098E800C80EB86FFB0E03D0F30EB86FFF0EB96F3A
:1098F80083AA04D0C80EBA6FFB0E03D0F00EBA6F5D
:10990800FF0EBB6F83A804D0C80EBC6FFB0E03D03C
:10991800ED0EBC6FFF0EBD6F83A604D0C80EBE6FE0
:10992800FB0E03D0EA0EBE6FFF0EBF6F83A404D0F8
:10993800C80EC06FFB0E03D0E70EC06FFF0EC16FDD
:1099480083A204D0C80EC26FFB0E03D0E40EC26F10
:10995800FF0EC36F83A004D0C80EC46FFB0E03D0E4
:10996800E10EC46FFF0EC56F800E806FF30E816F1E
:10997800831C826F836B81CF84F0856BC4C086F0B3
:10998800C5C087F0C2C088F0C3C089F0C0C08AF0E3
:10999800C1C08BF0BEC08CF0BFC08DF0BCC08EF0D3
:1099A800BDC08FF0BAC090F0BBC091F0B8C092F0C3
:1099B800B9C093F0B6C094F0B7C095F0B4C096F0B3
:1099C800B5C097F0B2C098F0B3C099F0B0C09AF0A3
:1099D800B1C09BF0AEC09CF0AFC09DF0ACC09EF093
:1099E800ADC09FF0AAC0A0F0ABC0A1F0A8C0A2F083
:1099F800A9C0A3F0A6C0A4F0A7C0A5F0B7EF62F075
:109A08001B6E1B5001E0010C74A202D074501200AE
:109A1800000E70EC62F00A0E266E03D0E5EC62F0E0
:109A280026062650FBE1236A000E146A156A166A98
:109A3800176ADAEC60F0E80601E097D0AA0E146E17
:109A4800010E156E166A176A080EDAEC60F0E80661
:109A580051E1266A26501C0FD96EDA6AE5EC62F0ED
:109A6800DF6E262A030E2664F5D71E047EE1AA0EB1
:109A78001F187BE1030E256EE80E246E15D0146ABC
:109A8800156A166A400E176EA90EDAEC60F0000926
:109A98000EE00B0E1A6E620EE82EFED71A2EFCD7B9
:109AA80000D02406D8A0250624502510E8E124502B
:109AB80025105BE0146A156A166A176A3A0EDAEC22
:109AC80060F0000952E1266A26501C0FD96EDA6A46
:109AD800E5EC62F0DF6E262A030E2664F5D71CBC7F
:109AE80003D0216A040E02D0216A0C0E206E20C019
:109AF80023F03BD0146A156A166A176AA90EDAECC5
:109B080060F01A6E020E1A6003D0236EA90E02D0FE
:109B1800010E236E226E030E256EE80E246E14D0FD
:109B2800146A156A166A176A2250DAEC60F000099E
:109B38000EE00B0E1A6E620EE82EFED71A2EFCD718
:109B480000D02406D8A0250624502510E9E1245089
:109B580025100AE0146A020E156E166A176A100EAE
:109B6800DAEC60F0000901E0236A23C06EF0F7EC3C
:109B780062F0235001E14AD7749048D7BEC0F6FF7F
:109B8800BFC0F7FF000EF86E0F0EF76403D0080091
:109B9800F55005D0F6CFE9FFF7CFEAFFEF502F0ACF
:109BA80013E0BEC0F6FFBFC0F7FF000EF86E0F0E41
:109BB800F76403D00800F55005D0F6CFE9FFF7CFDA
:109BC800EAFFEF505C0A03E10001BE4BBF2B000126
:109BD80020EE06F0BC51D926BD51DA22DE6ADE6AD3
:109BE800DE6ADD6ABEC0F6FFBFC0F7FF000EF86E82
:109BF8000F0EF76403D00800F55005D0F6CFE9FF43
:109C0800F7CFEAFFEF506A6E200E6A6012D0BCC030
:109C180062F0BDC063F0656A646AF2EC3FF0C36F3E
:109C280020EE12F0BC51D926BD51DA22DE6ADD6A77
:109C38005DD0BCC013F0BDC014F0BE0E156EEEECC6
:109C48003BF00001C36FC35151E1BCC0B6F0BDC0C9
:109C5800B7F0CEEC56F0C36F20EE14F0BC51D92605
:109C6800BD51DA2210EE0BF0DE50E126DD50E22283
:109C7800E750C26FC35108E0040EC31937E1C2B5FB
:109C880035D0050EC36F32D0C2B530D020EE12F0F9
:109C9800BC51D926BD51DA22DECFC0F0DDCFC1F0EC
:109CA80020EE0BF0C051D926C151DA22DFA8E9D73E
:109CB800BCC0D9FFBDC0DAFFDECF0BF0DDCF0CF0A2
:109CC800C0C00DF0C1C00EF063EC58F0000120EEEA
:109CD80006F0BC51D926BD51DA220BC0DEFF0CC0FC
:109CE800DEFF0DC0DEFF0EC0DEFFA3D7C35112009A
:109CF8000600D9CF05F0DACF06F0F2A01CD081BC5F
:109D080002D08994899281A802D089A20FD0938029
:109D1800939424EE5EF0010EDBBE07D0000EDE5CED
:109D2800020EDE5802E3939201D0938281B889B281
:109D380001D09384F290F2B281B079D081B889B21F
:109D48009392831C086E811C076E5EC409F05FC481
:109D58000AF00ABE03D0020E0A5C2BE2094A0A2A5C
:109D680009C05EF40AC05FF45CC409F05DC40AF07F
:109D7800600E0924D96E040E0A20DA6E08C0DFFFCF
:109D8800600E0924D96E060E0A20DA6E07C0DFFFBE
:109D9800094A0A2A0168010E026E09C003F00AC0C6
:109DA80004F0015003160250041603C05CF404C00A
:109DB8005DF481B889B29384938481A0FED781A889
:109DC80002D089A202D0939401D0938424EE5EF04D
:109DD800010EDBBE05D0000EDE5C020EDE5803E28B
:109DE8000101B05102E0939201D0938207A81ED0DE
:109DF8000BD0898202D0898405D0899417D089A292
:109E080015D08994899212D00850016E026A0250C6
:109E18000DE10150040AF3E0100AF1E0340AE9E028
:109E28001F0AF0E07F0AE7E01F0AE7E0F29206C0A7
:109E3800DAFF05C0D9FF75921100326A20EE04F0EE
:109E48002450D9262550DA22DF5001E197D020EEA0
:109E58002AF02450D9262550DA22DECF35F0DECF7D
:109E680036F0DECF37F0DECF38F02E0E24241A6E0F
:109E7800000E25201B6E35C01CF036C01DF037C003
:109E88001EF038C01FF0216A010E206E20EE01F08E
:109E98002450D9262550DA22DF50B1EC54F00009BD
:109EA80003E0010E326E6AD020EE04F02450D92669
:109EB8002550DA22DF6A20EE16F02450D9262550E4
:109EC800DA2210EE1EF02450E1262550E222E6CFD9
:109ED8002AF0E6CF2BF0E6CF2CF0E6CF2DF02A5073
:109EE800355C2E6E2B5036582F6E2C503758306EEE
:109EF8002D503858316EDE502E5CDE502F58DE5013
:109F08003058DE5031583AE220EE03F02450D9267A
:109F18002550DA22DF50336E346A345003E1020EE2
:109F2800335C2CE320EE16F02450D9262550DA2293
:109F3800DE503526DE503622DE503722DD503822FC
:109F48002E0E24241A6E000E25201B6E35C01CF020
:109F580036C01DF037C01EF038C01FF0216A010E50
:109F6800206E20EE01F02450D9262550DA22DF5049
:109F7800B1EC54F03306D8A03406CFD732501200D3
:109F88002F6C696664617461302E62696E20002FDF
:109F98006C696664617461312E62696E20002F6C91
:109FA800696664617461322E62696E20002F6C6983
:109FB8006664617461332E62696E20002F6C696675
:109FC80064617461342E62696E20002F6C69666466
:109FD800617461352E62696E20002F6C6966646158
:109FE8007461362E62696E20002F6C696664617434
:109FF80061372E62696E20002F6C69666461746136
:10A00800382E62696E20002F6C696664617461394C
:10A018002E62696E20002F6C696664617461612E1E
:10A0280062696E20002F6C696664617461622E62D9
:10A03800696E20002F6C696664617461632E6269C1
:10A048006E20002F6C696664617461642E62696EAB
:10A0580020002F6C696664617461652E62696E20E8
:10A06800002F6C696664617461662E62696E2000F7
:10A0780000000000000000000000000000000000D8
:10A0880000000000000000000000000000000000C8
:10A0980000000000000000000000000000000000B8
:10A0A8000000000000000000000000000BC015F0D8
:10A0B8000CC016F00F50101001E1120015C0D9FFA6
:10A0C80016C0DAFF0DC0DFFF0F501524116E1050B7
:10A0D8001620126EFF0E1124D96EFF0E1220DA6EB2
:10A0E8000DC0DFFF105004E1030E0F5C01E2120007
:10A0F80020EE01F01550D9261650DA220DC0DFFFE8
:10A1080020EE02F01550D9261650DA220DC0DFFFD6
:10A118000F501524116E10501620126EFE0E1124C9
:10A12800D96EFF0E1220DA6E0DC0DFFF0F50152416
:10A13800116E10501620126EFD0E1124D96EFF0EEE
:10A148001220DA6E0DC0DFFF105004E1070E0F5C1D
:10A1580001E2120020EE03F01550D9261650DA223B
:10A168000DC0DFFF0F501524116E10501620126E0F
:10A17800FC0E1124D96EFF0E1220DA6E0DC0DFFF1F
:10A18800105004E1090E0F5C01E2120015C011F035
:10A1980016C012F0111E121E114A122A030E1114B3
:10A1A800136E146A135015261450162213500F5E9E
:10A1B8001450105AFC0E0F160BD015C0D9FF16C03C
:10A1C800DAFF0DC0DFFF0F06D8A01006154A162AC1
:10A1D8000F501010F2E112000001915190118F11EF
:10A1E80003E1020E8E5D0FE320EE12F08C51D926AA
:10A1F8008D51DA22DE508E5DDE508F59DE50905937
:10A20800DE50915902E3020E2CD0966B6AD08CC0B6
:10A2180044F08DC045F08EC046F08FC047F090C026
:10A2280048F091C049F058EC2BF044C097F045C075
:10A2380098F046C099F047C09AF0000197519811DC
:10A2480099119A115DE09705981199119A11DBE01F
:10A25800972909E1982907E1992905E19A2903E154
:10A26800010E966F4DD08CC044F08DC045F08EC065
:10A2780046F08FC047F090C048F091C049F04A6A54
:10A288004B6A4C6A4D6A66EC22F0966F965138E13B
:10A2980020EE0EF08C51D9268D51DA22DE2806E107
:10A2A800DE2804E1DE2802E1DE2813E020EE0EF0CD
:10A2B8008C51D9268D51DA22DE2A000EDE22DE22CA
:10A2C800DE2220EE05F08C51D9268D51DA22000EBF
:10A2D800DB8097C08EF098C08FF099C090F09AC03C
:10A2E80091F020EE12F08C51D9268D51DA22DE50F1
:10A2F8008E5DDE508F59DE509059DE50915987E3BC
:10A3080096511200136814680B50D96EDA6ADE5041
:10A31800DE1001E181D00B50D96EDA6ADECF17F07A
:10A32800DDCF18F002D0174A182A17C0F6FF18C058
:10A33800F7FF000EF86E0F0EF76403D00800F55013
:10A3480005D0F6CFE9FFF7CFEAFFEF500D6E200EEC
:10A358000D6413D017C0F6FF18C0F7FF000EF86E93
:10A368000F0EF76403D00800F55005D0F6CFE9FFCB
:10A37800F7CFEAFFEF503A0AD6E117C0F6FF18C048
:10A38800F7FF000EF86E0F0EF76403D00800F550C3
:10A3980005D0F6CFE9FFF7CFEAFFEF503A0A41E1DF
:10A3A8000B50D96EDA6ADECF11F0DDCF12F011C092
:10A3B800F6FF12C0F7FF000EF86E0F0EF76403D019
:10A3C8000800F55005D0F6CFE9FFF7CFEAFFEF50C8
:10A3D8000D6ED00E0D24156E166AFF0E1622114A48
:10A3E800122A165019E10A0E155C16E217501118B8
:10A3F80013E11850121810E1155016100DE115C090
:10A4080013F016C014F0174A182A0B50D96EDA6ADE
:10A4180017C0DEFF18C0DDFF13C00BF014C00CF02E
:10A428001200136A146AF8D77350140D070EF32438
:10A43800D96E010EF420DA6EDECFE3F0DECFE4F061
:10A44800DECFE5F0DECFE6F0E4C0E3F0E5C0E4F00F
:10A45800E6C0E5F00001E66BE3C0E7F0E4C0E8F031
:10A46800260E806FFA0E816F7350140D070EF324B9
:10A47800D96E010EF420DA6EDECF82F0DECF83F0E3
:10A48800DECF84F0DECF85F07350140D070EF32471
:10A49800D96E010EF420DA6EDECF86F0DECF87F0BB
:10A4A800DECF88F0DECF89F0E7C08AF0E8C08BF015
:10A4B800B7EC62F0000E0001A66F030EA76F010E45
:10A4C800A96F000EA86F680EAA6FFF0EAB6F12EC93
:10A4D80048F01DEC4AF0CAC0E9F0CBC0EAF0E951F7
:10A4E800EA1105E0E9C0E1F0EAC0E2F0120082B446
:10A4F80015D07350200D000EF324A36F020EF42024
:10A50800A46F000EA56F030EA66F010EA86FA76BB0
:10A51800EB0EA96FAA6BCCEC0EF0EF6FEF510EE0CB
:10A52800530E806FFD0E816FEFC082F0836BB7EC26
:10A5380062F0EFC0E1F00001E26B1200FBEC55F0B5
:10A548000001E16BE26B1200020E0D5E000E0E5A66
:10A558000F5A105A20EE12F00B50D9260C50DA225E
:10A56800FE0EDE24116EFF0EDE20126EFF0EDE20C0
:10A57800136EFF0EDE20146E11500D5C12500E5833
:10A5880013500F581450105805E30B6A0C6A0D6AE3
:10A598000E6A120020EE26F00B50D9260C50DA2253
:10A5A800DECF11F0DECF12F0DECF13F0DECF14F0E5
:10A5B80020EE02F00B50D9260C50DA22DF50156E2F
:10A5C80015C016F0176A186A196A16500D02F3CFEB
:10A5D8001AF0F4CF1BF01C6A1D6A0E02F3501B26FA
:10A5E800F4501C22000E1D2217500D02F3501B269A
:10A5F800F4501C22000E1D2216500F02F3501C2688
:10A60800F4501D2217500E02F3501C26F4501D2240
:10A6180018500D02F3501C26F4501D22105016023B
:10A62800F3501D2617500F02F3501D2618500E0226
:10A63800F3501D2619500D02F3501D2611501A24EF
:10A648000B6E12501B200C6E13501C200D6E1450F4
:10A658001D200E6E1200E8C15CF070D022EC62F092
:10A668005C6EE81978E0150E5B6E4B0E5A6EBE0EE6
:10A67800E82EFED75A2EFCD75B2EFAD700D06BD027
:10A6880006EC5EF05D6E5D5066E05DB06D2A5DB211
:10A698006D060F0E6D16000E0B6EC00E7FEC5FF090
:10A6A80035EC62F0000E0B6EC00E7FEC5FF06D5063
:10A6B8000F0D8E0EF3240F6E0C0EF420106E1CEC92
:10A6C8005CF00D0E5B6E2D0E5A6ED80EE82EFED77E
:10A6D8005A2EFCD75B2EFAD75DA43DD00C6A0B6AC4
:10A6E8006DC00DF085EC60F0410E0001806FFC0E2E
:10A6F800816F6DC082F0836BB7EC62F06DC05CF067
:10A70800000E0B6E800E7FEC5FF035EC62F0000EF1
:10A718000B6E800E7FEC5FF06D500F0D8E0EF324E4
:10A728000F6E0C0EF420106E1CEC5CF0000E0B6E1D
:10A73800C00E7FEC5FF035EC62F00DD00101AC513A
:10A748005A6E5B6A5B5007E15A50010A87E0030AB8
:10A7580085E0010A95E05C5012001F6A206A186AB9
:10A76800196A01D0122A010E1E6E1250D96EDA6AC9
:10A77800200EDE1813E0F70E146E15681250D96E0D
:10A78800DA6ADF50166E176A14501626155017220B
:10A79800175003E1050E165C01E31E6A1EC01AF08D
:10A7A8001B6A1A501B1006E0DDD7196A010E186ED5
:10A7B800122A25D01250D96EDA6ADF50146E156A43
:10A7C80015501DE114502B0AF3E0060AEEE017D0ED
:10A7D8000A0E1F02F3CF14F0F4CF15F02002F35045
:10A7E80015261250D96EDA6ADF50145E000E155A1B
:10A7F800300E14241F6E000E1520206ED9D7D00EEF
:10A80800146E15681250D96EDA6ADF50166E176A20
:10A818001450162615501722175005E10A0E165C1B
:10A8280002E2010E01D0000E1C6E1D6A1C501D10A4
:10A83800CFE1185019100DE11FC014F020C015F019
:10A84800141E151E144A152A14C012F015C013F050
:10A8580012001FC012F020C013F012000101B46BE7
:10A868008980000E0B6E030E0C6E0E6AF60E0D6ECE
:10A87800010E106E0F6A5AEC50F0220E0001806F24
:10A88800FE0E816FB7EC62F00101BB6BBC6B2E0E44
:10A89800C1EC62F082B418D07350200D000EF3247E
:10A8A8000001A36F020EF420A46F000EA56F030E23
:10A8B800A66F010EA86FA76BB70EA96F010EAA6F3E
:10A8C800CCEC0EF00101B96F0101B9510AE05A0E42
:10A8D8000001806FFF0E816FB9C182F0836BB7EF03
:10A8E80062F0F2EC62F00B500C1026E0BA0E0B6E20
:10A8F800010E0C6ECDEC5AF00101B66FBA51100B77
:10A908005A6E000E5B6EB65132EC29F05AC0BDF19A
:10A918005BC0BEF1040E0101BD19BE1102E128ECB5
:10A9280060F0020EBD19BE1102E1A9EC5DF0BD0593
:10A93800BE1102E13CEC12F00101BB4BBC2B600ED6
:10A94800BB5D040EBC59A3E3FB0E0001806FFE0E35
:10A95800816FB7EC62F089901200236E2350D8A45F
:10A96800040C2050211001E1040C74B0030C74B4E1
:10A97800020C6EB608D0090ED8901C361D361E364D
:10A988001F36E82EF9D7200421101AE11CC014F054
:10A998001DC015F01EC016F01FC017F0180EDAEC17
:10A9A80060F0000945E11AC00DF01BC00EF0FE0E64
:10A9B8000F6EB4EC5EF000093BE0206A216A38D0E3
:10A9C8006EC022F0060E221609E020C014F021C045
:10A9D80015F0166A176A970EDAEC60F01CC014F0CE
:10A9E8001DC015F01EC016F01FC017F0190EDAECC6
:10A9F80060F000091DE11AC00DF01BC00EF0FC0E3E
:10AA08000F6EB4EC5EF0000908E0020E1B2620066B
:10AA1800D8A0210620502110EEE10D6A0E6AFD0E25
:10AA28000F6EB4EC5EF0000903E1216A010E206E9E
:10AA3800F7EC62F020502110D8A4010C000C0F0E86
:10AA4800C16E969496929690929A090E106E1E0E6A
:10AA58000F6EE40EE82EFED70F2EFCD7102EFAD775
:10AA680000D0090E106E1E0E0F6EE40EE82EFED7F3
:10AA78000F2EFCD7102EFAD700D0D00E0F6ECA0EAC
:10AA8800E82EFED70F2EFCD7000E0B6E300E7FEC93
:10AA98005FF0150E0F6EC60EE82EFED70F2EFCD7F0
:10AAA80000D0000E0B6E300E7FEC5FF0000E0B6EC8
:10AAB800300E7FEC5FF0000E0B6E390E7FEC5FF00E
:10AAC800000E0B6E140E7FEC5FF0000E0B6E560E30
:10AAD8007FEC5FF0000E0B6E6D0E7FEC5FF0000EEA
:10AAE8000B6E700E7FEC5FF0000E0B6E0C0E7FECA1
:10AAF8005FF0000E0B6E060E7FEC5FF0000E0B6E23
:10AB0800010E7FEC5FF0680E0F6EE40EE82EFED7A4
:10AB18000F2EFCD700D01200920E0001806FF80EA5
:10AB2800816FCFCF82F0836BCECF84F0856B73C0FB
:10AB380086F0876BB7EC62F00101E783735028E178
:10AB48008E0E0B6E0A0E0C6EEA0E0D6E020E0E6E57
:10AB5800106A050E0F6EC5EC5FF0930E0B6E0A0EB1
:10AB68000C6EAA0E0D6E020E0E6E106A130E0F6E8C
:10AB7800C5EC5FF0A60E0B6E0A0E0C6ED00E0D6EB5
:10AB8800020E0E6E106A0D0E0F6EC5EC5FF027D028
:10AB98008E0E0B6E0A0E0C6EEF0E0D6E020E0E6E02
:10ABA800106A050E0F6EC5EC5FF0930E0B6E0A0E61
:10ABB8000C6EBD0E0D6E020E0E6E106A130E0F6E29
:10ABC800C5EC5FF0A60E0B6E0A0E0C6EDD0E0D6E58
:10ABD800020E0E6E106A0D0E0F6EC5EC5FF0656A00
:10ABE800250E646EDCEC44F0E793899012007350F4
:10ABF800140D070EF324D96E010EF420DA6E000E40
:10AC0800DE24CA6F010EDE20CB6F000EDE20CC6F73
:10AC1800000EDE20CD6F7350140D070EF324D96E8D
:10AC2800010EF420DA6ECAC0DEFFCBC0DEFFCCC056
:10AC3800DEFFCDC0DEFF7350140D070EF324D96E6E
:10AC4800010EF420DA6EDECFCFF0DDCFD0F0050EA6
:10AC5800806FF40E816FCFCF82F0836BCECF84F0FC
:10AC6800856BCFC086F0D0C087F0CFC088F0D0C049
:10AC780089F0B7EC62F07350200D000EF324000148
:10AC8800A36F020EF420A46FCFC0A5F0D0C0A6F029
:10AC9800A76BA86B9EEC15F0CE6FCE5110E0EA0EB4
:10ACA800806FFA0E816FCFC082F0D0C083F0CEC023
:10ACB80084F0856BB7EC62F0010E6B6E010C6B6A69
:10ACC8001200880EF66E9F0EF76E000EF86E0CEEF0
:10ACD8008EF011EE2CF00900F5CFEEFFE550E150B3
:10ACE800FAE1E250F8E1B40EF66EBE0EF76E000E11
:10ACF800F86E02EEAAF010EE4AF00900F5CFEEFF6A
:10AD0800E550E150FAE10D0EF66EC60EF76E000E34
:10AD1800F86E0900F5CFEAF10C0EF66EC60EF76E66
:10AD2800000EF86E0900F5CF74F004EE5AF018EE34
:10AD380034F0EE6AE550E150FCE1E250FAE104EE4D
:10AD480000F0400EEE6AE806FDE103EE00F011EEB9
:10AD580000F0EE6AE550E150FCE1E250FAE102EE63
:10AD680000F0AA0EEE6AE806FDE101EE00F0B60E6C
:10AD7800EE6AE806FDE10001FE6B00EE6BF0090EDD
:10AD8800EE6AE806FDE175907592000EF86E000116
:10AD980049EF07F0B6C062F0B7C063F0656A646A4D
:10ADA800F2EC3FF0BB6FBB5102E0BB511200B6C0E2
:10ADB800D9FFB7C0DAFFDECF39F0DDCF3AF020EEA9
:10ADC8000EF0B651D926B751DA22DECF3BF0DECFEE
:10ADD8003CF0DECF3DF0DECF3EF05BEC59F00001F9
:10ADE800BB6FBB51E2E120EE12F0B651D926B75144
:10ADF800DA22DECFB9F0DDCFBAF0B9C0D9FFBAC0D8
:10AE0800DAFFDF50B86FB85103E1040EBB6FCDD73E
:10AE180020EE0BF0B951D926BA51DA22DFB616D096
:10AE2800B9C00BF0BAC00CF020EE14F0B651D92618
:10AE3800B751DA22DECF0DF0DDCF0EF0106A0B0E1F
:10AE48000F6ED9EC5DF00B500C10AFE0B6C0A3F05C
:10AE5800B7C0A4F0A66BA56B8CEC31F00001BB6FFA
:10AE6800BB51A3E1A4D7B6C062F0B7C063F0656A6E
:10AE7800646AF2EC3FF0BF6FBF5157E1BD6BBE6B28
:10AE8800B6C0D9FFB7C0DAFFDECF39F0DDCF3AF070
:10AE980020EE0EF0B651D926B751DA22DECF3BF0BC
:10AEA800DECF3CF0DECF3DF0DECF3EF05BEC59F07C
:10AEB8000001BF6FBF5139E120EE12F0B651D9261B
:10AEC800B751DA22DECFBAF0DDCFBBF0BAC0D9FF76
:10AED800BBC0DAFFE50EDE1810E020EE12F0B65126
:10AEE800D926B751DA22DECFBAF0DDCFBBF0BAC02F
:10AEF800D9FFBBC0DAFFDF5009E1BD4BBE2BB8510B
:10AF0800BD1906E1B951BE1910E002D0BD6BBE6B88
:10AF1800B6C0A3F0B7C0A4F0A66B010EA56F8CEC69
:10AF280031F00001BF6FBF51ABE0040EBF1902E161
:10AF3800070EBF6FBF511200706A6F6A0101A26BE2
:10AF4800A36B020EB46F8990B36BB26B736A030E76
:10AF5800736401D049D073500C0D530EF324D96E8D
:10AF6800010EF420DA6EDF6A73500C0D520EF324D2
:10AF7800D96E010EF420DA6EDF6A73500C0D500E94
:10AF8800F324D96E010EF420DA6EDE6ADD6A73509E
:10AF98000C0D540EF324D96E010EF420DA6EDE6A1D
:10AFA800DE6ADE6ADD6A73500C0D5B0EF324D96E1F
:10AFB800010EF420DA6E100EDF6E73500C0D5A0E6F
:10AFC800F324D96E010EF420DA6E020EDF6E735090
:10AFD8000C0D580EF324D96E010EF420DA6E240EEF
:10AFE800DE6EDD6A732AB3D7100E01015B6F020EA5
:10AFF8005A6F596B240E586F736A1200C0C0B6F0AE
:10B00800C1C0B7F0B96B010EB86F37EC57F06A6E74
:10B018006A5053E1C0C0D9FFC1C0DAFFDECF39F0B2
:10B02800DDCF3AF020EE0EF0C051D926C151DA2218
:10B03800DECF3BF0DECF3CF0DECF3DF0DECF3EF0A2
:10B048005BEC59F06A6E6A5038E1000120EE12F0AC
:10B05800C051D926C151DA22DECF0BF0DDCF0CF07A
:10B068000E6A0D6A106A200E0F6EFAEC61F000018C
:10B0780020EE12F0C051D926C151DA22DECF0BF0F2
:10B08800DDCF0CF020EE14F0C051D926C151DA22E0
:10B09800DECF0DF0DDCF0EF0106A0B0E0F6E48EC10
:10B0A80060F0C0C0D9FFC1C0DAFF10EE04F0DE5076
:10B0B800E126DD50E222010EE76E6A5012001A0EF8
:10B0C8000D240F6E000E0E20106E0F28D96E000E84
:10B0D8001020DA6EDF50126E116A1A0E0D24D96E26
:10B0E800000E0E20DA6EDF50111211C017F012C0D8
:10B0F80018F0196A1A6A0BC0D9FF0CC0DAFF030EE0
:10B10800DE1829E1140E0D240F6E000E0E20106EAD
:10B118000F28D96E000E1020DA6EDF50126E116AF9
:10B12800140E0D24D96E000E0E20DA6EDF501110A9
:10B13800136E1250146E156A166A14C016F013C0F6
:10B1480015F0146A136A1350171214501812155078
:10B15800191216501A1217C00BF018C00CF019C0AB
:10B168000DF01AC00EF01200226E2250D8A4040C62
:10B178002050211001E1040C74B0030C6EB608D005
:10B18800090ED8901C361D361E361F36E82EF9D704
:10B19800215006E1020E205C03E2246A110E02D05F
:10B1A800246A120E236E23C025F01CC014F01DC0A3
:10B1B80015F01EC016F01FC017F02550DAEC60F02D
:10B1C80000091DE11AC00BF01BC00CF0020E0E6E38
:10B1D8000D6A33EC5EF0000908E0020E1B2620061B
:10B1E800D8A0210620502110EDE1120E251807E104
:10B1F800146A156A166A176A0C0EDAEC60F0F7EC36
:10B2080062F020502110D8A4010C000C8980000E97
:10B218000B6E030E0C6E0E6AF60E0D6E010E106E9E
:10B228000F6A5AEC50F0220E0001806FFE0E816FFB
:10B23800B7EC62F00001CA6BCB6B2E0EC1EC62F06A
:10B2480082B416D07350200D000EF3240001A36FB2
:10B25800020EF420A46F000EA56F030EA66F010E58
:10B26800A86FA76BC70EA96FAA6BCCEC0EF0C96FBD
:10B278000001C95109E05A0E806FFF0E816FC9C0E5
:10B2880082F0836BB7EF62F0CA4BCB2BCBBFD5D71D
:10B29800CB5103E1640ECA5DD0E3FB0E806FFE0E56
:10B2A800816FB7EC62F0899089906B6A1200436AEB
:10B2B80020EE2AF03950D9263A50DA223B50DE18CF
:10B2C80009E13C50DE1806E13D50DE1803E13E502E
:10B2D800DE1839E039C024F03AC025F021EC4FF0EF
:10B2E800436E435030E12E0E39241A6E000E3A2078
:10B2F8001B6E3BC01CF03CC01DF03DC01EF03EC0A4
:10B308001FF0216A010E206E20EE01F03950D92677
:10B318003A50DA22DF50B8EC58F0000906E03B68F2
:10B328003C683D683E68010E436E20EE2AF03950B5
:10B33800D9263A50DA223BC0DEFF3CC0DEFF3DC0D2
:10B34800DEFF3EC0DEFF43501200D4C0DAF0D5C0A5
:10B35800DBF0DA0E0B6E86EC51F00BC0DCF00CC0A3
:10B36800DDF00001DDBF0B0CD890DC35D96EDD3582
:10B37800DA6EA00ED926010EDA22DECFD8F0DDCFA4
:10B38800D9F0D851D91105E0D8C0D9FFD9C0DAFF12
:10B39800DF6AD251D31105E0D2C0D9FFD3C0DAFF9A
:10B3A800DF6AD890DC35D96EDD35DA6EA00ED92685
:10B3B800010EDA22D2C0DEFFD3C0DDFFD251D31195
:10B3C800D8B4000CD60501E0000CD20E666E676A90
:10B3D800D40E686E696A09EC00F0D76FD751120075
:10B3E80003D00B4A0C2A0D2A0D50D96EDA6ADF50A9
:10B3F8000E6E0BC0F6FF0CC0F7FF000EF86E0F0EB6
:10B40800F76403D00800F55005D0F6CFE9FFF7CF71
:10B41800EAFFEF500E1813E10BC0F6FF0CC0F7FF60
:10B42800000EF86E0F0EF76403D00800F55005D033
:10B43800F6CFE9FFF7CFEAFFEF500009D2E10BC0E2
:10B44800F6FF0CC0F7FF000EF86E0F0EF76403D07E
:10B458000800F55005D0F6CFE9FFF7CFEAFFEF5027
:10B468000E6E0D50D96EDA6ADF500E5C0B6E0C6AE8
:10B47800D8A00C0612000BC012F00CC013F00DC0BF
:10B4880014F00EC015F00F06D8A010060F280CE116
:10B4980010280AE10B6A0C6A1200124A132A144A8D
:10B4A800152A0F06D8A0100612C0F6FF13C0F7FF22
:10B4B8000800F55015E014C0D9FF15C0DAFFDF50B9
:10B4C8000FE00F5010100CE014C0D9FF15C0DAFFC0
:10B4D80012C0F6FF13C0F7FFDE500900F518DDE0D3
:10B4E80012C0F6FF13C0F7FF0800F5CF11F014C023
:10B4F800D9FF15C0DAFFDF50115C0B6E0C6AD8A0BB
:10B508000C0612000CC012F00DC013F012501310EC
:10B51800D8B4090C12C0D9FF13C0DAFFDE50DE1010
:10B52800D8B4090C12C0D9FF13C0DAFFDECF0EF071
:10B53800DDCF0FF00EC0D9FF0FC0DAFFDF50D8B44F
:10B54800090C20EE02F01250D9261350DA2212C04C
:10B55800E1FF13C0E2FF00EE06F0E650E926E550F1
:10B56800EA22DE50EE1813E1DE50EE18D8A4090CDA
:10B5780012C0D9FF13C0DAFF10EE01F0DE50E12649
:10B58800DD50E222E750ECEC62F00E6E0EB0090CD2
:10B59800000C24EE5EF0DE50DE10FBE05AC413F01F
:10B5A8005BC414F0600E1324D96E040E1420DA6EF6
:10B5B800DF50116E600E1324D96E060E1420DA6E59
:10B5C800DF50126E134A142A0D68010E0E6E13C056
:10B5D8000FF014C010F00D500F160E5010160FC0BB
:10B5E8005AF410C05BF4F29E24EE5EF0DE06000E04
:10B5F800DD5AF28E0BC0D9FF0CC0DAFF12C0DFFF94
:10B6080024EE5EF0010EDBBE05D0000EDE5C020EFD
:10B61800DE5802E289B29382115012000E5002E005
:10B628000E5003E10C50ADEF62F00E50D96EDA6A9D
:10B63800040ED926DE50DE1014E00E50D96EDA6AF8
:10B64800040ED9260E50E16EE26A020EE126DE50A3
:10B65800E65CE650800A136EDE50800A1358D8B0B4
:10B6680012000E50D96EDA6A020ED926DECF0FF01C
:10B67800DDCF10F00E50D96EDA6ADECF11F0DDCFD3
:10B6880012F00F501124D96E10501220DA6E0CC02F
:10B69800DFFF0E50D96EDA6A020ED926DE2A000EB6
:10B6A800DD22000C0B500F02F3CF13F0F4CF14F08F
:10B6B800156A166A0B501002F3501426F45015221E
:10B6C800000E16220C500F02F3501426F4501522C7
:10B6D800000E16220B501102F3501526F4501622B4
:10B6E8000C501002F3501526F45016220D500F027C
:10B6F800F3501526F450162212500B02F35016265A
:10B708000C501102F35016260D501002F350162655
:10B718000E500F02F350162613C00BF014C00CF095
:10B7280015C00DF016C00EF01200630E806FFD0EEE
:10B73800816F98C182F099C183F0B7EC62F011D0A3
:10B74800030E0BD0050E5C6E0101986B996B2DD022
:10B758000A0E03D0010E01D0020E5C6E26D05C6A80
:10B7680024D098C15AF099C15BF05B5009E0020AF5
:10B778000DE00E0A0FE0010A11E02A0A13E0EFD7E4
:10B788005A500A0ADDE01E0ADDE0E9D75A50BC0A21
:10B79800E3E0E5D75A501C0ADBE0E1D75A50AC0A7F
:10B7A800D9E0DDD75A500F0ADAE15C501200140EC6
:10B7B8000001806FFE0E816FB7EC62F05D6A5E6A11
:10B7C800716A5F6A2ED0F2EC62F00B500C101EE02A
:10B7D8005F0E0B6E0C6ACDEC5AF05C6E5FA80BD056
:10B7E800DB0E0001806FFE0E816F5CC082F0836B00
:10B7F800B7EC62F00BD0000E7124D96EDA6A030E32
:10B80800DA225CC0DFFF712A5D4A5E2A5FAA07D090
:10B81800000E5D245A6E040E5E205B6E120081AC31
:10B8280002D05E04D0E35DC05AF05EC05BF0120047
:10B838000B0E116E620EE82EFED7112EFCD700D02B
:10B8480020D00B0E116E620EE82EFED7112EFCD7FB
:10B8580000D0010E0B6E0FC0F6FF10C0F7FF000EF0
:10B86800F86E0F0EF76403D00800F55005D0F6CF38
:10B87800E9FFF7CFEAFFEF507FEC5FF00F4A102A9D
:10B88800D7D70FC0F6FF10C0F7FF000EF86E0F0EE7
:10B89800F76403D00800F55005D0F6CFE9FFF7CFDD
:10B8A800EAFFEF500009CDE11200A20E0001806FFF
:10B8B800FA0E816FCFCF82F0836BCECF84F0856B89
:10B8C800B7EC62F05A6A5B6A7350140D070EF324E2
:10B8D800D96E010EF420DA6EDE6ADE6ADE6ADD6A8F
:10B8E8007350140D130EF324D96E010EF420DA6E82
:10B8F800DF6A7350140D0F0EF324D96E010EF42075
:10B90800DA6EDE6ADE6ADE6ADD6A5A4A5B2A5BBE86
:10B91800DBD75B5003E1040E5A5CD6E389906B6A6F
:10B928001200E60E0001806FFE0E816FB7EC62F028
:10B93800736A030E736401D02AD073500C0D530E32
:10B94800F324D96E010EF420DA6EDF6A73500C0D01
:10B95800520EF324D96E010EF420DA6EDF6A7350AA
:10B968000C0D500EF324D96E010EF420DA6EDE6A47
:10B97800DD6A73500C0D540EF324D96E010EF420B9
:10B98800DA6EDE6ADE6ADE6ADD6A732AD2D7736A25
:10B9980089900101B46B1200136A146A156A166A59
:10B9A8000F5010101110121029E0010E176E06D05A
:10B9B800D8900F36103611361236172A12AEF8D72D
:10B9C800D89013361436153616360F500B5C1050B7
:10B9D8000C5811500D5812500E5809E30F500B5EB9
:10B9E80010500C5A11500D5A12500E5A1380D890FC
:10B9F8001232113210320F32172EE2D713C00BF069
:10BA080014C00CF015C00DF016C00EF01200136E25
:10BA18000C0E131807E0F7EC62F08AEC62F00009EC
:10BA280001E1FF0C13504009D4EC62F01050D4EC43
:10BA380062F00F50D4EC62F00E50D4EC62F00D506E
:10BA4800D4EC62F0010E126E135002E1950E126EE4
:10BA5800080E131802E1870E126E1250D4EC62F031
:10BA68000C0E131802E1E5EC62F00A0E126EE5EC1A
:10BA780062F0116E11AE02D0122EF9D711501200D9
:10BA8800F6EC60F0CC0E63EC62F0660E63EC62F0EC
:10BA980046EC62F0156E155005E10F6A106A116ADE
:10BAA800126A1200136A146A1350150FD96EDA6AF3
:10BAB80046EC62F0DF6E134A142A14BEF5D7145010
:10BAC80003E1040E135CF0E318501710161003E19D
:10BAD800060E155CE2E315C00FF016C010F017C093
:10BAE80011F018C012F012000F501010111012109F
:10BAF80023E0010E136E06D0D8900F36103611369B
:10BB08001236132A12AEF8D70F500B5C10500C588F
:10BB180011500D5812500E5808E30F500B5E10507C
:10BB28000C5A11500D5A12500E5AD8901232113226
:10BB380010320F32132EE8D70BC00BF00CC00CF0EC
:10BB48000DC00DF00EC00EF01200070E0001806F40
:10BB5800FC0E816FB2C182F0836BB7EC62F0898012
:10BB68000101E7832AEE8EF0B2C1DFFF000EE8CFB5
:10BB78008FFA0D0EE8CF90FA000EE8CF91FA82A462
:10BB880003D0600EE8CF91FA82A406D090CA6AF07A
:10BB9800200E6A126AC090FA656A040E646EDCECC4
:10BBA80044F0E793B26B899012000BC012F00CC0FE
:10BBB80013F00DC014F00EC015F0166A176A0F06C0
:10BBC800D8A010060F2802E1102817E012C0D9FFEC
:10BBD80013C0DAFF124A132ADF50116E14C0D9FFBE
:10BBE80015C0DAFF144A152ADF50115C166E176A61
:10BBF800D8A0170616501710E2E016C00BF017C0B1
:10BC08000CF01200010E0B6E0C6A92868D828D84E8
:10BC180000D000D000D000D08D9400D000D000D04B
:10BC280000D00D6A0E6A80A602D00B500C12D89074
:10BC38000B368D9000D000D000D000D08D8000D081
:10BC480000D000D000D08D900D4A0E2A0EBEEBD742
:10BC58000E5003E1030E0D5CE6E30C501200070ED4
:10BC6800106ED00E0F6E0CD0E5EC62F0116E11283C
:10BC78000AE1A00E00D0E82EFDD70F06D8A01006C6
:10BC88000F501010F1E1FE0E111801E0000CE5EC68
:10BC980062F00BC0D9FF0CC0DAFFDF6E0B4A0C2A2A
:10BCA8000D06D8A00E060D500E10F1E1E5EC62F07D
:10BCB800E5EC62F0010C0BC011F00CC012F013D0CF
:10BCC8000F06D8A010060DC0D9FF0EC0DAFF0D4A26
:10BCD8000E2A11C0E1FF12C0E2FF114A122ADFCF7B
:10BCE800E7FFE7500BE00F50101008E0E9D711C04C
:10BCF800D9FF12C0DAFFDF6A114A122A0F06D8A04C
:10BD080010060F28F4E11028F2E112008C6A8A6A02
:10BD1800956893680101B06B716A899289949C6BEC
:10BD28009D6B09D0000E9C25D96E030E9D21DA6EFD
:10BD3800DF6A9C4B9D2B9DBFF5D79D05F3E39C6B5C
:10BD48009D6B09D08E0E9C25D96E0A0E9D21DA6E48
:10BD5800DF6A9C4B9D2B9DBFF5D79D05F3E3120031
:10BD68005EEC61F0000901E1000C0F50D4EC62F0C8
:10BD7800FD0E0F181EE0020E116E106A0DC0D9FFDD
:10BD88000EC0DAFFDF50D4EC62F00D4A0E2A10061E
:10BD9800D8A0110610501110F1E1E5EC62F0E5ECC5
:10BDA80062F0E5EC62F0126E12501F0B050A01E01A
:10BDB800000C010C15D00CC0F6FF0DC0F7FF000EEB
:10BDC800F86E0F0EF76403D00800F55005D0F6CFD3
:10BDD800E9FFF7CFEAFFEF50C1EC62F00C4A0D2AF9
:10BDE8000CC0F6FF0DC0F7FF000EF86E0F0EF764DB
:10BDF80003D00800F55005D0F6CFE9FFF7CFEAFFEA
:10BE0800EF500009D8E112000EC012F00FC013F075
:10BE180010C014F011C015F0F6EC60F0CC0E63EC15
:10BE280062F0990E63EC62F00C0E63EC62F0166A35
:10BE3800176A1650120FD96EDA6ADF5063EC62F097
:10BE4800164A172A17BEF5D7175002E0F6EF60F02A
:10BE5800040E165CEEE3F6EF60F05B6E390E5C6E76
:10BE6800F30E5D6E5A6A0AD05CC0F6FF5DC0F7FF3C
:10BE78005C4A5D2A0800F550F7E15A2A5B505A18C7
:10BE880007E05CC0F6FF5DC0F7FF0800F550ECE185
:10BE9800F80E0001806FFD0E816F5BC082F0836B2E
:10BEA8005CC084F05DC085F0B7EF62F00109122034
:10BEB800010001001700002D119420D00F0001018E
:10BEC800091220010001001700002D119420D00F45
:10BED800000100004F01000F0000000009FF0000F2
:10BEE800004F01000F0000000009FF00800102E878
:10BEF80005800102E8050C6E8D9200D000D000D0BC
:10BF080000D00BB002D08D9401D08D84000E0E6E3F
:10BF1800010E0D6E0CAE02D0898A01D0899AD89094
:10BF28000C368D908D808D900D4A0E2A0EBEF2D75C
:10BF38000E5003E1090E0D5CEDE38D8212009F0E99
:10BF4800136E146811C015F012C016F013501526A0
:10BF580014501622165005E11A0E155C02E2010E65
:10BF680001D0000E176E186A1750181005E05F0E02
:10BF78001114116E126A120011C011F012C012F0E1
:10BF880012000DC014F00EC015F00BC012F00CC05A
:10BF980013F010D014C0D9FF15C0DAFFDF50116EAE
:10BFA800144A152A12C0D9FF13C0DAFF11C0DFFFE7
:10BFB800124A132A0F06D8A010060F28EBE1102802
:10BFC800E9E1120020EE1AF00B50D9260C50DA22C3
:10BFD8000DC0DFFF20EE1BF00B50D9260C50DA22E3
:10BFE8000EC0DFFF20EE14F00B50D9260C50DA22D9
:10BFF8000FC0DFFF20EE15F00B50D9260C50DA22C7
:10C008001050DF6E12000BC00DF00CC00EF002D005
:10C018000B4A0C2A0BC0F6FF0CC0F7FF000EF86E97
:10C028000F0EF76403D00800F55005D0F6CFE9FFEE
:10C03800F7CFEAFFEF500009EBE10D500B5C0B6EF8
:10C048000E500C580C6E1200A20E0001806FFE0EEE
:10C05800816FB4C182F0836BB7EC62F08E0E0B6E09
:10C068000A0E0C6E0E6A0D6A010E106E0F6A5AECFB
:10C0780050F02AEE8EF0B4C1DFFF656A010E646EDF
:10C08800DCEC44F0B46B12000BC011F00CC012F0E1
:10C098000DC013F00EC014F00ED013C0D9FF14C099
:10C0A800DAFF11C0E1FF12C0E2FFDFCFE7FF134A5A
:10C0B800142A114A122A0F06D8A010060F28EDE1FB
:10C0C8001028EBE112000B6E0B500EE0FBEC62F057
:10C0D800200EE82EFED7FEEC62F0CC0E00D0E82E43
:10C0E800FDD700D000D01200FBEC62F0C00E00D0EB
:10C0F800E82EFDD7FEEC62F0350EE82EFED700F0F4
:10C108001200000EF2BE010E0E6E0C50030BAA6E4A
:10C118000BC0A9FF0DC0A8FFA69EA69CA684F29EF0
:10C12800550EA76EAA0EA76EA682A6B2FED7A69433
:10C138000EB002D0F29E01D0F28E120002D00B4A4D
:10C148000C2A0BC0F6FF0CC0F7FF0800F55009E0F9
:10C158000BC0F6FF0CC0F7FF0800F5500D180E10C5
:10C16800EEE10BC0F6FF0CC0F7FF0800F5500B6EB0
:10C178000C6A12005E0E626E5AC063F05BC064F017
:10C18800656A666A676A686A630E546E5CC055F0D1
:10C198005DC056F0620E576E81EC2FF065505A2440
:10C1A800D96E66505B20DA6EDF6A000C186E18AE26
:10C1B8000ED0189E0D6A0E6A0F6A106A370E0BECC5
:10C1C8005DF0196E010E196402D01950120014C0E6
:10C1D8000DF015C00EF016C00FF017C010F0185073
:10C1E8000BEF5DF0FBEC62F00A0E0C6EF80EE82E19
:10C1F800FED70C2EFCD700D0FEEC62F0E00E00D08B
:10C20800E82EFDD7CBEC62F0090E0C6E840EE82EFA
:10C21800FED70C2EFCD7FEEF62F0010E116E200E39
:10C228000B180C1011E0F70E0D6E0E680BC00FF016
:10C238000CC010F00D500F260E501022105003E1C4
:10C24800050E0F5C01E3116A11C00BF00C6A1200B5
:10C258005BC04EF05CC04FF009EC47F05D6E5D507E
:10C268000FE15BC00CF05CC00DF086EC5AF05D6E1F
:10C278005D5006E15BC0D9FF5CC0DAFFDE6ADD6AAB
:10C288005D5012009F0E0D6E0E68200E0B100F6E83
:10C29800000E0C10106E0D500F260E50102210506C
:10C2A80005E11A0E0F5C02E2010E01D0000E0B6EC2
:10C2B8000C6A1200130E0C6E880E0B6E0BD0E5EC98
:10C2C80062F0FF0A0AE0A00E00D0E82EFDD70B06A8
:10C2D800D8A00C060B500C10F2E10B500C10D8A48F
:10C2E800010C000C186A196A09D017C00CF00D6A05
:10C2F80016C00EF012EC5BF0184A192A18501424D4
:10C30800D96E19501520DA6EDF50176E1750EDE10F
:10C3180012008E0E0B6E0A0E0C6E0E6A0D6A010E5E
:10C32800106E0F6A5AEC50F0010EE8CF8EFA010138
:10C33800E783656A646EDCEC44F0E79312009F0EB5
:10C348000D6E0E680BC00FF00CC010F00D500F26CC
:10C358000E501022105005E11A0E0F5C02E2010E79
:10C3680001D0000E0B6E0C6A1200BF0E0D6E0E6827
:10C378000BC00FF00CC010F00D500F260E501022FD
:10C38800105005E11A0E0F5C02E2010E01D0000EFA
:10C398000B6E0C6A1200D00E0D6E0E680BC00FF0FB
:10C3A8000CC010F00D500F260E501022105005E151
:10C3B8000A0E0F5C02E2010E01D0000E0B6E0C6A31
:10C3C8001200B886AC84B898440EAF6EB06AAC98C8
:10C3D800AB8EAB88AB9A9D989D9AD08E9F8AF28E31
:10C3E800AC90AB9CAC9AAC8AA99112000BC011F02E
:10C3F8000CC012F008D011C0D9FF12C0DAFF0DC06E
:10C40800DFFF114A122A0F06D8A010060F28F3E101
:10C418001028F1E11200FBEC62F0200EE82EFED7A6
:10C42800FEEC62F0300EE82EFED7CBEC62F00C6E1C
:10C43800B00E00D0E82EFDD70C501200070E966EF5
:10C448008450070B0B6E928A80AA02D0080E0B2626
:10C45800020E0101AC1903E10B1C0F0B0B6E0B5004
:10C468001200106A100E0F6E05D0010E0B6E200E12
:10C478007FEC5FF00F06D8A010060F28F6E1102811
:10C48800F4E112000D6A0E6AD8900D320FEC62F0DA
:10C49800000901E00D8E0E2A070E0E64F5D70D5027
:10C4A8001200000EE8CF5AF4E8CF5BF4E8CF5CF452
:10C4B800E8CF5DF4E8CF5EF4E8CF5FF4000C0C6ED3
:10C4C8000D6A0C50010B67EC60F0D8900C320D2A05
:10C4D800070E0D64F6D7070C0B6E0B5007E0C66A03
:10C4E800010EC66E400EC76EC68A400CC66A020EA2
:10C4F800F8D7C2900F0EC16E070EB46E4F0EC86EFD
:10C50800946A948894829482826A120003EC63F09D
:10C51800E5EC62F05EEC61F0000901E0010CF7EC7B
:10C5280062F0000C0C50030BAA6E0BC0A9FFA69E6C
:10C53800A69CA68000F000F0A8501200AE0E0001E4
:10C54800806FFE0E816FB7EC62F089900101B46BC9
:10C5580012000B6E03D005EC63F004009EA8FBD715
:10C568000BC0ADFF1200820E596E80C018F081C05A
:10C5780019F0590E1A6EC3EF24F00B6E03D005ECB8
:10C5880063F004009EA8FBD70BC0ADFF1200928891
:10C5980080A803D0010E0B6E01D00B6A0B5012005D
:10C5A8000B6E0BC0C9FFC7B0FED7C7A0FED7C950D6
:10C5B80012000B6E02D0898889980B060B28FBE1C4
:10C5C8001200C968C7B0FED7C7A0FED7C95012006D
:10C5D8000B6E0B5001E0010C745012005EC40BF09E
:10C5E8005FC40CF0120001EC63F0E5EF62F089988B
:10C5F8009298120089989288120082801200829084
:06C608001200120001E720
:10F33800004F4B004449534B5F455252004E4F54C7
:10F348005F5245414459004E4F5F46494C45004E77
:10F358004F545F4F50454E4544004E4F545F454E05
:10F3680041424C4544004E4F5F46494C455F535916
:10F378005354454D000020000D0A20253258202501
:10F3880032582025327320253273202532732025E8
:10F3980032732025327320253273202532732025BD
:10F3A80032732025347320253473202534732025A7
:10F3B8003473202534732025347320253473202595
:10F3C800347320000D0A2530325825303258205326
:10F3D8005338303A53657420537461747573206DD3
:10F3E80061736B2025582025582025582025582042
:10F3F800255820255820255820255820000D0A2555
:10F408003032582530325820535338303A20496E1C
:10F418006372656D656E743A205365656B696E67D6
:10F4280020746F20256C752028256C582920000D24
:10F438000A48504469736B204D6B20494920283194
:10F448003846343632302920257320257320257319
:10F45800205374617274696E672E2E2E0D0A000D8A
:10F468000A2530325825303258205265636569764E
:10F47800656420525443206279746573202532589C
:10F4880020253258202532582025325820000D0AD0
:10F49800253032582530325820414D3A556E627524
:10F4A800666620726420632F682F733A2025642FC4
:10F4B80025642F256420733A256C6420000D0A25E5
:10F4C800303258253032582053656E64696E672093
:10F4D80052544320627974657320253258202532AE
:10F4E80058202532582025325820000D0A25303260
:10F4F80058253032582053533830783A5365656B65
:10F508003A205365656B696E6720746F20256C75AA
:10F518002028256C582920000D0A2530325825301E
:10F52800325820414D3A4275666620777220632F23
:10F53800682F733A2025642F25642F256420733A99
:10F54800256C64000D0A2530325825303258205376
:10F558005338303A4275666620777220256C6420ED
:10F56800627974657320727820000D0A52656365AC
:10F578006976656420525443206279746573202546
:10F58800325820253258202532582025325820005C
:10F598000D0A414D3A556E62756666207772206392
:10F5A8002F682F733A2025642F25642F2564207334
:10F5B8003A256C6420000D0A547269656420746FE2
:10F5C8002074616C6B207768696C7374206E6F743B
:10F5D80020616464726573736564000D0A53656E17
:10F5E80064696E67205254432062797465732025DC
:10F5F80032582025325820253258202532582000EC
:10F608000D0A5365656B20657272202564203E20C3
:10F6180025642C202564203E2025642C2025642088
:10F628003E202564000D0A414D3A427566662072F7
:10F638006420632F682F733A2025642F25642F25B3
:10F648006420733A256C6420000D0A253032582551
:10F6580030325820313A526561642072746E202528
:10F66800582C202564207265616420000D0A25301D
:10F678003258253032582053533830783A57726907
:10F68800746520256C642028256C582920000D0AF3
:10F6980025303258253032582053533830783A5371
:10F6A80074617475732C20756E697420256420004C
:10F6B8000D0A526420752025642072746E2025641A
:10F6C8002C20256420627974657320726561640D4D
:10F6D8000A000D0A25303258253032582053533845
:10F6E80030783A5265616420256C752028256C585D
:10F6F8002920000D0A25303258253032582053531E
:10F7080038303A53657420616464726573732025D8
:10F718006C5820000D0A25303258253032582053B5
:10F728005338303A436820696E6420436C656172CF
:10F7380020256420000D0A4D617820566563746F9A
:10F7480072206469736B20256420256C6420282549
:10F758006C582920000D0A2530325825303258209F
:10F7680053533830783A5374617475735B25645D0C
:10F7780020255820000D0A253032582530325820CF
:10F78800535338303A5365742072656C65617365FC
:10F7980020255820000D0A253032582530325820AF
:10F7A800535338303A536574206C656E677468201B
:10F7B800256C5820000D0A25303258253032582043
:10F7C800535338303A416D69676F20436C656172F5
:10F7D80020256420000D0A25303258253032582063
:10F7E800535338303A53657420766F6C756D6520C5
:10F7F800256420000D0A2530325825303258205310
:10F808005338303A466F726D617420706172616D61
:10F818007320000D0A2530325825303258205353B2
:10F8280038303A5270742051535441542025642082
:10F83800000D0A44736B73656C2069732025642C72
:10F84800206E756D62657220697320256420000D35
:10F858000A414D3A5365656B3A202564202564209A
:10F8680025642025642C20733A256C64000D0A2534
:10F878003032582530325820535338303A53657453
:10F8880020756E697420256420000D0A25303258D1
:10F89800253032582053533830783A4465736372B0
:10F8A800207520256420000D0A5265616420727459
:10F8B8006E2025582C202564206279746573207287
:10F8C800656164000D253032582530325820566560
:10F8D80063746F7220256C642028256C58292000D9
:10F8E8000D0A253032582530325820535338303AD3
:10F8F800556E6B6E6F776E20255820000D0A2530E7
:10F9080032582530325820535338303A43616E63A9
:10F91800656C20256420000D0A25303258253032C8
:10F928005820535338303A496E6974206469736BB0
:10F9380020000D0A253032582530325820535338CC
:10F94800303A52712073746174757320000D0A4146
:10F958004D3A556E6275666620777220256420627E
:10F9680079746573207278000D0A25303258253075
:10F97800325820535338303A44657363726962656C
:10F9880020000D0A2530325825303258205353387C
:10F9980030783A466D74206F70747300466F756ED8
:10F9A8006420616E205254432066696C652061743E
:10F9B8002025580D0A004C6F6F6B696E6720666FC3
:10F9C8007220616E205254432066696C650D0A00EE
:10F9D8000D0A5573696E67206469736B2067656FDC
:10F9E8006D6574727920257320000D0A414D3A2007
:10F9F800496E63723A2025642025642025642025F9
:10FA0800642C20000D0A2530325825303258202524
:10FA18006C642062797465732073656E74000D0AD6
:10FA2800577269746520256C642028256C58292034
:10FA3800733A256C5520002530325825303258202D
:10FA4800256C642062797465732073656E74200078
:10FA580046696E6446696C65206661696C656420F8
:10FA68007365617263680D0A000D0A414D3A42756B
:10FA78006666207772202564206279746573207227
:10FA880078000D0A475049422072633A25642025C0
:10FA9800642062797465730D0A000D0A25303258A6
:10FAA800253032582053533830783A436C656172A8
:10FAB80020000D0A57726974655F736563746F720D
:10FAC80073206661696C202564000D0A4469736BB4
:10FAD8002073656C656374206E756D626572202590
:10FAE80064000D0A5365656B20746F20256C6420D3
:10FAF8006661696C6564202564000D0A25303258FA
:10FB08002530325820535338303A5772697465207B
:10FB1800000D0A4F70656E696E67206578697374A9
:10FB2800696E6720257320000D0A476F7420256CC5
:10FB38007520202D20726573657474696E67005393
:10FB480065656B696E6720746F20736563746F7287
:10FB58002025580D0A0046696E6446696C65206662
:10FB680061696C656420726561640D0A000D0A5351
:10FB780065656B696E6720746F20256C6420282585
:10FB88006C5829000D0A2530325825303258205338
:10FB98005338303A5265616420000D0A25303258D6
:10FBA8002530325820535338303A4E4F5020000DEC
:10FBB8000A5472616E2045786563202558202020FC
:10FBC8002020004469736B206368616E67653A2082
:10FBD800256420200D0A000D0A4469736B205374B4
:10FBE800617475733A2025582C20000D0A576169F5
:10FBF80074696E6720666F72206361726420000DFD
:10FC08000A414D3A53656E642073746174757320AC
:10FC18002564000D566563746F7220256C64202876
:10FC2800256C582920000D0A46696C65202573202B
:10FC38006973206F70656E20000D0A57726F7465C6
:10FC4800206469736B6E6F3A202564002041544E1E
:10FC58002061737365727465642031202564000D1A
:10FC68000A52656164206265796F6E6420656E640E
:10FC7800000D0A5365656B206265796F6E642065B7
:10FC88006E64000D0A4F70656E696E67206E657749
:10FC980020257320000D0A20256C64206279746584
:10FCA800732073656E74000D0A46696C65202558CB
:10FCB80020697320257320000D0A4469736B202581
:10FCC8005820697320257320004E6F742061204CE2
:10FCD8004946206469736B0D0A000D0A25303258B5
:10FCE80025303258204578697420000D0A52656124
:10FCF80064696E67205254430D0A000D0A416D690C
:10FD0800676F2039313231440D0A000D0A53532FE1
:10FD180038302039313232440D0A000D0A44736BF1
:10FD280073656C20697320256420000D0A52656193
:10FD380064202564206279746573000D0A48737421
:10FD480020627974657332202564000D0A57726940
:10FD58007465206661696C202564000D0A53533868
:10FD6800306578656320256420000D0A4F70656E44
:10FD7800696E672025732020000D0A446562756747
:10FD880020697320256420000D0A50726F746F205B
:10FD9800697320256420000D0A5265616420636F31
:10FDA8006E66696720000D0A46696C656E616D654F
:10FDB8002025732000566563746F722069732025AF
:10FDC800580D0A00222A2B2C3A3B3C3D3E3F5B5DF6
:10FDD8007C7F000D0A48737420627974657320254E
:10FDE80064000D0A56616C75653A2025580D0A00A5
:10FDF80072633D25752046525F25730D0A000D0A72
:10FE08005374723E25733C200D0A20000D0A52657A
:10FE1800636569766532353620000D0A466F726D66
:10FE2800617474696E6720000D0A4E6F20636172F9
:10FE380064202564002F6C6966646174612E6269B0
:10FE48006E000D0A25732025582025580D0A007BC1
:10FE5800505025642025642025647D002A2A2056D8
:10FE68006572696679202A2A000D0A7362797465B9
:10FE78007331202564000D0A4D6F756E74696E67C5
:10FE880020004A616E2031302032303231000D0AB4
:10FE98004B3A257320563A2573000D0A414D3A44D2
:10FEA800534A202564000D0A414D3A57616B657528
:10FEB80070004C6F6164696E672E2E2E0068706446
:10FEC80069736B2E63666700436F6E74726F6C6C38
:10FED80065720020255820772041544E20000D0AD5
:10FEE800414D3A436C656172005B535251206F6615
:10FEF800665D00466D742065786974200031363A75
:10FF080035323A3133005B2532582025645D005B79
:10FF1800535251206F6E5D0048504469736B200046
:10FF28004E6F2063617264002D3E202558200044E6
:10FF3800534B53454C004E414D45255800444953B9
:10FF48004B255800566F6C756D65005458446174A4
:10FF5800610072633D256420005258446174610059
:10FF68005258627566003C69643E2000444542551B
:10FF7800470050524F544F00526561647900202564
:10FF8800303258007B4552527D000D0A44534A00D6
:10FF98005B4D4C415D005B4D54415D00302E313668
:10FFA80000556E6974004946432000454F492000BA
:10FFB80052454E2000535251200044415620004ED5
:10FFC800444143004E5246440052544300202558B1
:10FFD8000025325800207C20004430004431004481
:10FFE800320044330044340044350044360044377A
:07FFF800002563002B00004F
:020000040020DA
:08000000FFFFFFFFFFFFFFFF00
:020000040030CA
:0E000000FF06191EFF8181FF0FC00FE00F40A9
:00000001FF
